:020000040800F2
:10000000E04400109D010008415700083D2500080C
:100010003D57000853120008056B0008000000005F
:10002000000000000000000000000000B55E0008B5
:100030002D13000800000000FD5B0008AB5F000806
:10004000B7010008B7010008B7010008B7010008B0
:10005000B7010008B701000831130008B701000814
:10006000B7010008B7010008B7010008C91200086D
:10007000B7010008B7010008B7010008D512000851
:10008000B7010008B7010008650F0008B7010008B4
:10009000B7010008B7010008B7010008B701000860
:1000A000B701000891610008E1600008B70100088D
:1000B000B7010008B7010008B7010008B701000840
:1000C000B7010008B7010008B7010008B701000830
:1000D000B7010008D56A0008B7010008B701000899
:1000E000B7010008B7010008B7010008B701000810
:1000F000B7010008B7010008B7010008B701000800
:10010000B7010008B7010008B7010008B7010008EF
:10011000B7010008C56A00082D620008ED620008FA
:10012000ED120008FD120008B7010008B701000831
:10013000B7010008B7010008B7010008B7010008BF
:10014000B7010008B7010008B7010008B7010008AF
:100150000D1300081D130008B7010008B7010008BF
:10016000B7010008B7010008B7010008B70100088F
:10017000B7010008B7010008B7010008000000003F
:10018000B7010008B7010008DFF80CD000F0B8FD97
:10019000004800474D580208E044001006488047D8
:1001A00006480047FEE7FEE7FEE7FEE7FEE7FEE75C
:1001B000FEE7FEE7FEE7FEE7DD60000889010008D4
:1001C0000649074A0868504343F239021044086060
:1001D0004008704701490860704700006C02001039
:1001E0006D4EC64110B5431A934209D28318881840
:1001F00003E010F8011D03F8011D521EF9D210BDD5
:1002000040EA01039B0703D009E008C9121F08C098
:10021000042AFAD203E011F8013B00F8013B521E18
:10022000F9D210BDD2B201E000F8012B491EFBD279
:1002300070470022F6E710B513460A4604461946F1
:10024000FFF7F0FF204610BD10B5044604E00B7820
:1002500000F8013B03B1491C521EF8D2204610BDE4
:10026000421C10F8011B0029FBD1801A704710B501
:10027000002200E0521C835C8C5CA34201D1002B65
:10028000F8D1D8B2E1B2401A10BD30B50546002011
:10029000034600E05B1C934205D2EC5CC85C201A6C
:1002A00001D1002CF6D130BDF0B480EA0102D40FA8
:1002B0004200B2EB410F02D20246084611464A0004
:1002C00042D0C30DDDB2C1F3C752AD1A202D35DACD
:1002D000C1F3160141F4000204B15242C5F12006F7
:1002E00002FA06F12A411044B3EBD05F23D0C4B127
:1002F000012DA0EBC35009DCF0BC4FF0004202EA34
:10030000C352DBB200F5000000F0D6BB400000F1A4
:10031000807000EBC350A0F1807040EAD1704900BA
:1003200009E0490841EAC071A0EBC35000F50000A4
:10033000400800EBC350F0BC00F0B5BB61420122A5
:1003400002EB4101001BF6E7F0BC704781F0004171
:10035000AAE780F00040A7E780EA010210B502F0AA
:100360000043400022D04A001FD0010E01EB126171
:10037000C0F35600C2F3560240F4000042F40002FB
:10038000A0FB022000047F39140400D0401C50EA76
:10039000124001D44000491EC2B20C0604EBD0103A
:1003A000401C4008802A02D003E0002010BD20F04D
:1003B0000100002900DA0020184310BD30B480EAA3
:1003C000010202F0004530F0004221F0004013D05D
:1003D00090B1C30DD40DC2F31601C0F31600E41A98
:1003E00041F4000140F400027D34914201D3641CC9
:1003F00000E04900002C02DA30BC002070474FF4C6
:1004000000000023914201D3891A034340084FEAB8
:100410004101F7D151B1914202D14FF0004105E0C5
:1004200002D24FF0010101E06FF0010103EBC45073
:10043000284430BC00F037BB2DE9FE4F804681EAEE
:100440000300C00F0C46009021F0004123F000454E
:10045000B8EB0200A94105D24046214690461C4611
:100460000B46024623F00040104347D0270DC7F348
:100470000A00C3F30A510290401A019040286BDA37
:10048000C3F3130040F4801B0098924620B1002370
:10049000D2EB030A63EB0B0B01985946C0F1400203
:1004A000504600F0CFFA06460D4650465946019A8E
:1004B00000F0E7FA10EB08006141002487EA1152CE
:1004C00084EAE7731A4340D0009A62B3019A012A82
:1004D0004FEA075215DC001B61EB02014FF00042AE
:1004E00002EA0752CDE90042001C41F58011324674
:1004F0002B4600F077FB03B000F045B8404621469C
:10050000F9E7001B61EB0201001C41F580130018A4
:100510005B412018A2F5001747EB030140EAD570B4
:10052000B6196D4111E06D084FEA360645EAC0750F
:100530004FEA0752001B61EB0201001C41F58011DC
:1005400049084FEA30000019514132462B4603B0AA
:1005500000F01CB800F037BB0098012240000023D7
:10056000D0EB020263EBE073009821464FEAE0749F
:10057000B8EB000061EB0401E9E783F000435BE7BF
:1005800081F0004158E730BCBDE8C08F30BCBDE809
:10059000C04FFFF7DFBF2DE9FE4F81EA030404F0EF
:1005A000004421F0004100944FF0000B23F0004381
:1005B00050EA01045ED052EA03045BD0C3F30A544C
:1005C000C1F30A552C44A4F2F3340194A0FB025465
:1005D000C1F3130141F48011C3F3130343F48013F7
:1005E00001FB024400FB034E840A970A44EA81544B
:1005F00047EA8357A4FB076802958D0A05FB078528
:100600004FEA932C04FB0C542705029D4FEA065831
:1006100047EA1637B5EB08056EEB070C870E920E0E
:1006200047EA811742EA8312A7FB0201B6EB0B01EE
:1006300064EB00042B0D43EA0C335E1844EB1C50B2
:10064000DA465146E7FB0201C5F313044FEA0B33C8
:1006500043EA14534FEA0432019C43EA0603A4F12F
:100660000C040294009CCDE900B400F0BBFA03B086
:1006700000F003B800200146F9E730BCBDE8C08FA8
:100680002DE9F04D81EA030404F0004B21F0004510
:1006900014464FF0000A23F0004150EA050220D032
:1006A00054EA01021DD0C5F30A570246C5F31303ED
:1006B000C1F31300C1F30A5640F4801543F48013CC
:1006C000A7EB0608101BD64608F2FD3873EB0500B1
:1006D00002D308F1010801E092185B41B8F1000F64
:1006E00003DA00200146BDE8F08D00204FF48011B0
:1006F000064684460EE0171B73EB050705D3121B55
:1007000063EB050306434CEA010C49084FEA30004D
:1007100092185B4150EA0107EDD152EA030012D072
:1007200082EA040083EA0501084305D0101BAB41AF
:1007300006D20122002306E000224FF0004302E02F
:100740006FF0010253101AEB06004CEB085110EB4E
:100750000A0041EB0B01BDE8F04D00F034BA70B572
:1007600021F0004303430CD0C1F30A550024D5EB1C
:10077000040564EB0403D617AD1AB34102DB002075
:10078000014670BD201841EB025170BD002801DB0D
:10079000C0F10040002901DBC1F10041814201D2DA
:1007A0000120704700207047C10F80EAE0700844C4
:1007B000CA079623002100F07FB996230022114634
:1007C00000F07AB90EB5C10F80EAE0700844CA079C
:1007D000002140F233438DE80E000A460B4600F03C
:1007E00001FA03B000BD0EB540F233410291002181
:1007F000CDE900110A460B4600F0F4F903B000BD44
:1008000000F0004220F00040C10DC0F3160040F49B
:1008100000007F2901DA00207047962903DCC1F12E
:100820009601C84001E096398840002AF4D0404241
:10083000704720F00040C10DC0F3160040F40000E6
:100840007F2901DA00207047962903DCC1F1960167
:10085000C840704796398840704770B5C1F30A5256
:1008600001F000450024C1F3130140F2FF3341F4CD
:1008700080119A4201DA002070BD40F233439A425F
:10088000A2F2334203DC524200F0EBF800E0904069
:100890002C43F1D0404270BDC1F30A5210B5C1F3F0
:1008A000130140F2FF3341F480119A4201DA002033
:1008B00010BD40F233439A42A2F2334203DC52426B
:1008C00000F0CFF810BD904010BD00F0004230F0B5
:1008D00000400AD0C10D01F56071C0F3160042EA74
:1008E0000151C2084007114370470020014670477C
:1008F00030B5041E71F1000404DB4FF000444042A7
:1009000064EB0101141E73F1000405DB1C464FF07B
:100910000043524263EB04038B4208BF824230BD66
:1009200030B5041E71F1000404DB4FF00044404276
:1009300064EB0101141E73F1000405DB1C464FF04B
:100940000043524263EB0403994208BF904230BD1A
:1009500001F0004330B421F0004150EA010206D01A
:100960000A0DA2F56072C1F31301002A02DC30BC4B
:1009700000207047440F44EAC104C100E01830BCB5
:1009800000EBC25000F08FB8002801DBC0F100403E
:10099000002901DBC1F1004181427047002801DBE1
:1009A000C0F10040002901DBC1F1004188427047DD
:1009B00030B50B46014600202022012409E021FA2F
:1009C00002F59D4205D303FA02F5491B04FA02F52C
:1009D0002844151EA2F10102F1DC30BD2DE9F05FC3
:1009E0000546002092469B4688460646814640249E
:1009F0001BE0284641464746224600F032F853465F
:100A00005A46C01A914110D311461846224600F0AA
:100A100019F82D1A67EB01084F46224601200021E4
:100A200000F010F817EB00094E41201EA4F101045C
:100A3000DFDC484631462A46434600F000B830BC69
:100A4000BDE8C09F202A04DB203A00FA02F1002012
:100A500070479140C2F1200320FA03F319439040FC
:100A60007047202A04DB203A21FA02F00021704767
:100A700021FA02F3D040C2F1200291400843194606
:100A80007047202A06DBCB17203A41FA02F043EAEE
:100A9000E07306E041FA02F3D040C2F12002914037
:100AA0000843194670470029A8BF7047401C4900F9
:100AB00008BF20F00100704710B4B0FA80FC00FAC3
:100AC0000CF050EA010404BF10BC704749B1CCF1EE
:100AD000200421FA04F411FA0CF118BF012121437A
:100AE0000843A3EB0C01CB1D4FEA00614FEA102035
:100AF00042BF002010BC704700EBC35010440029D7
:100B0000A4BF10BC7047401C490008BF20F0010082
:100B100010BC7047420005D0C0F3C7525242914208
:100B200001DC0020704700EBC1507047F0B4002892
:100B300002DCF0BC00207047C0F3C751C0F31600C0
:100B400040F40000CA0701D14000491E3F2202EBD9
:100B50006105002211464FF4000626FA01F3134402
:100B6000D418844201D8001B1A464000491C17299A
:100B7000F3DD5100814202D24FF0FF3100E000214D
:100B800002EBC550F0BCFFF78EBF10B541000CD092
:100B9000C0F3C751962908DC7E2909DC06DB410237
:100BA00004D000F0004040F07E5010BD002010BD89
:100BB000C1F19604C4F1200100FA01F1E040FFF711
:100BC00072FFA04010BD10B5141E73F1000408DAC6
:100BD000401C41F1000192185B411A4301D120F001
:100BE000010010BD2DE9F04D92469B4611B1B1FABE
:100BF00081F202E0B0FA80F220329046FFF722FF45
:100C000004460F4640EA0A0041EA0B0153465A46A1
:100C1000084313D0114653EA010019D0C8F140022D
:100C20005046FFF71EFF05460E46504659464246BF
:100C3000FFF708FF084305D0012004E020463946AD
:100C4000BDE8F08D0020054346EAE0762C433743AB
:100C50000A986305E40AA0EB08000022FD0A44EAB2
:100C600047540A3002D500200146E9E70105101972
:100C70006941DDE9084500196941BDE8F04DA2E789
:100C8000C1F30A52C1F3130140F2FF3341F4801162
:100C90009A4202DA00200146704740F233439A42FA
:100CA000A2F2334202DC5242FFF7DBBEFFF7CABEBC
:100CB00010B500F0004420F00040C20DC0F3160053
:100CC00040F400007F2A07DA7D2A00DA7D22763A96
:100CD00000FA02F1002008E0962A09DCA2F1760170
:100CE00000FA01F1C2F19602D040FFF7DCFE01E00C
:100CF000963A9040002C00D0404210BD0020704732
:100D0000064C074D06E0E06840F0010394E8070058
:100D100098471034AC42F6D3FFF73AFAE45005088E
:100D2000245105082DE9F04D00231A461B1A8A416B
:100D300003DB00200146BDE8F08DC1F30A52C1F388
:100D4000130141F480154FF0000BD10702D10018B8
:100D50006D41521E0027044640F2FF11384601EB58
:100D6000620A3E468046024600204FF48011FFF79B
:100D700078FEC2197141BB1846EB0100B4EB030CBD
:100D800075EB000C04D3E41A65EB000517460E461C
:100D9000241908F101006D4180463428E3DDF9197A
:100DA00046EB0600091BA84103D24FF0FF32134661
:100DB00001E0002213461BEB070046EB0A51BDE899
:100DC000F04DFFF700BF70B58C1810F8015B15F0FF
:100DD000070301D110F8013B2A1106D110F8012BAD
:100DE00003E010F8016B01F8016B5B1EF9D12B07D2
:100DF00005D40023521E0DD401F8013BFAE710F888
:100E0000013BCB1A921C03E013F8015B01F8015B74
:100E1000521EF9D5A142D8D3002070BDF0B581B0E3
:100E20004FF68311C3F62261FFF796FA4FF07A511D
:100E3000FFF73AFA0446FFF7E3FC05462046002197
:100E40000027FFF7A3FC002818BF013D2846FFF745
:100E5000ABFC01462046FFF779FA4FF08841FFF7D7
:100E60007BFA0546FFF7E5FC044628464FF044416F
:100E7000FFF71AFA0646B7EB542F0CBF2E46002494
:100E80002046FFF79AFC01463046FFF75FFA054619
:100E90004FF07E502946FFF759FA44F6E007C0F6B6
:100EA000050757F82410FFF757FA064607EB8400AA
:100EB00041682846FFF750FA01463046FFF7F4F93B
:100EC00001B0F0BDF0B581B04FF68311C3F62261D9
:100ED000FFF742FA0446FFF793FC0546204600213F
:100EE0000027FFF753FC002818BF013D2846FFF7F5
:100EF0005BFC01462046FFF729FA4FF08841FFF7D7
:100F00002BFA0546FFF795FC044628464FF044416E
:100F1000FFF7CAF90646B7EB542F0CBF2E46002444
:100F20002046FFF74AFC01463046FFF70FFA054618
:100F30004FF07E502946FFF709FA44F6E007C0F665
:100F4000050757F82410FFF707FA064607EB840059
:100F500041682846FFF700FA01463046FFF7A4F93A
:100F600001B0F0BD10B500200AF09EFC10BD30B5F8
:100F700089B005460C461022002105A808F087FD1F
:100F8000224605A905A80BF0FFFA9DF8140000F011
:100F90008000E8B100BF00200AE005A9095C4A0012
:100FA00005AB411C595C42EAE11105AA1154401CF1
:100FB0000F28F2DB9DF823104906090E8DF8231047
:100FC00000BF9DF8230080F087008DF8230016E015
:100FD00000BF00200AE005A9095C4A0005AB411CDE
:100FE000595C42EAE11105AA1154401C0F28F2DBBA
:100FF0009DF823104906090E8DF8231000BFD4F880
:10100000140110280FD100BF002009E004F20111E3
:10101000095C05AA125C514004F201121154401CF3
:101020001028F3DB5DE09DF8140000F08000E8B1CB
:1010300000BF00200AE005A9095C4A0005AB411C7D
:10104000595C42EAE11105AA1154401C0F28F2DB59
:101050009DF823104906090E8DF8231000BF9DF856
:10106000230080F087008DF8230016E000BF0020E9
:101070000AE005A9095C4A0005AB411C595C42EA3B
:10108000E11105AA1154401C0F28F2DB9DF8231032
:101090004906090E8DF8231000BF802104F20110CB
:1010A000D4F81421815405E0002104F20110D4F891
:1010B00014218154D4F81401401CC4F814011028E0
:1010C000F2D300BF002009E004F20111095C05AA77
:1010D000125C514004F201121154401C1028F3DB41
:1010E00000BF00BF00200AE004F1F101095C04F236
:1010F0000112125C514004F1F1021154401C1028FD
:10110000F2DB00BF102204F1F10101A808F0ADFBF1
:101110002246294601A80BF037FA1022002105A823
:1011200008F0B5FC09B030BD10B50446102200210E
:1011300004F1F10008F0ABFC0020C4F81401F02227
:101140000021204608F0A3FC10BD70B504460D46F2
:101150002246102128460BF045FA70BD2DE9FF41CB
:1011600004460F461546D4F8140100283BD0D4F8A5
:101170001401C0F11000A84204D2D4F81401C0F147
:10118000100000E028460646B2B204F20111D4F87D
:1011900014315818394608F068FBD4F8140130446B
:1011A000C4F81401D4F81401102801D3B54201D1B8
:1011B00000F048B800BF00200AE004F1F101095C2A
:1011C00004F20112125C514004F1F1021154401C6E
:1011D0001028F2DB00BF224604F1F10108460BF0B3
:1011E000D3F93744AD1B21E000BF002008E004F133
:1011F000F101095C3A5C514004F1F1021154401CC8
:101200001028F4DB00BF102204F1F101684608F059
:101210002CFB2246694668460BF0B6F91022694657
:1012200004F1F10008F021FB1037103D102DDBD840
:10123000AAB2394604F2011008F017FBC4F81451A1
:1012400000BFB5E703BCBDE8FC81002800DC4042DC
:10125000704700BFFEE7000010B5024600200AE01C
:1012600012F8014B84EA2023DBB2054C34F813302A
:1012700083EA002398B20B1EA1F10101F0DC10BD3E
:101280007C18050870B5054608263146002031F067
:10129000E3F80446256000206060204670BD000031
:1012A00070B504460D4600BF44B9064805800320CA
:1012B00023F086FE01E000BF00BFFCE700BF012075
:1012C00070BD0000F07F001010B500200AF0C8FAD1
:1012D00010BD000010B5044A12685068024A126836
:1012E0005268116D884710BD5002001010B50249B8
:1012F00048683DF0C3F810BD0000001010B5024969
:1013000048683DF0BBF810BD0000001010B5024960
:1013100008683DF0B3F810BD0000001010B5024998
:1013200008683DF0ABF810BD0000001070470000E9
:1013300010B50120094909680140814200D100E04F
:10134000002149B1012001F0E9FE054908683DF09E
:101350001EFB012001F0E2FE10BD0000140401405C
:10136000000000102DE9F04105460E4614463146B6
:101370002846FFF709FB03D84FF07E50BDE8F08107
:1013800031462846FFF70AFB12D221462846FFF7CE
:10139000FBFA0DD831462046FEF7D8FF0746214616
:1013A0002846FEF7D6FF80463946FFF707F8E5E7FF
:1013B00021462846FFF7F2FA01D20020DEE700209E
:1013C000DCE72DE9F04105460E4614463146284635
:1013D000FFF7DAFA02D80020BDE8F081314628464E
:1013E000FFF7DCFA12D221462846FFF7CDFA0DD2DC
:1013F00031462046FEF7AAFF074631462846FEF74B
:10140000A5FF80463946FEF7D9FFE5E72146284685
:10141000FFF7C4FA02D84FF07E50DDE74FF07E5060
:10142000DAE72DE9F04706460F4614461D463946D1
:101430003046FFF7A9FA02D80020BDE8F087394608
:101440003046FFF7ABFA12D221463046FFF79CFA3E
:101450000DD839462046FEF779FF8046394630469A
:10146000FEF774FF81464146FEF7A8FFE5E72146F7
:101470003046FFF793FA12D229463046FFF784FA36
:101480000DD821462846FEF761FF804629463046A2
:10149000FEF75FFF81464146FEF790FFCDE7294604
:1014A0003046FFF77BFA01D20020C6E70020C4E7F0
:1014B00010B504460A280ED00D2C10D008488069BB
:1014C00001682046884707480168002907D0204660
:1014D000BDE810400847BDE8104000F08FBC10BDCB
:1014E0000C300010380400202DE9FF5F8346DDE951
:1014F0000E45984691468A464FF0FF3601274FF435
:10150000B47004F5B47405F5B47503E0A4F5B474CF
:10151000A5F5B4758442F9DA002D65DD5A2C11DA8F
:10152000002C00DA00245A2D01DA284600E05A2067
:10153000CDE90040CDE9027643464A465146584639
:1015400005F072FB5A3C5A3D002D4DDD5A2C14DA41
:10155000002C00DA00245A2D01DA284600E05A2037
:10156000C4F15A01C0F15A008DE8430043464A468F
:1015700051465846039605F057FB5A3C5A3D002DFC
:1015800032DD5A2C12DA002C00DA00245A2D01DA4E
:10159000284600E05A200DF1040C00948CE8C100AC
:1015A00043464A465146584605F03EFB5A3C5A3D92
:1015B000002D19DD5A2C14DA002C00DA00245A2DE3
:1015C00001DA284600E05A20C4F15A01C0F15A005D
:1015D0008DE8830043464A4651465846039705F036
:1015E00023FB5A3C5A3D97E700F000B83FBCBDE8EA
:1015F000C09F00002DE9FF4780463F4816461D4624
:10160000027D0F46012A1CD0A8EB0600791B50EA88
:1016100001036ED0A2F1010906F0F0FE00F5806032
:10162000824600F05CFF00FB09F4504600F05CFFCE
:1016300000FB09F1002C0BDAC4F500708012404267
:1016400009E004B032464046BDE8F04700F05AB821
:1016500004F50074A012002904DAC1F500718912A2
:101660004C4202E001F500718C12002804DD411C9F
:1016700001EBD171491003E000EBD0714910401E1D
:1016800000EBD0704210002C04DD601C00EBD07029
:10169000401003E004EBD4704010641E04EBD473DC
:1016A00008EB0104ADF800403C18ADF80240A8EB8F
:1016B00002045B10B21AADF80440ADF808203144C2
:1016C000FC1AEA1AADF80C102844ADF80A20ADF85F
:1016D0000E000023ADF806401A460421684600F0CB
:1016E00017F93946404605F075FD2946304605F0A4
:1016F00071FD00F003B800000C3000100FBCBDE815
:10170000F08700002DE9F84F0E468046A2EB080452
:101710009D1B994692464FF0000B54EA050017D0E6
:101720002046FFF792FD07462846FFF78EFD8742C9
:101730000ADA20462C4605464046B0460646504644
:10174000CA4681464FF0010B002C07DD204606E01B
:101750003146404600F058B800F070B86042A042F0
:1017600003D064426D42D0464E4604EBD4704FEA3B
:101770006009002D01DAC9F10009DFF888A04FF0F7
:1017800000079AF8160080B131E000BF05FB079012
:1017900090FBF4F03044BBF1000F0AD0DAF83820A7
:1017A00008EB0701526890477F1CA742EEDD00F06E
:1017B00030B8DAF8381008EB07034A6801461846D3
:1017C000F1E700BF05FB079090FBF4F03044009078
:1017D000384606F0FBF948B9BBF1000F0AD0DAF839
:1017E000380008EB07014268009890477F1CA74229
:1017F000E8DDDCE7DAF8381008EB07004A68009902
:10180000F3E700000C30001018BCBDE8E04FFFF714
:10181000A3BF18BCBDE8E08F70B5074C0D46064667
:10182000B4F92810B4F926002B463246FFF7E2FE41
:10183000E684258570BD00000C300010064B1A7D33
:10184000012A05D0521E02EBD272521000F006B8E7
:101850009A6B5268104700000C3000102DE9F05FC1
:101860000646884640F2C32050434FF47A7190FBFD
:10187000F1F702FB02F002EBD27100EB610B2149A0
:101880001446301B896B32447F1C0B6841469847D5
:10189000012533E005FB05F004FB040159451ADD81
:1018A000BC4217DD174B06EB050AA6EB05099B6B3F
:1018B000AAF1010208EB04011B6809F10100984735
:1018C000104BAAF10102A8EB04019B6B09F1010086
:1018D0001B689847641E0B4B3219301B9B6B92465A
:1018E00008EB05011B6881469847064B5246A8EB5A
:1018F00005019B6B48461B6898476D1CBD42C9DDBE
:1019000000F002B80C30001030BCBDE8C09F0000F1
:101910002DE9FF4F40F6FF740F46664283B09B46A9
:10192000814600210BE000BF09EB8100B0F9020005
:10193000A04200DA0446B04200DD0646491CB94226
:10194000F2DB6548006900280DD0B0F90620A2EB53
:101950000B01B14200DA0E46B0F90200A0EB0B0019
:10196000A04200DD0446B1E0DFF870A1002005468A
:10197000CAF8000086E0781E854201DA6B1C00E0A0
:10198000002309EB850C09EB8302BCF90200B2F9D4
:101990000210A04242D1A14214D139F92330059A54
:1019A00039F9251003EB020C4B4A0598926B084459
:1019B00004EB0B011368604501DA624629E0024638
:1019C000604626E02846A4464FF000087A1E0BE049
:1019D00008B1401E00E0781E09EB8003B3F9023025
:1019E000634504D108F101089045F1DB2346A34289
:1019F00047D01A1B39F92500A1EB040C059B92EA8C
:101A00000C0F08D4344A184404EB0B01926B136892
:101A10000246984735E005F077F832E0A14230D031
:101A200001DBA04203DDA0422BDBA14229DCE04622
:101A300088420ADC0346A04223DC0846A14220DBA0
:101A4000B8F900C0B2F9001008E00B46A14218DC5A
:101A5000A04216DBB2F900C0B8F90010E21AA1EBFF
:101A60000C0151430029A0EB030202DD01EB6201EE
:101A700002E0A1EB6201491CC01A91FBF0F0604446
:101A8000C9E76D1CBD42FFF676AF0598009004EBE8
:101A90000B00019000208046054612E01049B8F185
:101AA000000F31F915A008D0009901EB0A02084493
:101AB0000949896B0B680199984788F001085046DD
:101AC0006D1C064909688D42E8DB641CB4427FF74F
:101AD0004BAF07B000F006B80C300010AC0400208B
:101AE000DE54012030BCBDE8C08F0000014AD08424
:101AF000118570470C30001010B5002000F058FB25
:101B00006FF07F4000F056FB012000F069FB0020E1
:101B100000F06EFB002000F073FB002000F04EFB95
:101B2000034800F04DFBBDE81040002000F050BB22
:101B3000F04704082DE9F04FDFF824B191B04FF0E1
:101B4000FF35BBF922200692DBF81830BBF9249050
:101B50009C69A189814206D8E289824203D3471A4F
:101B6000D4F8008012E0D4E9018100296AD00A8803
:101B7000824267D84D88854264D3801A496880B212
:101B800001EB8000B0F90070B0F90250781C59D018
:101B9000187DA17C10FB01FA217CCDE90801BBF97D
:101BA0002A60304600F0DAFFC0B207FB0A810E90CF
:101BB000A27C0127CDF814B00297CDE90321DBF810
:101BC0001800DDE90832C17D807DCDE9000149467C
:101BD000069800F0D9FC681C16D046F0020000F010
:101BE000BDFFA27C05FB0A81CDE9041BCDE9027291
:101BF000DBF81800DDE90832C17D807DCDE9000108
:101C00004946069800F0C0FCDBF818005D46417DAF
:101C1000007D814213D9022E11D086F0040000F01D
:101C20009DFFA869037D427D13FB029102EB09032E
:101C3000857D099A069812FB050200F0F5FD0E98C5
:101C400000F08CFFDBF81830BBF92210627C9B7D22
:101C500012FB0311ABF8221011B000F003B8000022
:101C60000C30001030BCBDE8C08F00000348806914
:101C70008169807D497C11FB00F070470C300010B9
:101C8000022008807047806982898A4202D8C2890E
:101C90008A4207D2806838B102888A4204D84088D4
:101CA000884201D301207047002070472DE9F0439E
:101CB0002B4C054687B0A069B4F92A602946806993
:101CC00000F050F8002848D041680088281A01EB3D
:101CD000C0053046AF7800F041FF814668680121B9
:101CE000CDE90404CDE90217A069C27D817DCDE96B
:101CF0000012037D2A78B4F92410B4F9220000F010
:101D000043FCA069417D027D91421BD9C07D11FB3E
:101D100000F812FB00F7022E14D000F0C8F90646B6
:101D200000F0AAF900F046FAB4F922002978421826
:101D3000B4F9241001EB0803394400F075FD304676
:101D400000F038FA484600F009FFA269B4F9220011
:101D50006978927D11FB0200608407B0BDE8F083D2
:101D60000C30001006E002888A4202D842888A427B
:101D700002D280680028F6D17047000070B5094D86
:101D800004462146A8698069FFF7ECFF002808D0C7
:101D900041680088201A11F83000A969897D10FB7C
:101DA00001F070BD0C30001001200880704710B5A4
:101DB0008069FFF7D7FF002800D0012010BD2DE972
:101DC000F04180461D4616460F46042000F0C6FE30
:101DD00004462B4632463946404600F025FD204653
:101DE000BDE8F04100F0BABEB0F90630B0F9042009
:101DF000B0F90210B0F90000FFF7E1BF00B500F044
:101E00005DF903498A8C10448884088C488400BD9D
:101E10000C3000102DE9FC47060055D000F04EF9BB
:101E2000384C8146B4F9228000F05EF9A18C074657
:101E3000C81BA0843EE000BF47F6FF71304600F0AB
:101E4000F3FA82460146304600F0D4FA054694F88B
:101E50002C0000F0030001283CD0022836D00020DE
:101E6000618C6A46081A6084ADF80000691E084457
:101E7000ADF80400A08CADF80200A9F101010844FE
:101E8000ADF806005146304600F0EEF9BDF802000C
:101E9000A0845146304600F0D1F9064430780A2833
:101EA0001AD00D2818D0BDF800002844608430787E
:101EB00018B1761C30780028BED1A08C3844A0849C
:101EC000A08D20F00300A08500F01EB805EBD570B2
:101ED0004010C5E72846C3E794F82C0000F0030043
:101EE00001280BD0022809D0208C608430780A2881
:101EF000DDD1A18C01EB0900A084D8E7A4F82280F1
:101F0000F4E700000C3000100CBCBDE8F0870000C6
:101F1000024B59849A84FFF77DBF00000C300010FB
:101F20002DE9F04107460A4815460E46B0F92C0047
:101F300040F0020000F05CF904462A46314638467B
:101F4000FFF7E6FF2046BDE8F04100F051B9000080
:101F50000C30001047F6FF73AFF300802DE9FF410E
:101F60001E4617460C46050017D0002C15D00C490C
:101F70006A46D1E90101CDE90001214602A800F03D
:101F800079FA02A800F0BCFD33463A4621462846BD
:101F900000F082F9684600F0B3FD00F003B80000DD
:101FA0000C30001003BCBDE8FC817CB5DDE90645C2
:101FB000CDE90045FFF798FA7CBD000030B40C462F
:101FC0000349896B0B680146204630BC1847000066
:101FD0000C300010FFF70EBB2DE9F0410446B0F9BC
:101FE00002000D461E468119B4F900001746384418
:101FF000FFF77CFD08E000BFB4F90600811934F951
:10200000040F3844FFF708FC6D1E002DF4DCBDE81A
:10201000F0812DE9F04107460D4616461C4600F0BA
:10202000ABFB32462146384600F0A6FB621E691C17
:10203000384600F0DBFB621E691C3046BDE8F0410B
:1020400000F0D4BBB0F90630B0F90420B0F90210AA
:10205000B0F90000FFF7DDBF00F0C8BBFFF7FEBB23
:1020600000F0E2BBB0F90630B0F90420B0F902107C
:10207000B0F90000FFF7F4BF10B500F0F7FBBDE8C2
:10208000104000F004BC0000014989694968084714
:102090000C30001010B5040008D0002020806080B3
:1020A00000F0F0FBA08000F0F0FBE08010BD10B568
:1020B00000F0E2FBBDE8104000F0E9BB0348806996
:1020C000417DC07D11FB00F0704700000C30001016
:1020D00000F086B910B5044600F0F6F90146204636
:1020E000BDE8104000F086B90949002091F82C1095
:1020F00001F00C020649042A896906D0082A01D099
:102100000C2A01D1087D40087047087D401E7047A9
:102110000C30001070B513492E20087000F0A2F8A2
:10212000114C251D201D256100F092FC0F48A06375
:102130000F482561A06101202075032084F83C0030
:102140006FF0704020636063002000F0BFFC6FF010
:102150007F4000F0E9FC0748E061BDE8704000F016
:10216000B0BB00005C0200100C30001090030508AA
:10217000F0470408C42A0508B0F90220B1F9063076
:102180009A4213DCB1F90220B0F906309A420DDC14
:10219000B0F90020B1F904309A4207DCB1F900101F
:1021A000B0F90400814201DC012070470020704733
:1021B00000F08CBC00F0B8BCFFF79EBC00F0CEBCB9
:1021C000024A916900B19061084670470C300010D6
:1021D00002498A7D88751046704700000C30001057
:1021E00002490A7D08751046704700000C30001047
:1021F000024AB2F92C109085084670470C30001046
:10220000024AB2F92A105085084670470C30001077
:102210002DE9F041084E04460568F069016828463A
:1022200088470746F0694168284688472844206067
:102230003846BDE8F08100000C3000102DE9F04177
:102240000C4606460025064F05E0F8694168304611
:10225000884706440544641EF7D22846BDE8F0814D
:102260000C300010704700001CB5094B1B681BB1F7
:102270006A4604F09FFC1CBD1368009352680192EB
:10228000044ABDF800305384BDF802309384EFE770
:10229000600200100C3000102DE9FF4F85B00024C3
:1022A0009A4690460D46A146DDF814B0FFF710FFA0
:1022B000064625B1286800906868019002E06846EB
:1022C000FFF7E8FE18F00C0F02D05546012713E087
:1022D000BDF902402DE02946059800F0A5F8014619
:1022E0006D1A0598FFF7AAFF05990844059005A8FF
:1022F00000F0B4F810B97F1C002DECD108F00C00F0
:10230000042804D0082802D00C2812D105E0BDF919
:10231000060007FB1604641C0BE0BDF90600BDF9BE
:102320000210401A07FB1600401C00EBD07001EBB6
:1023300060045546CDF814B042E02946059800F0F7
:1023400073F807460146ED1B059800F053F818F0A6
:1023500003010ED0012938D002290DD1BDF9041096
:10236000BDF90020891A091A01EBD17102EB610154
:1023700001E0BDF900108946164A401E4844A2F803
:102380002290ADF80C00ADF808909484A019401E7E
:10239000ADF80E00ADF80A4002AA39460598FFF7DD
:1023A00063FF39460598FFF749FF059908440590F2
:1023B000FFF784FE044405A800F050F8002801D17E
:1023C000002DBAD109B000F007B8BDF90410091A00
:1023D000491CD0E70C30001030BCBDE8C08F0000B5
:1023E00003488069017DC07D11FB00F0704700004B
:1023F0000C30001073B50D460098002478B10949DF
:102400008969096949B10A68294690477CBD6846CF
:10241000FFF7FEFEFFF738FE04446D1EF7D5204699
:102420007CBD00000C30001073B50D4600980024F0
:1024300080B109498969096951B14A6829469047BB
:102440007CBD6846FFF7E4FE20B10A2802D0641C78
:10245000AC42F6DB20467CBD0C300010016811F860
:10246000012B12B10A2A02D002E00120704701605C
:102470000020704770B5B1F90040B2F900309C42BD
:1024800000DD23460380B1F90250B2F90240A542B3
:1024900000DD2C464480B1F90460B2F90450AE422C
:1024A00000DC35468580B1F90610B2F9062091426C
:1024B00000DD1146C1809D4201DBA14201DA00200E
:1024C00070BD012070BD00004FF0FF3128B100BF8A
:1024D00010F8012B491C002AFAD10846704700F574
:1024E000806000F001B8000010B50022C0F30B00BE
:1024F000B0F5006F02DD0122A0F50060B0F5806F3D
:1025000001DDC0F5006083110B4C00F03F00C0F10D
:10251000400134F813004843402906D004EB43033C
:10252000C1F140015B8803FB010020308009002AD3
:1025300000D0404210BD00004C03050822F028FDE9
:10254000002022F03DFD03E063210020FEF7A8FEFD
:10255000FAE700F0D5B9FF23C2B2C0F30721C2EBFE
:10256000C202C1EBC1017F327F3192FBF3F291FBDA
:10257000F3F1000C55232A3090FBF3F002EBC1017C
:1025800001EB8010704700002DE9F04F05468DB03B
:102590007548DDF860901A9C00681E4617464FF09B
:1025A000000888B11B9A199BCDE90442CDE902933A
:1025B000DDE91623CDE90023046833463A46284670
:1025C000A0470DB000F0D4B8DDE91602EB1901EB1D
:1025D000060C10435B1EACF1010C012806D0C9F1BA
:1025E00008000590002002910990BAE05F4AB2F914
:1025F0000680A8EB0100002807DD361A002EE0DD7A
:102600004146DDF8648000FB0844B2F90A00ACEBF7
:102610000000002802DD361A002ED2DDB2F90800D3
:10262000181A002800DD3F1AB2F904200020AA423F
:1026300033DD501B3F1A4B46B9F1040F1FD004DCA9
:10264000012B0CD0022B28D111E0484AB2F904200A
:10265000521B2A44082B1AD0102B1ED119E020F04F
:10266000070204EBE004154400F0070015E020F039
:10267000030204EBA004154400F003000DE020F079
:10268000010204EB6004154400F0010005E004447D
:1026900001E004EB400415460020002F91DD1B9A59
:1026A000199BCDE9030248468DE8190033463A46A6
:1026B000284600F027F984E71799029808440B9000
:1026C0002A49401E0090B1F90620824241DC0846AA
:1026D000B0F90A10029881423BDB4FF0000B0395E2
:1026E000DA46089433E000BFBBF1000F05D108982B
:1026F0004FF0080B10F8018B08900599ABEB090B14
:1027000038FA01F008FA09F101F0FF0803D117497E
:10271000097B890715D4154949780A911B9919B184
:10272000095C1248417001E01049487016990398FD
:10273000009B4218521E029900F076F80B490A9845
:102740004870039916980AF1010A08440390BA45A3
:10275000CADB0998401C09900B9802901998044410
:102760000998B042A8DB2CE7600200100C30001082
:1027700030BCBDE8C08F00000D4B30B4B3F906404B
:102780008C4212DCB3F90A408C420EDBB3F90440F0
:10279000844200DD2046B3F90830934200DA1A463D
:1027A000824202DB30BC00F0F9B830BC7047000058
:1027B0000C3000100C4AB2F906308B4213DCB2F92F
:1027C0000A308B420FDBB2F9043083420BDCB2F9E2
:1027D0000830834207DB137BDB0701D000F068B9C8
:1027E000527800F047B970470C3000100D4B30B4F0
:1027F000B3F90440844212DCB3F9084084420EDB92
:10280000B3F906408C4200DD2146B3F90A30934209
:1028100000DA1A468A4202DB30BC00F0DDB830BC78
:10282000704700000C30001030B40F4CB4F9045065
:10283000854200DD2846B4F90850954200DA2A4660
:1028400082420EDBB4F906508D4200DD2946B4F910
:102850000A409C4200DA23468B4202DB30BC00F087
:10286000D9B830BC704700000C3000100148007827
:10287000704700000C30001001484078704700009D
:102880000C3000104FF4C8707047F020704700F013
:10289000E8B800F00701C1EB01220721B2FBF1F219
:1028A000C0F3C203C3EB0323B3FBF1F1C0F3811008
:1028B00000EB001000EB800002EB012101EB004077
:1028C000704710B500F02AF900F0CDF8044600F08A
:1028D0000AF8042000F042F9002000F03FF900F06F
:1028E000C7F8204610BD10B50024E0B2FFF7CFFFB7
:1028F0000146E0B200F0BDF8641CFF2CF5DD10BD10
:10290000FFF729BE2DE9FF4F83B01E46DDE91175A3
:10291000934689460024DDF850A0DDF8408034E07D
:102920004046B8F1010F07D002280FD0042817D075
:10293000B8F1080F27D11DE0CDE900BA04EB090179
:102940002A46139B039804F08DFA1CE0CDE900BAE7
:1029500004EB09012A46139B039804F0E5FA12E000
:10296000CDE900BA04EB09012A46139B039804F051
:1029700063FB08E004EB09015B462A46CDF800A0A2
:10298000039804F0E1FB3D44641CB442C8DB07B08B
:1029900000F000B830BCBDE8C08F00002DE9F04168
:1029A0000C4E04461546307B0F46C00705D10EE09D
:1029B0003946204600F07CF8641CAC42F8DDBDE8E6
:1029C000F08172783946204600F054F8641CAC421D
:1029D000F7DDF4E70C3000102DE9F0410C4E07460E
:1029E0001546307B0C46C00705D10EE0214638461F
:1029F00000F05EF8641CAC42F8DDBDE8F08172784E
:102A00002146384600F036F8641CAC42F7DDF4E7A6
:102A10000C3000102DE9F0411D4616460C460746C5
:102A200005E0324621463846FFF7B8FF641CAC4249
:102A3000F7DDBDE8F08100008AB281B2034810B52D
:102A40000068036B9847C0B210BD00005002001030
:102A500000210180418040F28F118180EF21C180EF
:102A60007047FFF716BF10B522F0C8F8002010BD60
:102A7000704770472DE9F0410C4C05460E46206822
:102A80001746816E884768B1A5F28F15C6F1EF0130
:102A900068428AB2BBB281B22068C46AA446BDE86B
:102AA000F0416047BBB2B2B2A9B2F5E750020010E4
:102AB00070B50C460546FFF7BFFFC2B22146284657
:102AC000BDE87040C2F1FF02FFF7D4BF064910B560
:102AD0004A6B824206D04863FFF73BFDBDE81040D9
:102AE00000F004B810BD00000C30001010B5044612
:102AF000002004F081FB01490C5410BD0C30001083
:102B00001CB504466846FFF7A3FF6A462146024803
:102B1000FFF7B0FC1CBD0000103000100148FFF7AB
:102B200097BF000010300010064910B50A6B8242B2
:102B300006D00863FFF70DFDBDE8104000F004B8B3
:102B400010BD00000C30001010B50446012004F048
:102B500053FB01490C5410BD0C300010064910B550
:102B60000A7B82EA00035B0703D50B784C780C7074
:102B70004B700873104610BD0C300010042101602A
:102B800070471021016070472DE9F04105460C4661
:102B90000026606800B100BF134800F04EF80746F9
:102BA000124800F04AF80743114800F046F807437E
:102BB000AFB9606860B1D4E900010843A168084377
:102BC000E1680843A9680B4A11400843A86007E080
:102BD000A8680849084021680843A86000E0012669
:102BE0003046BDE8F08100000000045000010450B0
:102BF00000020450E030C0FF024611B902F140006B
:102C000000E00148704700000C03045070B5054611
:102C10000C460026284600F010F858B9D4E9000107
:102C20000843A1680843E96844F238029143084325
:102C3000E86000E00126304670BD0146886800F07B
:102C40000100704770B505460C460026606800B16B
:102C500000BF2846FFF7F1FF20BB606870B1A16894
:102C600020680843E1680843216908436169084313
:102C7000E9680E4A11400843E8600BE0E16820680B
:102C800008432169084361690843E968074A11401C
:102C90000843E8606068296B21F00F010143296354
:102CA00000BF00E00126304670BD00003CC0F0FFD0
:102CB000C26822F003020A43C260704770B500F197
:102CC0003004C1F3012504EB85031C6801F01F06E5
:102CD0001F25B540AC4301F01F06C2F38465B54023
:102CE0002C431C6070BD00008168024A1140091D20
:102CF00081607047C0FFFF7F8168034A114041F047
:102D00001001816070470000C0FFFF7F70B500F1C7
:102D10001404C1F3406504EB85031C68C1F3045639
:102D20000725B540AC43C1F3045502FA05F52C4321
:102D30001C6070BD30B5D0F8B030C1F31204A343AD
:102D400002F01805034CEC400C402343C0F8B030AF
:102D500030BD0000FFFF07008268044B1A4001F0FD
:102D6000804343F000431A4382607047C0FFFF3F37
:102D700008B50549896C0143034A91641146896C81
:102D80000140009100BF08BD0010024008B5054990
:102D9000C96C0143034AD1641146C96C01400091DA
:102DA00000BF08BD0010024008B50549C96C0143C9
:102DB000034AD1641146C96C0140009100BF08BDAF
:102DC0000010024008B50549C96C0143034AD164AB
:102DD0001146C96C0140009100BF08BD00100240BF
:102DE00008B50549C96C0143034AD1641146C96C51
:102DF0000140009100BF08BD0010024008B5054920
:102E0000C96C0143034AD1641146C96C0140009169
:102E100000BF08BD0010024008B50549896D014397
:102E2000034A91651146896D0140009100BF08BDBC
:102E30000010024008B50549096E0143034A1166B6
:102E40001146096E0140009100BF08BD001002400C
:102E5000F0B503460024506800B100BF08461D6865
:102E600000F010070126BE40354000F01007012693
:102E7000BE40B54201D1012500E0002585BB506868
:102E800088B1186801F0100640F6F875B540A843FF
:102E9000D2E9005635439668354301F01006B54037
:102EA000284318600BE0186801F01006F825B540BB
:102EB000A84301F010061568B54028431860D86B88
:102EC00001F010060725B540A843D2E90356354363
:102ED0005669354301F01006B5402843D86301E038
:102EE000FFE701242046F0BD4FF480314160704778
:102EF00002214160704708214160704710B50246C9
:102F0000044B5B5CD35823F00103024C645C135107
:102F100010BD0000E8E7040810B50246044B5B5CF6
:102F2000D35823F00103024C645C135110BD000020
:102F30001CE8040810B50246044B5B5CD35843F010
:102F40000103024C645C135110BD0000E8E7040863
:102F500010B50246044B5B5CD35843F00103024CAE
:102F6000645C135110BD00001CE8040810B5024653
:102F7000044B5B5CD35843F00203024C645C135176
:102F800010BD00001CE8040801460868C0F34000BA
:102F9000704701460868C0F3C000704730B503466B
:102FA000044C645C1C5924F440541443014D6D5C82
:102FB0005C5130BD82FF030830B50346054C645CAC
:102FC0001C4464686FF30F041443024D6D5C1D4490
:102FD0006C6030BDE8E7040830B50346054C645C1E
:102FE0001C4464686FF30F041443024D6D5C1D4470
:102FF0006C6030BD1CE8040830B50346054C645CC9
:103000001C5944F21005AC431443024D6D5C5C51F5
:1030100030BD000082FF030810B50346024C645C1B
:103020001C44E26010BD0000E8E7040810B5034648
:10303000024C645C1C44E26010BD00001CE8040803
:1030400030B50346044C645C1C5924F080041443DE
:10305000014D6D5C5C5130BD82FF030830B5034605
:10306000044C645C1C5924F440641443014D6D5CB1
:103070005C5130BD82FF030830B50346044C645CEC
:103080001C5924F020041443014D6D5C5C5130BD8B
:1030900082FF030810B50346024C645C1C44A26026
:1030A00010BD0000E8E7040810B50346024C645C5C
:1030B0001C44A26010BD00001CE8040830B50346A3
:1030C000044C645C1C5924F040041443014D6D5CB5
:1030D0005C5130BD82FF030830B5D0F8A8308D00B8
:1030E0000F24AC40A3438D000F24AC4094FAA4F409
:1030F000B4FA84F402FA04F42343C0F8A83030BDD3
:1031000030B50346044C645C1C5924F440741443E9
:10311000014D6D5C5C5130BD82FF030801490860C0
:103120007047000014040140024909688143014AC4
:103130001160704704040140024909688143014A53
:103140001160704724040140024909688143014A23
:103150001160704700040140024909688143014A37
:103160001160704720040140024909680143014A87
:103170001160704704040140024909680143014A93
:103180001160704724040140024909680143014A63
:10319000116070470C040140024909680143014A6B
:1031A000116070472C040140024909680143014A3B
:1031B0001160704700040140024909680143014A57
:1031C0001160704720040140024909680143014A27
:1031D0001160704708040140024909680143014A2F
:1031E000116070472804014070B504460025207A1C
:1031F00000287BD0206800284BD0607A20B10128BD
:1032000009D0022815D10DE02068FFF78DFF206856
:10321000FFF7CAFF0FE02068FFF796FF2068FFF76F
:10322000A3FF08E02068FFF7BFFF2068FFF79CFFBF
:1032300001E0012500BF00BFA07A50B3A07A0128A9
:1032400004D002280DD003281FD117E0206841497F
:10325000096881433F4A116000BF2068FFF7B4FF4F
:1032600016E020683B49091F09688143394A121F4B
:10327000116000BF2068FFF787FF09E02068FFF7B3
:10328000A3FF2068FFF780FF02E045F0020500BFC2
:1032900000BF606800285AD0607A20B1012809D0A8
:1032A000022815D10DE06068FFF746FF6068FFF760
:1032B00083FF10E06068FFF74FFF6068FFF75CFF77
:1032C00009E06068FFF778FF6068FFF755FF02E0EC
:1032D00045F0040500BF00BFA07A58B3A07A0128CA
:1032E00005D0022810D0032822D11AE023E060681C
:1032F0001849203109688143164A2032116000BF05
:103300006068FFF769FF15E0606812491C310968C1
:103310008143104A1C32116000BF6068FFF73CFF18
:1033200008E06068FFF758FF6068FFF735FF01E0CD
:10333000012500BF0BE02068FFF706FF2068FFF7BC
:10334000F3FE6068FFF708FF6068FFF7F5FE2846A8
:1033500070BD00000C04014000BF2348006940F428
:1033600000402149086100BF00BF0846006940F4E1
:103370008040086100BF00BF0846006940F400704B
:10338000086100BF00BF0846006940F48070086112
:1033900000BF00BF0846006940F08000086100BF20
:1033A00000BF0846006940F04000086100BF00BF50
:1033B0000846006940F02000086100BF00BF0846D1
:1033C000006940F01000086100BF00BF08460069B6
:1033D00040F00800086100BF00BF0846006940F0E7
:1033E0000200086100BF704700200240016941F0FF
:1033F000010101617047416921F004014161704799
:10340000416921F4004141617047416921F00101A6
:1034100041617047416941F0040141617047416970
:1034200041F4004141617047416941F0010141614E
:103430007047000070B50446002508E02846691C66
:103440008DB247F23051884201D9012070BD164833
:1034500000F0CEF80028F1D10025FFF77DFF1CB960
:103460001148FFF7D7FF02E00F48FFF7D8FF0E48DB
:1034700000F070F808E02846691C8DB247F2305120
:10348000884201D90120E1E7074800F0B1F800289F
:10349000F1D100250448FFF7AEFF0348FFF7B0FF66
:1034A00000F05EF80020D1E70020024070B504462D
:1034B000002508E02846691C8DB247F23051884249
:1034C00001D9012070BD224800F092F80028F1D106
:1034D0000025FFF741FF00BF1D48406940F0020092
:1034E0001B49486100BFFF2C06D9A4F58074012157
:1034F000174800F02DF903E00021154800F028F9E5
:1035000000BF1348406964F3CA001149486100BF15
:10351000084600F01FF808E02846691C8DB247F203
:103520003051884201D90120CCE7094800F060F809
:103530000028F1D1002500BF0548406920F00200B5
:103540000349486100BF00F00BF80020BAE7000013
:1035500000200240416941F4803141617047000020
:1035600000BF22480068C0F34020D8B100BF1F4808
:10357000006820F400701D49086000BF00BF0846C5
:10358000006840F4006008600846006820F40060AD
:10359000086000BF00BF0846006840F40070086083
:1035A00000BF00BF00BF11480068C0F38020D8B141
:1035B00000BF0E48006820F480600C49086000BF1E
:1035C00000BF0846006840F4805008600846006864
:1035D00020F48050086000BF00BF0846006840F437
:1035E0008060086000BF00BF7047000000200240FC
:1035F00001460869C0F3004070470146086900F0C1
:1036000001007047416941F00041416170474169E3
:1036100041F00041416170472DE9F04705460E46F3
:1036200014464FF000090027B84614B90020BDE841
:10363000F08709E04046411C1FFA81F847F23051FB
:10364000884201D90120F2E73848FFF7D1FF00286E
:10365000F0D18046FFF780FE3448FFF7E5FEA14633
:103660005BE00021324A11605160082C1BD300201E
:1036700014E02F49D1E90021090241EA1261120246
:103680002B4BC3E90021F91D091A715C9C46DCE94A
:10369000003C1943264BC3E9001C401C0828E8DB0A
:1036A0000837083C1AE0002015E02149D1E9002143
:1036B000090241EA126112021D4BC3E90021A9F17E
:1036C0000101091A715CD3E900C341EA0C011A46F1
:1036D000174B06C3401CA042E7D3002414480068DF
:1036E000286013484068686009E04046411C1FFAA2
:1036F00081F847F23051884201D9012097E70B4801
:10370000FFF776FF0028F0D180460848FFF775FFE5
:1037100010B10648FFF76AFE0835002CA1D1034816
:10372000FFF773FEFFF71CFF002080E70020024038
:103730005803002010B503460AB9002010BD002030
:1037400002E01C5C0C54401C9042FAD30020F5E7C8
:10375000426922F4006242EAC122426170470000DD
:10376000024981600249816070470000230167457A
:10377000AB89EFCD0249816002498160704700004A
:1037800023016745AB89EFCDC26A0A43C262704725
:10379000F0B502460B46186890FAA0F0B0FA80F433
:1037A00087E00120A0401D6805EA000100297FD0C4
:1037B0005868012802D0586802281DD19868956879
:1037C00091FAA1F6B6FA86F677000326BE40B54315
:1037D00091FAA1F6B6FA86F6760000FA06F63543B7
:1037E000956000BFDD6818685668864300FB05F7E2
:1037F0003E43566000BF00BF1869D56891FAA1F634
:10380000B6FA86F677000326BE40B54391FAA1F6D4
:10381000B6FA86F6760000FA06F63543D56000BFA4
:10382000586802282DD1FF2914D85869156A91FAD1
:10383000A1F6B6FA86F6B7000F26BE40B54391FA58
:10384000A1F6B6FA86F6B60000FA06F6354315621A
:1038500000BF16E05869556A0E0A96FAA6F6B6FA3F
:1038600086F6B7000F26BE40B5430E0A96FAA6F6B6
:10387000B6FA86F6B60000FA06F63543556200BF82
:1038800000BF5868156891FAA1F6B6FA86F6770077
:103890000326BE40B54391FAA1F6B6FA86F6760045
:1038A00000FA06F63543156000BF00E000E000BFF7
:1038B000641C1868E04000287FF473AFF0BD024636
:1038C00010690840884201D1012070470020FCE7C0
:1038D000024610690840884201D10120704700204B
:1038E000FCE7024610690840884201D10120704778
:1038F0000020FCE7024610690840884201D10120FF
:1039000070470020FCE781627047816270478162E6
:103910007047816170478161704730B5036891FAE3
:10392000A1F4B4FA84F465000324AC40A34391FAF3
:10393000A1F4B4FA84F4640002FA04F423430360AB
:1039400030BD30B5036891FAA1F4B4FA84F465008F
:103950000324AC40A34391FAA1F4B4FA84F46400C4
:1039600002FA04F42343036030BD30B5036891FAD2
:10397000A1F4B4FA84F465000324AC40A34391FAA3
:10398000A1F4B4FA84F4640002FA04F4234303605B
:1039900030BD30B5036891FAA1F4B4FA84F465003F
:1039A0000324AC40A34391FAA1F4B4FA84F4640074
:1039B00002FA04F42343036030BD30B5036891FA82
:1039C000A1F4B4FA84F465000324AC40A34391FA53
:1039D000A1F4B4FA84F4640002FA04F4234303600B
:1039E00030BD30B5036891FAA1F4B4FA84F46500EF
:1039F0000324AC40A34391FAA1F4B4FA84F4640024
:103A000002FA04F42343036030BD30B5036891FA31
:103A1000A1F4B4FA84F465000324AC40A34391FA02
:103A2000A1F4B4FA84F4640002FA04F423430360BA
:103A300030BD30B5036891FAA1F4B4FA84F465009E
:103A40000324AC40A34391FAA1F4B4FA84F46400D3
:103A500002FA04F42343036030BD30B5036891FAE1
:103A6000A1F4B4FA84F465000324AC40A34391FAB2
:103A7000A1F4B4FA84F4640002FA04F4234303606A
:103A800030BD10B5426921EA020302EA010443EAAB
:103A90000443836110BD000002480068401C0149D6
:103AA00008607047480300204FF47A71B0FBF1F2D0
:103AB000521E4FF0E0235A6100229A6105221A61DA
:103AC00000BF70472DE9F04104460025C02C29D1E4
:103AD000204600F05DF8B0F5400F17D0A0F540008B
:103AE000403820B1402806D0802819D108E002F0E3
:103AF000EFF8054615E000F0EDF800B1224D10E0BA
:103B000000F0F0F808B14FF400450AE002F0E0F8E8
:103B1000074602F0A9F8064602F0B6F8054600E0AE
:103B200000BF00BFB4F5407F2AD1204600F030F836
:103B3000B0F1407F18D01549084430B1B0F5807F0E
:103B400007D0B0F5007F19D108E002F0C1F80546B2
:103B500015E000F0BFF800B10B4D10E000F0C2F826
:103B600008B14FF400450AE002F0B2F8074602F04F
:103B70007BF8064602F088F8054600E000BF00BF6B
:103B80002846BDE8F08100000024F40000FFFFFC9F
:103B9000014603480068084040EA014070470000C1
:103BA000881002402DE9F04104460025032C29D15C
:103BB000204600F085F8B0F5403F17D06FF4403153
:103BC000084420B1012806D0022819D108E002F0EB
:103BD0007FF8054615E000F07DF800B1374D10E0A4
:103BE00000F080F808B14FF400450AE002F070F8E8
:103BF000074602F039F8064602F058F8054600E09C
:103C000000BF57E00C2C29D1204600F059F8B0F540
:103C1000402F17D0A0F54020001F20B1042806D067
:103C2000082819D108E002F053F8054615E000F025
:103C300051F800B1214D10E000F054F808B14FF4F4
:103C400000450AE002F044F8074602F00DF8064687
:103C500002F01AF8054600E000BF2BE0302C29D115
:103C6000204600F02DF8B0F5401F17D0A0F5401009
:103C7000103820B1102806D0202819D108E002F011
:103C800027F8054615E000F025F800B10B4D10E0CF
:103C900000F028F808B14FF400450AE002F018F8E7
:103CA000074601F0E1FF064601F0EEFF054600E0A1
:103CB00000BF00BF2846BDE8F08100000024F400EA
:103CC000014603480068084040EA01407047000090
:103CD0008810024002480068C0F38020704700004E
:103CE0000010024002480068C0F340007047000026
:103CF000901002400248006800F0F0007047000099
:103D0000001002400248006800F470607047000034
:103D10009410024002480068C0F3C00070470000E1
:103D2000001002400248C06800F0700070470000B8
:103D3000001002400248C06800F003007047000015
:103D4000001002400248C068C0F30620704700001F
:103D50000010024002480068C0F340607047000055
:103D6000001002400349896821F003010143014A20
:103D70009160704700100240016821F0400101602D
:103D80007047016821F0400101607047416821F0EF
:103D9000080141607047016841F0400101607047CF
:103DA00030B50246012300BF1068C0F38010A0BBED
:103DB000D1E900042043CC6820430C6920434C69BE
:103DC00020438C692043CC6920430C6A204314684B
:103DD0004FF6BF75AC43204310604C69886840EAD9
:103DE0001440546840F60475AC4320435060886822
:103DF000B0F5006F07D21803546824F480540443CC
:103E0000546000BF00BF086AB0F5005F04D1486A83
:103E100084B2146100BF00BF0023184630BD0146C4
:103E20000868C0F38010704701460868C0F380102E
:103E30007047426822F010020A4342607047000057
:103E4000014908607047000000000020026A8A43B0
:103E500002627047026A0A43026270476FF0020111
:103E6000016170476FF00401016170476FF0080154
:103E7000016170476FF01001016170476FF001013F
:103E80000161704730B5846824F43F4541EA02047B
:103E90001C432543856030BD016821F001010160AC
:103EA0007047016821F0010101607047016821F04D
:103EB000010101607047816821F480418160704791
:103EC000C16821F00101C1607047C16821F00101A2
:103ED000C1607047816821F080018160704701688E
:103EE00041F0800101607047016841F0010101600B
:103EF0007047016841F0010101607047016841F0BD
:103F0000010101607047016841F0010101607047E3
:103F1000C16841F00101C1607047C16841F0010111
:103F2000C1607047C16841F00101C160704701463E
:103F3000886A704710B5024613682C4882420ED03A
:103F4000B2F1804F0BD02A48824208D029488242E1
:103F500005D02948824202D02848824204D123F069
:103F600070004C6840EA04032048824217D0B2F146
:103F7000804F14D01E48824211D01E4882420ED07B
:103F80001D4882420BD01D48824208D01C48824204
:103F900005D01C48824202D01B48824204D123F43F
:103FA0004070CC6840EA040313608868D06200BFA8
:103FB0000888906200BF0D4882420BD00F488242B1
:103FC00008D00F48824205D00E48824202D00E48E7
:103FD000824203D10869106300BF00BF00BF50696F
:103FE00040F00100506100BF002010BD002C0140D6
:103FF0000004004000080040000C00400034014074
:104000000040014000440140004801400146086969
:10401000C0F34000704701460869C0F38000704754
:1040200001460869C0F3C000704701460869C0F343
:10403000001070470146086900F001007047014612
:10404000C868C0F3400070470146C868C0F38000EC
:1040500070470146C868C0F3C00070470146C86891
:10406000C0F3001070470146C86800F001007047B7
:1040700070B50246012901D1002420E0042901D1B4
:1040800001241CE0102901D1022418E0402901D1AB
:10409000032414E0B1F5807F01D104240FE0B1F5D1
:1040A000806F01D105240AE0B1F5805F01D10624BB
:1040B00005E0B1F5803F01D1072400E00824234644
:1040C000064CE55C02F1180428190468044DEE5C06
:1040D0000425B540AC43046070BD000055FF0308E3
:1040E0005EFF030870B50246012901D1002420E0DB
:1040F000042901D101241CE0102901D1022418E077
:10410000402901D1032414E0B1F5807F01D10424BA
:104110000FE0B1F5806F01D105240AE0B1F5805FB1
:1041200001D1062405E0B1F5803F01D1072400E06C
:1041300008242346064CE55C02F11804281904689B
:10414000044DEE5C0425B5402C43046070BD0000B6
:1041500055FF03085EFF030870B50246012901D12F
:10416000002420E0042901D101241CE0102901D100
:10417000022418E0402901D1032414E0B1F5807F26
:1041800001D104240FE0B1F5806F01D105240AE0CC
:10419000B1F5805F01D1062405E0B1F5803F01D182
:1041A000072400E008242346064CE55C02F11804CD
:1041B00028190468044DEE5C0825B5402C430460C2
:1041C00070BD000055FF03085EFF03082DE9F041B4
:1041D00006460C4615460127B4F5805F21D007DC62
:1041E000012C0CD0102C10D0B4F5807F2BD112E014
:1041F000B4F5803F1BD0B4F5801F24D11DE02946C3
:10420000304601F03BFB07461EE02946304601F0F0
:1042100087FB074618E02946304601F0D9FB0746E0
:1042200012E02946304601F025FC07460CE02946FD
:10423000304601F061FC074606E02946304601F0B1
:104240009DFC074600E000BF00BF3846BDE8F08196
:1042500081637047016470478268024B1A400A43C9
:1042600082607047F8BFFEFF826822F008020A43AE
:104270008260704781627047426822F070020A4390
:10428000426070471021016270474021016270470F
:10429000416821F490414160816821F02A018160E8
:1042A0007047024611B902F1280001E002F1240032
:1042B0007047016821F0010101607047016841F019
:1042C00001010160704700002DE9F04104460D46F0
:1042D00001270026204600F08FF8002868D1E96801
:1042E0006868084329690843A96908432168324A74
:1042F000114008432060A868616821F440510143DF
:10430000616000BF6869A16821F440710143A16048
:1043100000BF2A48844204D10320FFF743FC06462D
:104320001FE02748844204D10C20FFF73BFC0646DF
:1043300017E02448844204D13020FFF733FC0646BE
:104340000FE02148844204D1C020FFF7BBFB0646A2
:1043500007E01E48844204D14FF44070FFF7B2FBDF
:1043600006462EB3286818B300273146AB69286883
:10437000B3F5004F12D14FEA410808EB5008B8FBE3
:10438000F0F81FFA88F24FF6F07802EA080CC2F350
:1043900042084CEA080CC4F80CC007E001EB5008D6
:1043A000B8FBF0F81FFA88F8C4F80C8000BF00BF13
:1043B0003846BDE8F0810000F369FFEF00380140A6
:1043C0000044004000480040004C004000500040C5
:1043D0000146C869C0F3400070470146C869C0F390
:1043E000800070470146C869C0F3C00070470146AD
:1043F000C869C0F3801070470146086800F00100EA
:10440000704708B501464FF0E02212690092084655
:1044100000BF421C02B1401C06E04FF0E0221269CE
:1044200002F4803202B1401E0028F6D108BD00001F
:104430002DE9F04393B000201090119012901821B4
:104440000AA8FBF7F6FE0020069007900890099056
:1044500018216846FBF7EDFE4FF08050FE490968D1
:1044600021F040510143FC4A883AC2F8881000BF4D
:10447000C013FEF799FC0120FEF796FC0420FEF71E
:1044800093FC0220FEF790FCDF20009003200190B7
:104490000020049069464FF09040FFF779F93020F2
:1044A000009003200190002004906946EB48FFF73C
:1044B0006FF90220009003200190002004906946CB
:1044C000E748FFF765F9DF214FF09040FFF75CF90F
:1044D0003021E248FFF758F90221E148FFF754F98B
:1044E00000200146DF4A126885000F23AB409A4343
:1044F00085000F23AB4093FAA3F3B3FA83F301FAD9
:1045000003F31A43D74BA83BC3F8A82000BF1846B3
:1045100000210A460346D44D6D5C5D5944F21006F5
:10452000B5431543D04E765C9D5100BF00BF00BF20
:10453000CD4D6D5C5D5925F440551543CA4E765CF2
:104540009D5100BF202200BFC74D6D5C5D5925F015
:1045500020051543C44E765C9D5100BF0A4600BF3E
:10456000C14D6D5C5D5925F040051543BE4E765C2E
:104570009D5100BF802200BFBB4D6D5C5D5925F091
:1045800080051543B84E765C9D5100BF821500BF73
:10459000B54D6D5C5D5925F440751543B24E765CA2
:1045A0009D5100BF021500BFAF4D6D5C5D5925F4F4
:1045B00040651543AC4E765C9D5100BF1221AB4B5C
:1045C0001B68C3F30220052500260346C3F1070834
:1045D000B8F1040F02D94FF0040801E0C3F1070855
:1045E000C44603F10408B8F1070F02D24FF00008E7
:1045F00001E0A3F1030847464FF0010808FA0CF860
:10460000A8F1010808EA050808FA07F84FF00109BF
:1046100009FA07F9A9F1010909EA060948EA0902B4
:1046200000BF002904DB1007030E9148435407E044
:104630001007050E8D480C3001F00F031B1FC554E9
:1046400000BF122000280DDB00BF00BF00F01F02DA
:10465000012191404209920002F1E022C2F80011CA
:1046600000BF00BF00BF002010901190129010A951
:104670008048FEF7CBFA00200A900B200B90002018
:104680000C904FF400500D9003200E9000200F90DE
:104690000AA97848FEF7D6FA77487849896821F060
:1046A000E0710143754A916000BF4FF4E01006903D
:1046B0000020079006A91046FEF766FA00BF6D4875
:1046C00080686F4908406B49886000BF00BF08469A
:1046D00080686C49084040F080506649886000BF9F
:1046E000694800686949B0FBF1F000EB8000800088
:1046F0000A21B0FBF1F400E0641E002CFCD1644AF6
:1047000006215C48FEF7DAFA022261495948FEF7B1
:10471000FDFA7F225E495748FEF70CFB5D4A0C21EB
:104720005448FEF7CBFA02225A495248FEF7EEFAF5
:104730007F2258494F48FEF7FDFA574A12214D484B
:10474000FEF7BCFA022254494A48FEF7DFFA7F22FC
:1047500051494848FEF7EEFA504A18214548FEF7FD
:10476000ADFA02224D494348FEF7D0FA7F224B4969
:104770004048FEF7DFFA4A4A4FF480713D48FEF7A1
:104780009DFA022246493B48FEF7C0FA7F2244497F
:104790003848FEF7CFFA434A4FF483713548FEF7A5
:1047A0008DFA02223F493348FEF7B0FA7F223D4995
:1047B0003048FEF7BFFA3C4A4FF486712D48FEF7A9
:1047C0007DFA022238492B48FEF7A0FA7F223649AB
:1047D0002848FEF7AFFA354A4FF489712548FEF7AD
:1047E0006DFA022231492348FEF790FA7F222F49C1
:1047F0002048FEF79FFA2E4A4FF48C711D48FEF7B1
:104800005DFA02222A491B48FEF780FA7F222849D6
:104810001848FEF78FFA274A4FF400711548FEF743
:104820004DFA022223491348FEF770FA7F222149EC
:104830001048FEF77FFA104A521E40F206210D483A
:10484000FEF73CFA02220C49491E0A48FEF75EFABE
:104850007F220949491E2FE08810024000080048C5
:1048600000040048A8000240E6FE03080CED00E04A
:1048700000E400E000000450010052C700030450AF
:10488000C0FFFF5FC0FFFF7F00000020400D03005E
:104890002000F014400020198000501D00018021EC
:1048A0000002B0250008302E001060320020903643
:1048B0000040C03A000021430A48FEF73BFA0A4A8A
:1048C0004FF403710748FEF7F9F90222064905483B
:1048D000FEF71CFA7F2204490248FEF72BFA13B0B8
:1048E000BDE8F08300000450010000802DE9F04194
:1048F0008EB0182108A8FBF79CFC182102A8FBF732
:1049000098FC4FF000504949896D0143474A916531
:104910001146896D0140019100BF00BF0120114681
:10492000C96C0143D1641146C96C0140019100BFBB
:1049300000BF20200290032003900020069002A9CF
:104940004FF09040FEF724FF3621394B1B68C3F32C
:104950000220062400250346C3F1070CBCF1040F16
:1049600002D94FF0040C01E0C3F1070C674603F1D4
:10497000040CBCF1070F02D24FF0000C01E0A3F1D0
:10498000030C66464FF0010C0CFA07FCACF1010C6D
:104990000CEA040C0CFA06FC4FF0010808FA06F8C1
:1049A000A8F1010808EA05084CEA080200BF00293E
:1049B00004DB1007030E1F48435407E01007040EE2
:1049C0001B480C3001F00F031B1FC45400BF3620DE
:1049D00000280DDB00BF00BF00F01F020121914045
:1049E0004209920002F1E022C2F8001100BF00BFAC
:1049F00000BF382008900020099002200B90002072
:104A00000C900D9008AA0C490C48FEF721FA0A48B0
:104A10000A49096800F0100304229A409143074AAA
:104A2000116000BF0EB0BDE8F08100000010024030
:104A30000CED00E000E400E072004035007400403E
:104A400070B50120FEF794F90220FEF791F903F00A
:104A50008BF905460022052100F074FE044621462C
:104A60000B2003F099F90B2003F04BF903F07CF9CC
:104A700005460022052100F065FE044621460F2070
:104A800003F08AF90F2003F03CF903F06DF90546B5
:104A90000022052100F056FE04462146382003F08E
:104AA0007BF9382003F02DF903F05EF9054600226A
:104AB000052100F047FE04462146392003F06CF939
:104AC000392003F01EF903F04FF9054600220521B5
:104AD00000F038FE04462146442003F05DF94420EE
:104AE00003F00FF903F040F905460022052100F01C
:104AF00029FE04462146452003F04EF9452003F0E7
:104B000000F970BD2DE9F0418AB0002007900890AF
:104B10000990182101A8FBF78CFB1020FEF736F94D
:104B20000420FEF733F98020FEF730F90120FEF76C
:104B30002DF90220FEF72AF90820FEF727F94FF495
:104B40006871E048FEF7DFFE40F20F41DE48FEF7F5
:104B5000DAFE41F20571DD48FEF7D5FE4FF4F8713B
:104B6000DB48FEF7D0FE4FF41041C803FEF7CBFE42
:104B70004FF47850D649886100BF47F64F40019006
:104B8000032002900020059001A9CE48FEF700FE08
:104B90002020019001200290002003900490022028
:104BA000059001A9C748FEF7F3FD4FF46840019056
:104BB000032002900020059001A9C348FEF7E8FDFC
:104BC0000320019001200290002003900120049016
:104BD0000020059001A9BC48FEF7DAFD0C200190E9
:104BE00001200290002003900490059001A9B6488E
:104BF000FEF7CEFD0120019002900020039004906A
:104C00000120059001A9B148FEF7C2FD40F2044021
:104C1000019001200290002003900490059001A9CA
:104C2000AA48FEF7B5FD4FF4607001900120029094
:104C3000002003900490059001A9A248FEF7A8FD6A
:104C40004FF400400190002002900120059001A93E
:104C50009C48FEF79DFD4FF480500190012002908A
:104C60000220039000200490059001A99748FEF7C8
:104C70008FFD4FF4804001900020029001200590AC
:104C800001A99248FEF784FD4FF4D87001900120ED
:104C90000290002003900490059001A98C48FEF733
:104CA00077FD4FF47950019001200290002003908D
:104CB00004900120059001A98548FEF769FD4FF495
:104CC00040400190002002900120059001A98048F9
:104CD000FEF75EFD4FF470700190002002900120FD
:104CE000059001A97848FEF753FD4FF470600190DC
:104CF000032002900020059001A94FF09040FEF79C
:104D000047FD4FF4104001900120029000200390D5
:104D100004900120059001A94FF09040FEF738FD66
:104D20004FF48060019001200290002003900490D5
:104D30000120059001A96448FEF72AFD0A20019090
:104D4000032002900020059001A96148FEF720FD94
:104D50004FF4407001900120029000200390012048
:104D600004900020059001A95848FEF711FD032189
:104D70004FF47020574AC3B252F8232022EA10425F
:104D8000030C93FAA3F3B3FA83F301FA03F31A4380
:104D9000504BC4B243F8242000BF012007900020EC
:104DA000089001208DF8240000208DF825000220B5
:104DB0008DF8260007A8FEF717FA01200146444A9D
:104DC000D26890FAA0F3B3FA83F35C000323A34004
:104DD0009A4390FAA0F3B3FA83F35B0001FA03F36A
:104DE0001A433B4BDA6000BF00211A46126890FA62
:104DF000A0F3B3FA83F35C000323A3409A4390FA31
:104E0000A0F3B3FA83F35B0001FA03F31A43304BC8
:104E10001A6000BF0621304B1B68C3F30220002438
:104E200025460346C3F1070CBCF1040F02D94FF02D
:104E3000040C01E0C3F1070C674603F1040CBCF15C
:104E4000070F02D24FF0000C01E0A3F1030C6646FD
:104E50004FF0010C0CFA07FCACF1010C0CEA040C4D
:104E60000CFA06FC4FF0010808FA06F8A8F1010850
:104E700008EA05084CEA080200BF002904DB100715
:104E8000030E1648435407E01007040E12480C3076
:104E900001F00F031B1FC45400BF062000280DDBC8
:104EA00000BF00BF00F01F020121914042099200A3
:104EB00002F1E022C2F8001100BF00BF00BF0AB03B
:104EC000BDE8F081001000480008004800040048D8
:104ED000000C0048080001400CED00E000E400E098
:104EE00000B591B0282107A8FBF7A3F9182101A864
:104EF000FBF79FF94FF480501E49096E01431D4A8C
:104F000011661146096E0140009100BF00BF0220EA
:104F1000FDF758FF382001900220029003200390F3
:104F20000020049005900520069001A91248FEF784
:104F30002FFC002007904FF4827008904FF4E0603F
:104F4000099002200A9001200B9040020C90002052
:104F50000D900E900F900720109007A90748FEF7BC
:104F60001FFF00210548FEF764FF0448FEF70EFF0F
:104F700011B000BD001002400004004800300140A4
:104F800030B591B0282107A8FBF753F9182101A8E3
:104F9000FBF74FF94FF480405749896D0143564A5A
:104FA00091651146896D0140009100BF00BF02204C
:104FB000FDF708FF4FF420400190022002900320EB
:104FC000039000200490012005900520069001A97F
:104FD0004A48FEF7DDFB04200121494A126884009B
:104FE0000F23A3409A4384000F23A34093FAA3F313
:104FF000B3FA83F301FA03F31A43414BA83BC3F816
:10500000A82000BF18460421102203463D4C645CD2
:105010001C5944F21005AC4314433A4D6D5C5C518D
:1050200000BF002200BF374C645C1C5924F440547C
:105030001443344D6D5C5C5100BF00BF00BF314C68
:10504000645C1C5924F0200414432E4D6D5C5C51AB
:1050500000BF00BF00BF2B4C645C1C5924F040040F
:105060001443284D6D5C5C5100BF802200BF254C6D
:10507000645C1C5924F080041443224D6D5C5C5127
:1050800000BF002200BF1F4C645C1C5924F4407414
:1050900014431C4D6D5C5C5100BF00BF00BF194C38
:1050A000645C1C5924F440641443164D6D5C5C51DF
:1050B00000BF002007904FF4827008904FF4E0602A
:1050C000099000200A900B90C8010C9008200D90C8
:1050D00080200E9000200F900720109007A90A480A
:1050E000FEF75EFE00210848FEF7A3FE0648FEF725
:1050F0004DFE11B030BD0000001002400004004819
:10510000A80002401AFF03080038004030B585B0FF
:1051100014216846FBF78DF84FF40030FDF78AFE46
:1051200002F02AFE054600220F2100F02BFB044668
:105130002146192002F044FE192002F0F3FD40F24E
:105140008F10ADF800000020019018200290002080
:105150000390049069460448FEF7ECFE0248FEF70F
:10516000BEFE05B030BD00000044014030B585B042
:1051700014216846FBF75DF84FF48020FDF75AFED6
:1051800002F0FAFD05460022052100F0FBFA044674
:1051900021461A2002F014FE1A2002F0C3FD40F24C
:1051A0008F10ADF800000020019040F2E73002902F
:1051B00000200390049069460348FEF7BBFE0248B6
:1051C000FEF78DFE05B030BD0048014000B593B03C
:1051D00014210EA8FBF72DF8202106A8FBF729F8CB
:1051E00018216846FBF725F80120FDF715FE002081
:1051F000ADF838000F9040F69F701090002011908D
:105200000EA94FF08040FEF795FE4FF08040FEF76C
:1052100066FE00214FF08040FFF71EF84FF48051EA
:105220008804FEF799FF6020069000200790089000
:1052300009900A9006AA4FF480518804FEF7C6FF31
:105240004FF480518804FEF74DFF00214FF080405D
:10525000FFF70AF84FF08040FEF72DFE00231A46B4
:1052600019464FF08040FEF70DFE00214FF08040C0
:10527000FFF702F84FF08040FEF72CFE0220FDF70A
:10528000AFFD4FF4006000900220019000200290DA
:10529000039004900120059069460248FEF778FAD1
:1052A00013B000BD0004004800B593B014210EA84F
:1052B000FAF7BFFF202106A8FAF7BBFF18216846BE
:1052C000FAF7B7FF0220FDF7A7FD0020ADF8380080
:1052D0000F9040F69F701090002011900EA9224868
:1052E000FEF728FE2048FEF7FAFD00211E48FEF7D3
:1052F000B3FF10211C48FEF72FFF6020069000200E
:105300000790089009900A9006AA10211648FEF707
:105310005DFF10211448FEF7ABFE00211248FEF796
:10532000A3FF1148FEF7C7FD00231A4619460E4891
:10533000FEF7A8FD00210C48FEF79EFF0A48FEF785
:10534000C9FD1020FDF74CFD1020009002200190B7
:1053500000200290039004900220059069460348C3
:10536000FEF716FA13B000BD00040040001000481C
:1053700030B585B014216846FAF75BFF1020FDF7C1
:105380004BFD02F0F9FC05460022062100F0FAF977
:1053900004462146362002F013FD362002F0C2FCFE
:1053A00040F28F10ADF800000020019063200290C1
:1053B00069460748FEF7BEFD0548FEF790FD00214F
:1053C0000348FEF759FF0248FEF784FD05B030BDE3
:1053D0000010004030B585B014216846FAF729FF67
:1053E0002020FDF719FD02F0C7FC0546002201212F
:1053F00000F0C8F904462146372002F0E1FC3720CE
:1054000002F090FC40F28F10ADF8000000200190F7
:10541000F920029069460748FEF78CFD0548FEF723
:105420005EFD00210348FEF727FF0248FEF752FD0C
:1054300005B030BD0014004030B58FB01C2108A865
:10544000FAF7F7FE182102A8FAF7F3FE4FF04070C2
:105450005949096821EA104182B21143564A883AF3
:10546000C2F8881000BF4FF480101146896D0143C7
:1054700091651146896D0140019100BF00BF042074
:10548000FDF7BCFC0820FDF7B9FC4FF480500290FA
:10549000022003900320049000200590069008202D
:1054A000079002A94548FEF773F9042002900220F4
:1054B0000390032004900020059006900820079098
:1054C00002A93F48FEF764F9022201213D48FDF799
:1054D00003FE002201213B48FDF78EFD0022012141
:1054E0003848FDF75BFD002201213648FDF7C4FD79
:1054F000002201213348FDF7E1FD802201213148DE
:10550000FDF79EFD002201212E48FDF7F9FD002246
:1055100001212C48FDF7A2FD022200212948FDF7B8
:10552000DBFD102200212748FDF766FD0022114611
:105530002448FDF733FD002211462248FDF79CFD6B
:10554000002211461F48FDF7B9FD802200211D48A9
:10555000FDF776FD002211461A48FDF7D1FD002225
:1055600011461848FDF77AFD02F00EFC05460022B0
:10557000032100F027F904462146352002F034FCCF
:10558000352002F0E0FB4FF4E13008900020099054
:105590000A900B900C200C9000200D900E9008A902
:1055A0000948FEF791FE0848FEF772FE0648FEF72E
:1055B00085FE0FB030BD0000881002400008004892
:1055C000000C0048000402400050004030B58FB08D
:1055D0001C2108A8FAF72DFE182102A8FAF729FEC7
:1055E0004FF440305149096821EA104182B2114319
:1055F0004E4A883AC2F8881000BF4FF480401146E6
:10560000096E014311661146096E0140019100BF08
:1056100000BF0220FDF7F2FBC020029002200390A1
:10562000032004900020059006900720079002A90F
:105630003F48FEF7ADF8022206213E48FDF74CFD3B
:10564000002206213B48FDF7D7FC002206213948FD
:10565000FDF7A4FC002206213648FDF70DFD0022CF
:1056600006213448FDF72AFD802206213148FDF746
:10567000E7FC002206212F48FDF742FD002206210B
:105680002C48FDF7EBFC022205212A48FDF724FDFA
:10569000102205212748FDF7AFFC002205212548EF
:1056A000FDF77CFC002205212248FDF7E5FC0022E5
:1056B00005212048FDF702FD802205211D48FDF748
:1056C000BFFC002205211B48FDF71AFD0022052121
:1056D0001848FDF7C3FC02F057FB054600221146AF
:1056E00000F070F804462146252002F07DFB2520BD
:1056F00002F029FB4FF4966008904FF48050099017
:1057000000200A904FF4C0600B900C200C900020F9
:105710000D900E9008A90848FEF7D6FD0648FEF742
:10572000B7FD0548FEF7CAFD0FB030BD8810024036
:1057300000040048000402400038014000BFFEE7BA
:1057400000BFFEE7F0B503460C4603F00701C1F1C8
:105750000700042801D9042001E0C1F10700064632
:10576000081D072801D2002000E0C81E05460120C0
:10577000B040401E2040A8400127AF407F1E174088
:105780003843F0BDF0B503460C4603F00701C1F104
:105790000700042801D9042001E0C1F107000646F2
:1057A000081D072801D2002000E0C81E0546012080
:1057B000B040401E2040A8400127AF407F1E174048
:1057C0003843F0BDF0B503460C4603F00701C1F1C4
:1057D0000700042801D9042001E0C1F107000646B2
:1057E000081D072801D2002000E0C81E0546012040
:1057F000B040401E2040A8400127AF407F1E174008
:105800003843F0BD2DE9F04704460F4616461D46C5
:105810003946E069FAF7A0FD82463146FAF79CFD69
:1058200081462968FAF798FD8046616CFAF73CFDDD
:1058300060643946A069FAF78FFD82463146FAF76F
:105840008BFD81466968FAF787FD8046216CFAF77F
:105850002BFD20643946206AFAF77EFD82463146E8
:10586000FAF77AFD8146A968FAF776FD8046A16CC1
:10587000FAF71AFDA064BDE8F087000070B5024693
:10588000106A20F001001062136A5568946924F0D0
:1058900003041D4E04EA06000E6840EA060423F0E5
:1058A00002000E6940EA060323F001004E6840EA58
:1058B0000603164882420BD01548824208D015488C
:1058C000824205D01448824202D01448824213D149
:1058D00023F008004E6940EA860323F004008E6836
:1058E00040EA860325F480708E6940EA060525F4B7
:1058F0000070CE6940EA460555609461C8685063FF
:1059000000BF1362002070BD8FFFFEFF002C01401E
:105910000034014000400140004401400048014083
:105920002DE9F04104460D46206A20F01000206267
:10593000266AD4F80480A76927F440771E483840C7
:10594000296840EA012726F02000296940EA01166B
:1059500026F01000696840EA0116184884420BD00E
:105960001748844208D01748844205D0164884421C
:1059700002D01648844213D126F08000696940EABB
:10598000811626F04000A96840EA811628F480605C
:10599000A96940EA810828F40060E96940EAC10881
:1059A000C4F80480A7612046E968FEF751FC26622E
:1059B0000020BDE8F0810000FF8FFFFE002C0140B9
:1059C00000340140004001400044014000480140D3
:1059D00070B50246106A20F480701062136A556830
:1059E000D46924F003041D4E04EA06000E6840EA60
:1059F000060423F400700E6940EA062323F4807045
:105A00004E6840EA0623164882420BD0154882426F
:105A100008D01548824205D01448824202D014486A
:105A2000824213D123F400604E6940EA862323F4B6
:105A300080608E6840EA862325F480508E6940EAB3
:105A4000061525F40050CE6940EA46155560D4612C
:105A5000C868D06300BF1362002070BD8FFFFEFFD7
:105A6000002C01400034014000400140004401404E
:105A70000048014070B50246106A20F48050106260
:105A8000146A5568D36923F44073154818400E68AA
:105A900040EA062324F400500E6940EA063424F458
:105AA00080504E6840EA06340E4882420BD00E48C1
:105AB000824208D00D48824205D00D48824202D071
:105AC0000C48824204D125F480408E6940EA861554
:105AD0005560D361C868106400BF1462002070BDB7
:105AE000FF8FFFFE002C01400034014000400140C8
:105AF000004401400048014030B50246106A20F4DD
:105B000080301062136A546D164D04EA05000D686A
:105B100040EA050423F400300D8A40EA054323F4EB
:105B200080308D8840EA05430F4882420BD00F48F1
:105B3000824208D00E48824205D00E48824202D0EE
:105B40000D48824206D1506820F480308D6940EAC9
:105B5000052050605465C868956D906500BF13625C
:105B6000002030BD8FFFFEFF002C014000340140BB
:105B700000400140004401400048014030B5024669
:105B8000106A20F480101062136A546D154820408A
:105B90000D6840EA052423F400100D8A40EA0553FD
:105BA00023F480108D8840EA05530F4882420BD0C1
:105BB0000E48824208D00E48824205D00D488242EB
:105BC00002D00D48824206D1506820F480208D69B1
:105BD00040EA852050605465C868D06500BF1362F4
:105BE000002030BDFF8FFFFE002C0140003401403B
:105BF000004001400044014000480140704700005F
:105C000030B5032310200C21CA05154CE46824F09C
:105C1000730443EA00052C43114DEC602C462469C3
:105C2000104D2C4042EA01252C430D4D2C6100BF44
:105C300000BF2846006940F080702946086100BF17
:105C400000BF0846006840F08060086000BF00BFE9
:105C500000BF03480068C0F3C0600028F8D030BD22
:105C600000100240FF80FFF9014600BF0448806831
:105C700000F0F0000009034A125C21FA02F07047BC
:105C800000100240B8FF0308014600BF05488068C5
:105C900000F4E060044A02EB1020027821FA02F0DE
:105CA0007047000000100240C8FF0308014600BF13
:105CB0000548806800F46050044A02EBD020027866
:105CC00021FA02F07047000000100240C8FF0308EC
:105CD00010B500BF2948806800F00C0030B10428DE
:105CE00022D0082822D00C2826D121E0FEF712F875
:105CF00060B9FEF70FF810B1FDF7FCFF01E0FEF709
:105D000001F8000A1E4951F820000BE0FEF702F8E6
:105D100010B1FDF7EFFF01E0FDF7F4FF00091849AE
:105D200051F82000044625E0164C23E0164C21E0F3
:105D300000F02CF804461DE0FDF7ECFF60B9FDF71C
:105D4000E9FF10B1FDF7D6FF01E0FDF7DBFF000A28
:105D50000B4951F820000BE0FDF7DCFF10B1FDF717
:105D6000C9FF01E0FDF7CEFF0009054951F8200009
:105D7000044600BF00BF204610BD000000100240D6
:105D8000D0FF03080024F40000127A0070B5FDF77C
:105D9000D1FF0546012D04D0022D20D0032D22D1A4
:105DA0001FE0FDF7B7FF60B9FDF7B4FF10B1FDF7D5
:105DB000A1FF01E0FDF7A6FF000A254951F82000E8
:105DC0000BE0FDF7A7FF10B1FDF794FF01E0FDF731
:105DD00099FF00091E4951F82000044621E01D4C9E
:105DE0001FE01D4C1DE0FDF795FF60B9FDF792FF28
:105DF00010B1FDF77FFF01E0FDF784FF000A1449B1
:105E000051F820000BE0FDF785FF10B1FDF772FFA0
:105E100001E0FDF777FF00090D4951F82000044625
:105E200000BF00BFFDF77EFF012101EB1010B4FBA6
:105E3000F0F6FDF787FF46430848C06800F0C060F1
:105E4000012101EB50604000B6FBF0F070BD000096
:105E5000D0FF03080024F40000127A000010024072
:105E600008B5014600910098000E009A02F47F02E6
:105E700000EB1220009A02F47F4200EB0220009A0D
:105E800000EB02600090009808BD08B50146009143
:105E90000098000E009A02F47F0200EB1220009A94
:105EA00002F47F4200EB0220009A00EB02600090B7
:105EB000009808BD704770B502460C4600210020CE
:105EC00000231578302D3ED15578782D02D05578A5
:105ED000582D38D102212BE0555C412D02DB555C59
:105EE000462D0BDD555C612D02DB555C662D05DD15
:105EF000555C302D19DB555C392D16DC555C302D89
:105F000005DB555C392D02DC555C303D0AE0555C03
:105F1000412D05DB555C462D02DC555C373D01E02B
:105F2000555C573D05EB031301E0002005E0491CDB
:105F30000B2902D2555C002DCED100BF555C9DBB14
:105F40002360012030E02AE0555C15B92360012070
:105F500024E0555C6B2D02D0555C4B2D04D119B15A
:105F60009B022360012019E0555C6D2D02D0555C29
:105F70004D2D04D119B11B05236001200EE0555CA5
:105F8000302D09DB555C392D06DC555C303D03EBCB
:105F9000830605EB460301E0002004E0491C0B29C1
:105FA00001D20128D0D100BF70BD704770B500206C
:105FB0004549096821F007010143434A116000BFC8
:105FC00000BF00BF4048006800F007000028F8D17B
:105FD0004FF400703D49096821F4C06101433B4A18
:105FE000116000BF00BF00BF38484069C0F3802087
:105FF0000028F8D100BF3648006840F480303449AA
:10600000086000BF00BF00BF31480068C0F34040D7
:106010000028F8D0032010210C228B0540EA01044F
:1060200044EA02241C432A4DED682A4E35402C4395
:10603000274DEC6000BF00BF2846C06840F080706C
:106040002946C86000BF00BF0846006840F0807065
:10605000086000BF00BF00BF1D480068C0F340607B
:106060000028F8D003201A49896821F00301014370
:10607000174A916000BF00BF00BF1548806800F05C
:106080000C000C28F8D180201149896821F0F0011A
:1060900001430F4A916000BF00201146896821F436
:1060A000E0610143916000BF00BF1146896821F49F
:1060B00060510143916000BF0748FDF7F5FC0648B9
:1060C000FDF7BEFE70BD00000020024000700040E1
:1060D000001002408C80FFF90060540070470000FF
:1060E00010B52948FDF7A6FF01284CD100BF26486E
:1060F000FDF78CFF012807D12348FDF7A0FF0128F9
:1061000002D12148FDF7AAFE1F48FDF784FF0128B0
:1061100007D11D48FDF798FF012802D11A48FDF765
:10612000A1FE1948FDF77CFF012807D11648FDF7AD
:1061300090FF012802D11448FDF798FE1248FDF7A0
:1061400074FF012807D11048FDF788FF012802D10C
:106150000D48FDF78FFE0C48FDF76CFF012807D1B5
:106160000948FDF780FF012802D10748FDF786FEA8
:1061700000BF2AF0DDFA0548007800F0010010B1F8
:10618000642034F06FFB10BD00480140780200101D
:1061900010B52548FDF74EFF012844D100BF224825
:1061A000FDF734FF012807D11F48FDF748FF0128FC
:1061B00002D11D48FDF752FE1B48FDF72CFF0128B8
:1061C00007D11948FDF740FF012802D11648FDF715
:1061D00049FE1548FDF724FF012807D11248FDF7B5
:1061E00038FF012802D11048FDF740FE0E48FDF7A8
:1061F0001CFF012807D10C48FDF730FF012802D110
:106200000948FDF737FE0848FDF714FF012807D1BC
:106210000548FDF728FF012802D10348FDF72EFEAF
:1062200000BF1CF0F1FB10BD0044014010B52C482C
:10623000FDF700FF012852D100BF2948FDF7E6FE17
:10624000012807D12648FDF7FAFE012802D124488B
:10625000FDF704FE2248FDF7DEFE012807D12048A5
:10626000FDF7F2FE012802D11D48FDF7FBFD1C4899
:10627000FDF7D6FE012807D11948FDF7EAFE0128EF
:1062800002D11748FDF7F2FD1548FDF7CEFE0128B3
:1062900007D11348FDF7E2FE012802D11048FDF7AF
:1062A000E9FD0F48FDF7C6FE012807D10C48FDF7B0
:1062B000DAFE012802D10A48FDF7E0FD00BFFDF734
:1062C000EBFB0848007800F0010040B100BF064831
:1062D0000068401C0449086000BF08F005FC10BDC0
:1062E00000100040780200107C03002010B5284800
:1062F000FDF7A0FE012849D100BF2548FDF786FE25
:10630000012807D12248FDF79AFE012802D1204832
:10631000FDF7A4FD1E48FDF77EFE012807D11C48AD
:10632000FDF792FE012802D11948FDF79BFD1848A0
:10633000FDF776FE012807D11548FDF78AFE0128F2
:1063400002D11348FDF792FD1148FDF76EFE0128BA
:1063500007D10F48FDF782FE012802D10C48FDF756
:1063600089FD0B48FDF766FE012807D10848FDF7B7
:106370007AFE012802D10648FDF780FD00BF0548DE
:10638000007800F0010008B12AF0EEF910BD00001D
:1063900000140040780200102DE9F0470546012D59
:1063A00002DB0020BDE8F08705EBC500334901EBB7
:1063B00000104068002801DA0020F3E705EBC50073
:1063C0002E4901EB0014A06E08B9022001E0A06E76
:1063D000401E86B204F13802A36E02EB03129168EC
:1063E00004F1380202EB03121068F9F7AFFF81469F
:1063F0002349F9F7B1FF0746D4E90601F9F7A6FFEB
:1064000081464FF08141F9F7A7FF80463946F9F7F9
:10641000D5FFE06604F13801A26E01EB02114A6873
:1064200004F1380101EB06114968501AFAF7C5F971
:1064300020676078012804D11248E16EF9F78CFFDB
:1064400003E01148E16EF9F787FF60674FF07C5079
:10645000216FF9F781FF07463946606FF9F7AEFF04
:10646000A0674FF07850216FF9F776FF0746616F0C
:10647000F9F772FFE067012094E700004C3000104C
:10648000D00F49409A99193FCDCC4C3F2DE9F047A8
:1064900005460C4605B114B90020BDE8F08700267A
:1064A0000027B04607E055F828103046F9F7FCFE03
:1064B000064608F10108A045F5D314493046F9F71E
:1064C0007DFF06464FF0000810E055F828003146E1
:1064D000F9F73CFF82464FF080412EF057F9814694
:1064E0003946F9F7E1FE074608F10108A045ECD36B
:1064F0002046FAF762F9804641463846F9F75EFFD2
:106500000746384636F087FDC7E7000000004040E8
:106510000146012901DB0020704701EBC100164A4A
:1065200002EB00104068002801DA0020F4E70020A8
:1065300001EBC102104B03EB0212106201EBC1022E
:1065400003EB0212506201EBC10203EB0212D062B4
:1065500001EBC10203EB02121063012001EBC10247
:1065600003EB02121072002001EBC10203EB0212D6
:1065700090660120D0E700004C30001010B50246B4
:10658000012A01DB002010BD02EBC200084C04EB25
:1065900000104068002801DA0020F4E702EBC20096
:1065A000034C04EB0013D86F08604FF07E50EAE70D
:1065B0004C30001010B50246012A01DB002010BD4E
:1065C00002EBC200084C04EB00104068002801DA1E
:1065D0000020F4E702EBC200034C04EB0013986FB9
:1065E00008604FF07E50EAE74C30001010B50246CC
:1065F000012A01DB002010BD02EBC200084C04EBB5
:1066000000104068002801DA0020F4E702EBC20025
:10661000034C04EB0013586F08604FF07E50EAE71C
:106620004C300010F0B504460F4615461E46012CAE
:1066300001DB0020F0BD04EBC4000C4901EB0010AD
:106640004068002801DA0020F4E71FB139462046EF
:10665000FFF7CCFF1DB129462046FFF7ABFF1EB167
:1066600031462046FFF78AFF0120E3E74C30001057
:1066700010B5002404E0204600F0AEF8601C04B21F
:10668000012CF8DB10BD000010B50146002044E0ED
:1066900000EBC002234B03EB02125268002A3ADAE5
:1066A00000EBC00203EB0212506001B910BD0A7882
:1066B00000EBC0031B4C04EB03135A7000EBC00348
:1066C00004EB03138A689A6100EBC00304EB031325
:1066D000CA68DA6100EBC00304EB03134A689A62EC
:1066E00000EBC00304EB03130A695A614A7800EB1C
:1066F000C00304EB03139A7000EBC00304EB031315
:106700004A69C3F8802000EBC00304EB03138A69D5
:10671000C3F88420CAE7421C10B20128B8DB4FF04E
:10672000FF30C3E74C30001030B500EBC003124C13
:1067300004EB0313383303EB01131A60002400EB5E
:10674000C0030D4D05EB0313383303EB01135C60FD
:1067500000EBC0032C4604EB0313383303EB0113A7
:106760009A60002400EBC00305EB0313383303EBFE
:106770000113DC6030BD00004C30001010B5044641
:10678000012C01DB002010BD04EBC400114901EB1A
:1067900000104068002801DA0020F4E704EBC40090
:1067A0000C4901EB0010007803280CD004EBC40066
:1067B00001EB00100078042805D004EBC40001EBC5
:1067C0000010007820B9204600F006F80120DAE732
:1067D0000020D8E74C30001010B50446012C01DB36
:1067E000002010BD002004EBC401154A02EB01118A
:1067F0000870401E04EBC40102EB01114860012047
:1068000004EBC40102EB011148700E4804EBC40113
:1068100002EB01118861052004EBC40102EB0111B8
:106820008862002004EBC40102EB0111887020464D
:10683000FFF76EFE08B90020D3E70120D1E7000082
:106840004C300010000048422DE9FF4F87B08246CF
:1068500088461546BAF1010F03DB03200BB000F0A8
:106860002DB90AEBCA00934901EB001040680028DB
:1068700001DA0320F2E70AEBCA008E4901EB0014AB
:10688000C4F80C80216A0A9808442062A07818B9DC
:10689000D4F81890E76902E0D4F81C90A769207832
:1068A00005287AD2DFE800F003133EF5FB005046DE
:1068B000FFF72EFE40466169FAF766F802D8C5F880
:1068C000009000E02F60012020700020C6E74046C5
:1068D0006169FAF759F80AD20020E062206B401C87
:1068E0002063A16A88421BD3C5F8009018E00020FD
:1068F0002063E06A401CE062A16A884210D3002154
:1069000050466269FFF710FF012150466269FFF7A8
:106910000BFF022150466269FFF706FF022020703C
:1069200000209BE740466169FAF738F836D200202C
:106930002063E06A401CE062A16A88422CD32F6089
:10694000207A88B90120207200206063A06E02289E
:1069500002DB0020A06602E0A06E401CA06650464C
:106960006269A16EFFF7E0FE04F13800A26E00EB51
:10697000021001684046FAF711F87DD804F138009A
:10698000A16E00EB0110C0F8008004F13800A26E87
:1069900000EB0210216A41606EE089E00020E062B5
:1069A000206B401C2063A16A884265D3C5F8009023
:1069B000207A012804D100202072606A401C6062A5
:1069C00004F13800A26E00EB021081684046F9F72E
:1069D000DBFF10D804F13800A16E00EB0110C0F805
:1069E000088004F13800A26E00EB0210216AC16039
:1069F0000120606304E0606B10B1606B401C606359
:106A0000606A032838D3A16A606B884234D30026B9
:106A10001EE004F1380202EB0612916804F138021C
:106A200002EB06121068F9F791FC03A941F8260061
:106A300004F1380101EB0611CA6804F1380101EBD9
:106A400006114968501AF9F7B8FE4DF82600761C71
:106A5000032EDEDB032103A8FFF718FD06900321B8
:106A60006846FFF713FD83460698C4F88800C4F80B
:106A70008CB00420207000BF606A642803D80E49DF
:106A8000206A884201D9032020700220E6E606E051
:106A9000FFE75046FFF73CFD2F600320DEE650463F
:106AA000FFF77AFC5046FFF733FD2F600420D5E650
:106AB0000020D3E64C30001080EE360030BCBDE83C
:106AC000C08F000010B50249486837F0DFFD10BDE7
:106AD0000000001010B50A49086837F0D7FD0848D3
:106AE0000068408D012806DD1BF084FF18B90449B9
:106AF000086837F0B8FC0A201BF096FF10BD0000B4
:106B00000000001000BFFEE730B50B4C23680C2BD3
:106B100010DA0A4A190009D002EB410535F9025C86
:106B2000854203DB22F81150491EF5D122F81100ED
:106B30005B1C236030BD0000AC040020DE5401204B
:106B40002DE9F04180461D4614460E461046069F2C
:106B5000F9F71AFF02D13046BDE8F08131462046F0
:106B6000F9F7F4FB044629463846F9F7EFFB2146CE
:106B7000F9F724FC044631464046F9F7E7FB214685
:106B8000F9F7EAFB2946BDE8F041F9F78DBB012092
:106B9000704710B54943541A0368914202D300214B
:106BA000016010BD5B1C03FB03F1A142FAD35B1E25
:106BB000036010BDF7B5114C0D46206920B1114698
:106BC000FBF7DAFA002806D0A069006920B18268D4
:106BD000294600989047FEBD094E0BE06846FBF73A
:106BE00017FB0746A069016838468847316809B134
:106BF000384688476D1EF1D5FEBD00000C300010F0
:106C00003804002070B50D4604460AE014F8010B64
:106C10007F2804D914F8011B6D1E41EA0020FAF701
:106C200047FC6D1EF2D570BD2DE9F04FDFF818B2AC
:106C300095B0814690460C469BF81400219FF9F7C9
:106C4000D2FD0022814BF9F7F7FB4FF0FF32F9F745
:106C500086FD8A46054656464046F9F7B3FD80460E
:106C600033462A460091F9F788FCF9F771FE06468B
:106C70002A46534640460099F9F7DEFBF9F768FECD
:106C800005461E98F9F79EFDDFF8C481714B424618
:106C9000F9F781FC0022704BF9F7F2FCF9F758FE86
:106CA00082461F98F9F78EFD42466A4BF9F773FC4E
:106CB0000022694BF9F7E4FCF9F74AFE804650469A
:106CC000FAF700F904904046FAF7FCF803905046B2
:106CD000FAF7A4F802904046FAF7A0F88046314649
:106CE0000846F9F739FBF9F7A4FD2946069008464E
:106CF000F9F732FBF9F79DFD059030460499F9F755
:106D00002BFB099028460499F9F726FB0A90304698
:106D10000399F9F721FB824628460399F9F71CFBF2
:106D20000C9030460299F9F717FB0D90284602990E
:106D3000F9F712FB0E9041463046F9F70DFB0F9024
:106D400041462846F9F708FB10900998F9F7BDFD70
:106D500008F09AFBF9F781FD05460C98F9F7B5FDA7
:106D600010F006FFF9F779FDDBF81010E9B1012FFB
:106D700002D07A1C0DD018E0B1F90620121B824215
:106D800000DA1046B1F90210091BA9420DDD0D46CB
:106D90000BE0B1F90620121BAA4200DA1546B1F940
:106DA0000210091B814200DD0846002111910646B0
:106DB000129143E0314611A8069AFFF7EAFE3146E8
:106DC00012A8059AFFF7E5FE3046F9F7EDFC14909E
:106DD0000A99F9F7D9FD0AD20E9914980091DDE9C4
:106DE00009120D9BFFF7ACFEF9F70AFD00E01298BF
:106DF000514680461498F9F7D1FD0AD2109914989B
:106E0000009151460F9B0C9AFFF79AFEF9F7F8FC98
:106E100000E011982099002905DD07FB064108EBE9
:106E20000902484405E0A9EB000207FB0641A9EB73
:106E30000800DBF838301B689847761EAE42B9DA96
:106E400015B000F00BB800000C3000100000F83F47
:106E50004AD8124DFB2109400080664030BCBDE895
:106E6000C08F00002DE9F05F1C468B46DDE90A71FA
:106E700005192A4891F8009091F80180007B164688
:106E800010F003014FF0800013D001292DD002290A
:106E900024D18146317829FA04F0014204D04246D7
:106EA00059462846FBF7E6FD641C6D1C082C17D0DC
:106EB00018E0824631782AFA04F0014201D04246B5
:106EC00000E04A4628466D1C5946FBF7D3FD641C7A
:106ED000082C01D10024761C7F1EEBD100F020B8D5
:106EE0000024761C7F1ED5D1F8E78046317828FA39
:106EF00004F0014209D059462846FBF79DFDC0F138
:106F0000FF0259462846FBF7B5FD641C6D1C082C92
:106F100001D10024761C7F1EE8D1DFE70C30001081
:106F200030BCBDE8C09F00002DE9F05F1C4605198C
:106F30003E488B46DDE90A79007B167810F00301A4
:106F400090464FF0C0001AD0022935D15FEA0901FE
:106F500053D08246C4F103004100C1F106022AFA6F
:106F600002F03040C84005D019F8002059462846A4
:106F7000FBF780FD641C6D1C042C38D03AE05FEAFE
:106F800009011BD04FEA000AC4F103004100C1F11E
:106F900006022AFA02F03040C840594619F800208B
:106FA00028466D1CFBF766FD641C042C02D118F802
:106FB000016F00247F1EE7D100F03AB84FEA0009C4
:106FC000C4F103004000C0F1060129FA01F2324089
:106FD000C24028466D1C5946FBF74CFD641C042C2E
:106FE00002D118F8016F00247F1EE9D1E4E718F8F8
:106FF000016F00247F1EADD1DEE78146C4F103009E
:107000004000C0F1060129FA01F23240C24003D02B
:1070100059462846FBF72EFD641C6D1C042C02D13A
:1070200018F8016F00247F1EE8D1C5E70C3000106E
:1070300030BCBDE8C09F00002DE9F05F1C4605197B
:107040003E488B46DDE90A79007B167810F0030193
:1070500090464FF0F0001AD0022935D15FEA0901BD
:1070600053D08246C4F101008100C1F104022AFA22
:1070700002F03040C84005D019F800205946284693
:10708000FBF7F8FC641C6D1C022C38D03AE05FEA78
:1070900009011BD04FEA000AC4F101008100C1F1CF
:1070A00004022AFA02F03040C840594619F800207C
:1070B00028466D1CFBF7DEFC641C022C02D118F87C
:1070C000016F00247F1EE7D100F03AB84FEA0009B3
:1070D000C4F101008000C0F1040129FA01F232403C
:1070E000C24028466D1C5946FBF7C4FC641C022CA8
:1070F00002D118F8016F00247F1EE9D1E4E718F8E7
:10710000016F00247F1EADD1DEE78146C4F101008E
:107110008000C0F1040129FA01F23240C24003D0DC
:1071200059462846FBF7A6FC641C6D1C022C02D1B4
:1071300018F8016F00247F1EE8D1C5E70C3000105D
:1071400030BCBDE8C09F00002DE9F0410646204854
:10715000069F1C46007B1546884610F0030003D0AE
:1071600002280ED127BB2FE04FB914E02878414602
:107170003A5C3046FBF77EFC641E6D1C761C002CCE
:10718000F4DCBDE8F0812A7841463046FBF772FC1A
:10719000641E6D1C761C002CF5DCF2E7287820B10B
:1071A0003A5C41463046FBF765FC641E6D1C761C5C
:1071B000002CF3DCE5E72A781AB141463046FBF7AC
:1071C00059FC641E6D1C761C002CF4DCD9E7000011
:1071D0000C300010034A527D002A01D1FAF72EBB71
:1071E000704700000C3000100170012070470078DB
:1071F00070470120704700000249097B490700D50C
:10720000401E70470C30001070B50D4604004FF062
:1072100000060CD10FE0641C6D1E7F2804D914F801
:10722000011B6D1E41EA0020FAF72EFF064420786C
:1072300008B1002DEFDA304670BD0246002008E0AC
:10724000521C7F2B02D9401C521C01E00A2B05D096
:10725000401C1378002B01D08842F1DB70470346B5
:10726000002070472DE9FF5F05460E4691464FF01E
:10727000000AD34600200390029005F130042660F6
:10728000C4F80490D4E90001F9F760F8E061D4F89B
:107290001CA0A06AF9F719FB07468846E069F9F7D0
:1072A00014FB21F000413A464346CDE90001F9F7CD
:1072B0001FFB00D8DA46A16CA06BF9F76FFB22D850
:1072C000E06AF9F702FBCDE900015046F9F7FDFA53
:1072D00021F000410746DDE90023F9F721FB05D243
:1072E00094F8460010B14FF0000B52E04FF07E5B77
:1072F00000215046F9F748FB4BD251462069F9F777
:107300002BF8039045E0E16CA06BF9F73DFB22D828
:10731000E06AF9F7DAFACDE900015046F9F7D5FA53
:1073200021F000410746DDE90023F9F7F9FA05D21B
:1073300094F8460010B14FF0000B2AE04FF07E5B4E
:1073400000215046F9F72AFB23D251462069F9F76C
:1073500003F803901DE0E06AF9F7B7FA074688469C
:107360005046F9F7B2FA21F000413A464346CDE9DA
:107370000001F9F7D5FA05D294F8460010B14FF0A4
:10738000000B06E04FF07E5B51462069F8F7E4FF02
:10739000039094F8440010B9002003908346E06BFA
:1073A0000399F8F781FFE06394F84700012814D1AE
:1073B000D4E90F01F9F7F2FA02D2206CE0631BE086
:1073C000206C80F000473846E16BF9F7E7FA13D2FA
:1073D000206C80F00040E0630EE0A16CE06BF9F7F8
:1073E000DDFA02D2A06CE06306E0E16CE06BF9F735
:1073F000CBFA01D2E06CE06394F84500012802D199
:107400006069029001E000200290D4E90701F8F7DA
:107410009DFF01900299F8F79FFF07465946E06BE0
:10742000F8F79AFF0190E169E068F8F795FF00909E
:107430000199F8F739FF80463946F8F735FFA06320
:10744000E06920626068A060E16CA06BF9F79CFACB
:1074500001D2E06C00E0A06B0746A16CF9F794FA4A
:1074600008D2E16CA06BF9F78FFA01D2E06C02E070
:10747000A06B00E0A06CA063A06B04B000F000B8AB
:1074800030BCBDE8C09F00002DE9F74FCCB04C9850
:1074900000F10804002600270020099008904D986C
:1074A0004B904E984A904A994B98F8F74FFF0546F3
:1074B0003B952846A169F8F749FFFE490860284630
:1074C000F9F703FA21F000410022FB4BCDE902015C
:1074D000F9F70EFA7ED8F9493B98F8F73DFFF84ADC
:1074E000F8490390F9F73EFF4390F4493B98F8F7C9
:1074F00033FF00234FF04042F2490390F9F791FF28
:107500004490EE493B98F8F727FF4FF07E53EC4A42
:10751000EC490390F9F785FF4590E8493B98F8F767
:107520001BFF4FF08043002259420390F9F779FF87
:107530004690E2493B98F8F70FFFE34B4FF07E523D
:10754000DF490390F9F76DFF4790DC493B98F8F766
:1075500003FFDD4B1A0200210390F9F762FF489008
:10756000D6493B98F8F7F8FED74A4FF07E51039082
:10757000F9F727FF4990D549CE480068F8F7ECFEA7
:10758000CF4AD0490390F9F7EDFE3C90CF49C94866
:107590000068F8F7E1FE00234FF04042C94903902C
:1075A000F9F73FFF3D90C949C2480068F8F7D4FE9B
:1075B0004FF07E53C24AC3490390F9F732FF3E9021
:1075C000C249BC480068F8F7C7FE4FF0804300226C
:1075D000594200E0CEE10390F9F723FF3F90BB4909
:1075E000B4480068F8F7B8FEB74B4FF07E52B44984
:1075F0000390F9F716FF4090B449AE480068F8F7D9
:10760000ABFEB14B1A0200210390F9F70AFF41903B
:10761000AE49A8480068F8F79FFEAB4A4FF07E518C
:107620000390F9F7CEFE429000BF14E000270FE070
:107630003CAA52F8271043AA52F826000FF038FE51
:10764000C6EBC6010AAA02EB810141F827007F1CA4
:10765000072FEDDB761C072EE8DB002619E000275C
:1076600014E0C6EBC6020AAB03EB820252F8271005
:10767000099AC2EBC20203EB8203089A53F8220074
:10768000F9F782F901D2099608977F1C072FE8DBEA
:10769000761C072EE3DB0998C0EBC0000AA901EBBA
:1076A0008001089851F8200007900998C0EBC000AD
:1076B000874901EB8001089851F820800998C0EBB8
:1076C000C000844901EB8001089851F82090099886
:1076D000C0EBC000804901EB8001089851F820A060
:1076E000B8F1000F06D17D4A7D49079836F0DEFDDE
:1076F00006903FE0B8F1010F07D10023794A78499D
:10770000079836F0F9FD069034E0B8F1020F07D182
:10771000754B724A7249079836F0EEFD069029E0E3
:10772000B8F1030F07D1714B00226E49079836F06C
:10773000E3FD06901EE0B8F1040F07D16C4B6A4AD6
:107740006649079836F0D8FD069013E0B8F1050FAA
:1077500007D1674B654A0021079836F0CDFD0690AA
:1077600008E0B8F1060F05D1614A5F49079836F085
:10777000B0FD0690B9F1000F06D1514A5149079862
:1077800036F094FD059044E0B9F1010F08D10023D3
:107790004FF040424B49079836F0AEFD059038E077
:1077A000B9F1020F08D14FF07E531A4645490798A8
:1077B00036F0A2FD05902CE0B9F1030F08D14FF08F
:1077C000804300225942079836F096FD059020E04C
:1077D000B9F1040F08D13C4B4FF07E52384907985D
:1077E00036F08AFD059014E0B9F1050F07D1364B4C
:1077F0001A020021079836F07FFD059009E0B9F1E3
:10780000060F06D1304A4FF07E51079836F061FDE1
:107810000590BAF1000F06D1364A3749079836F07D
:1078200045FD04903FE0BAF1010F07D10023334A30
:107830003149079836F060FD049034E0BAF1020F48
:1078400007D12F4B2B4A2C49079836F055FD049051
:1078500029E0BAF1030F07D12A4B002227490798E4
:1078600036F04AFD04901EE0BAF1040F07D1264B12
:10787000234A2049079836F03FFD049013E0BAF1FF
:10788000050F07D1204B1F4A0021079836F034FD21
:10789000049008E0BAF1060F05D11B4A1849079871
:1078A00036F017FD0490E06A0699F8F7FDFCE062F7
:1078B000206B2BE0D0020020000014400000A0400C
:1078C000000080BF000040C0000040400000F041C8
:1078D00084000020480100200C020020CDCCCCBD4B
:1078E0009A9999BECDCC4CBECDCCCC3DCDCC4C3EA6
:1078F0009A99993E0AD7A3BC8FC275BD0AD723BDFA
:107900000AD7A33C0AD7233D8FC2753D0499F8F7E7
:10791000CBFC206394F8480028B1606B0599F8F718
:10792000C3FC606301E0002060630021E06AF9F7B6
:107930002BF801D20020E0620021206BF9F724F837
:1079400001D200202063D4E90B01F8F7ADFC0390CD
:10795000616BF8F7A9FCA0634FF08040616BF8F70A
:10796000FBFC0390E16AF8F79FFC80F00040E063C5
:10797000606B20643C492846F9F710F806D2206A6B
:1079800020614FF0000B0120208552E03749284646
:10799000F8F7FAFF04D2606A20614FF0000B48E06C
:1079A00000BF25F0004032490390F8F7EDFF02D800
:1079B0004FF0000B3DE04FF07E512846F8F7E4FF12
:1079C00006D2208D012803D100202061208521E0EE
:1079D00085F000404FF07E510390F8F7DFFF02D2B0
:1079E000DFF890B016E0E169206CF8F7B5FC039081
:1079F000A169E06BF8F7B0FC01902946A06BF8F79D
:107A0000ABFC00900199F8F74FFC02900399F8F74E
:107A10004BFC83464FF07E515846F8F7BFFF01D824
:107A20004FF07E5B13495846F8F7AEFF01D8DFF8F8
:107A300044B0A069E061A56159462069F8F734FCBB
:107A40002061216A2069F8F7A9FF01D2206A20612C
:107A5000616A2069F8F798FF01D2606A20612069A5
:107A60004FB000F009B800000000A0400000A0C026
:107A70009A99993E000080BF30BCBDE8C08F2DE9C7
:107A8000F04F91B0044688469146C4F810804946AC
:107A90002069F8F75BFC0546276BE06AF8F715FFED
:107AA000CDE908012846F8F710FF21F00041CDE9A3
:107AB0000601DDE90823F8F733FF62D20D95284669
:107AC000616AF8F743FC0E904FF08041606AF8F766
:107AD00043FC29460990F8F73CFC8346A16AF8F775
:107AE000E3FB0F90A06CF8F7F0FE21F00041CDE928
:107AF0000601206CF8F7E9FE21F00041CDE9020112
:107B0000606CF8F7E2FE21F00041CDE90001DDE90B
:107B10000223F8F791FCCDE90401DDE90623F8F72B
:107B20008BFCCDE90801F8F713FF82465146606CE3
:107B3000F8F744FC0A905146206CF8F73FFC0B9094
:107B40005146A06CF8F73AFC0C900F990C98F8F796
:107B500003FC09900E990B98F8F7FEFB07900D991E
:107B60000A98F8F7F9FB06900799F8F79DFB08903B
:107B70000999F8F799FB83466169F8F7EDFB06462A
:107B800000E0002631463846F8F78EFB07463846B7
:107B9000A16BF8F703FF00D2A76B3846E16BF8F74B
:107BA000F3FE00D2E76B2763216B61630DAB3A46AE
:107BB00029462046FDF726FE616AA1626562606B78
:107BC00011B000F000B830BCBDE8C08F1C49897D01
:107BD000012906D002290ED0032918D0042914D176
:107BE0001EE0801DC11700EB117121F00F01401A3A
:107BF0000C2808DB09E0C11700EB917121F00301AB
:107C0000401A022801DA0120704700207047142131
:107C100090FBF1F201FB12000C28F4DB10380BE0B2
:107C2000182190FBF1F201FB12000C28EBDBA0F114
:107C300010010229E7D314380228E6D2E3E7000056
:107C40000C3000100FB4054B10B503A9044A02987C
:107C500002F0EAF810BC5DF814FB0000697E010830
:107C6000B00400200FB41CB50A46521ECDE9000234
:107C700007A9054B6A46069802F0D6F8009A00213B
:107C800011701CBC5DF814FB7FB000080FB4084BEA
:107C900010B504A902AA039802F0C6F8044602A986
:107CA000002003F01AFB204610BC5DF814FB000016
:107CB000DBB20008490050EAC12018BF04204A0D79
:107CC00018BF40F0010040F2FF72B2EB515F08BFF5
:107CD00040F00200012808BF05207047410008025B
:107CE00018BF04200A0E18BF40F001004FF07F4279
:107CF00032EA010108BF40F00200012808BF052058
:107D0000704700280DDB00BF00BF00F01F020121FB
:107D100091404209920002F1E022C2F8001100BF36
:107D200000BF704700280DDB00BF00BF00F01F023E
:107D3000012191404209920002F1E022C2F80011B3
:107D400000BF00BF704700280DDB00BF00BF00F080
:107D50001F02012191404209920002F1E022C2F883
:107D6000001100BF00BF704702480068C0F3022046
:107D7000704700000CED00E002480068C0F30220EC
:107D8000704700000CED00E002480068C0F30220DC
:107D9000704700000CED00E010B5002804DB0A0776
:107DA000130E054A135406E00A07140E034A00F0A6
:107DB0000F031B1FD45410BD00E400E018ED00E0D9
:107DC00010B5002804DB0A07130E054A135406E019
:107DD0000A07140E034A00F00F031B1FD45410BDF2
:107DE00000E400E018ED00E010B5002804DB0A070D
:107DF000130E054A135406E00A07140E034A00F056
:107E00000F031B1FD45410BD00E400E018ED00E088
:107E10002DE9F0414F1E00EBC7010446D1E90001F6
:107E200015461E4637F006020DD02A463346F8F7AF
:107E3000B2FB7F1E04EBC703D3E90023F8F7FCFA7B
:107E400037F00602F1D1022F25D0042F13D0062FD0
:107E500018BFBDE8F0812A463346F8F79CFBD4E909
:107E60000A23F8F7E9FA2A463346F8F794FBD4E9EF
:107E70000823F8F7E1FA2A463346F8F78CFBD4E9F1
:107E80000623F8F7D9FA2A463346F8F784FBD4E9F3
:107E90000423F8F7D1FA2A463346F8F77CFBD4E9F5
:107EA0000223F8F7C9FA2A463346F8F774FBD4E9F7
:107EB0000023BDE8F041F8F7BFBA000000221346E6
:107EC00010460149F8F7DCBB0000F03F0122F8F74B
:107ED00046BCF8F7B1BA0022134610461146F8F72F
:107EE000CFBB40F2013200204FF0E041F8F737BC41
:107EF000024A00201107F8F732BC000001FDFFFF25
:107F000000214FF07E50F8F759BAF8F7CDB90021AB
:107F10000846F8F753BA61214FF0E040F8F7FABD90
:107F20006FF05E010807F8F7F5BD02E008C8121F00
:107F300008C1002AFAD170477047002001E001C152
:107F4000121F002AFBD170470149086070470000EA
:107F5000740200102DE9FC4104460CB1012100E03F
:107F60000021084640F26F21F9F79AF925462C4680
:107F70002E686F68D7E90401CDE900016868D0F880
:107F80000CC097E80F00E047204609F03AFBD6E91D
:107F90000401CDE900012868D0F808C096E80F0078
:107FA000E047204609F02DFBD6E90401CDE90001A8
:107FB0002868D0F80CC096E80F00E047BDE8FC81C7
:107FC00021490968096DB1F8BC1001801E49096892
:107FD000096DB1F8BE1041801B490968096DB1F8FF
:107FE000B810818018490968096DB1F8BA10C180CC
:107FF00015490968096DB1F8C41001811249096871
:10800000096DB1F8C61041810F490968096DB1F8D1
:10801000C81081810C490968096DB1F8CA10C18185
:1080200009490968096DD1F8D41001610649096848
:10803000096DD1F8D810416103490968096DD1F87B
:10804000DC108161704700006001001010B504462B
:108050001F480068006A808820801D480068006A08
:10806000C08860801A480068006AC089A0801848EB
:108070000068006A008AE08015490968096A086A90
:10808000F8F7D7FB208112490968096A486AF8F7AE
:10809000D0FB60810E490968096AC86BF8F7C9FB13
:1080A000A0810B490968096A086CF8F7C2FBE081F6
:1080B00007480068006A806A206105480068006A15
:1080C000C06A606102480068006A006BA06110BD70
:1080D0002002001010B5044625480068D0F8F400CE
:1080E0004088208022480068D0F8F40080886080B2
:1080F0001F480068D0F8F400408AA0801C4800683F
:10810000D0F8F400008AE08019490968D1F8F41029
:10811000486FF8F78EFB208115490968D1F8F410F3
:10812000886FF8F786FB608111480068D0F8F4008A
:10813000B0F86C00A0810E480068D0F8F400B0F8E8
:108140007000E0810A480068D0F8F400C06F206138
:1081500007480068D0F8F400D0F880006061044857
:108160000068D0F8F400D0F88400A06110BD0000D1
:108170002004002070B50446254800688068808887
:108180002080234800688068C08860802049096892
:108190008968086AF8F74DFBA0801D49096889685D
:1081A000486AF8F746FBE080194909688968086A57
:1081B0001849F8F703F90546F8F73BFB2081144905
:1081C00009688968486A1349F8F7F8F80546F8F726
:1081D00030FB60810E49096889684869F8F729FB16
:1081E000A0810B49096889688869F8F722FBE0815A
:1081F000074800688068006B206105480068806857
:10820000406B6061024800688068806BA06170BD4F
:108210002402001000007A4403480068807C012892
:1082200000D170470020FCE760010010034800689F
:10823000007F012800D170470020FCE720020010D9
:10824000044800680078032801D10120704700200D
:10825000FCE70000200400200448006800790228A0
:1082600001D1012070470020FCE70000240200102B
:108270000C480068006D90F8AC00012802D10A4952
:10828000C8740CE007480068006D90F8AC00022844
:1082900002D10549C87402E003200349C8740248AA
:1082A000C07C70476001001098710010054800689C
:1082B000007F012800D1704702480068006A4078BA
:1082C000F9E70000200200100C480068D0F8F40024
:1082D0000078012802D10A49C8740CE007480068F8
:1082E000D0F8F4000078022802D10549C87402E0F1
:1082F00003200349C8740248C07C70472004002052
:1083000098710010054800680079022801D1012009
:1083100070470248006880680078F9E7240200107E
:1083200000B501202FF0CEFE00BD10B5012028F0D1
:10833000ABF910BD10B5032008F0DAFF10BD10B581
:1083400002202FF03DFF10BD014800688078704783
:108350006001001008207047052070470820704712
:108360000148006800787047640100100148006807
:10837000C07F7047200200100248006890F87D001E
:108380007047000020040020014800680078704712
:108390002402001000B502202FF094FE00BD000062
:1083A00010B508480068007F012806D1022028F097
:1083B0006BF90320044981F836010821014800685F
:1083C000C17710BD200200109871001010B5042074
:1083D00008F08EFF10BD10B503202FF0F1FE10BD88
:1083E00004480068006A4078022801D101207047E3
:1083F0000020FCE7200200100120704710B5002289
:10840000002801DA01224042002902DA42F0020289
:108410004942814204DD0B460146184642F00402FF
:10842000890200EBD07301EB630191FBF0F0801047
:108430000311124C00F00F00C0F1100134F81300CA
:1084400010FB01F0102906D004EB4303C1F1100129
:108450005B8813FB01000830C11700EB117000119D
:10846000510701D5C0F58060D10701D0C0F500608B
:10847000910701D5C0F5805010BD00006E030508BE
:108480002DE9F041064606F1540406F1080520786E
:10849000C0F38100012802D1304635F0D1FE00271B
:1084A000A068401CA060A188A06848434FF47A717E
:1084B000B0FBF1F7B7F5167F0ED9207820F0030056
:1084C000801C2070207820F00C00001D2070207887
:1084D00000F00300BDE8F0812A6811686A6810683E
:1084E000F8F75CFA1CD8A078401CA0700020E0705F
:1084F000A07806282FDDA968286A08602078C0F3D4
:10850000401040BB207820F02000203020706078A0
:10851000401C6070607803281DD1A068E0601AE0FC
:108520000020A070E078401CE070E078062812DDA2
:10853000A968686A08602078C0F3401058B12078B4
:1085400020F0200020706078401C60706078032864
:1085500001D1A068E060607803281BD12078C0F3C7
:10856000001048B1E1692A681068F8F70DFA3FD2A7
:1085700028680068E0613BE02078C0F3001038BB59
:10858000A1692A681068F8F709FA31D228680068EA
:10859000A0612DE0607804281BD12078C0F3001082
:1085A00048B1A1692A681068F8F7F8F920D228685C
:1085B0000068A0611CE02078C0F3001040B9E169B8
:1085C0002A681068F8F7E0F912D228680068E061BC
:1085D0000EE0607805280BD1304606F0A1FD20782A
:1085E00020F003002070207820F00C00001D207087
:1085F000207800F003006DE77047000010B50446D6
:108600000CB1012100E0002108464F21F8F748FE97
:10861000616809B1012100E0002108465021F8F706
:108620003FFE0121204633F081FB5621204633F0E6
:10863000B3FB0021204633F0AFFB0021204633F08E
:10864000ABFB0021204633F071FB0020A075228A8D
:1086500001210348006801F084F9002010BD0000EA
:10866000CC0100102DE9F05F04460E461746E08964
:10867000C11700EB51714FEAE109E089C11700EB26
:1086800051714FEAE10BD4F818A0354611E0B4F867
:108690000E804FEAE87108EB5171CA1009FB05A082
:1086A000FF2101F05EF90120044909684855681C62
:1086B00085B2BD42EBDB00F003B80000CC01001036
:1086C00030BCBDE8C09F70B50646DDE9044500201A
:1086D00070BD0120704700000848006800F12401C7
:1086E00006480068007F30B991F80C01012800D1DC
:1086F00070470020FCE70120FAE70000200200108C
:1087000010B50B480068007801280FD108490968A6
:10871000886C20F000410C464FF07C512046F8F761
:1087200033F901D8012010BD0020FCE70120FAE751
:10873000200400202DE9F0410E4C0F48006800791C
:10874000B0B90E49D1F8E401F8F7BFF805460E4676
:10875000A06FF8F7BAF821F0004107462A463346E1
:10876000F8F7C6F802D80120BDE8F0810020FBE749
:108770000120F9E77C03001024020010987100101A
:108780002DE9F04104460D46E089C11700EB517117
:10879000C910228A51438EB22DB93246A169206A8E
:1087A00001F033F82EE0012D1CD1002012E0216AE7
:1087B000095CA269125C91420AD0E189CA1701EBF7
:1087C0005272D21090FBF2F20F4B1B6801279F549C
:1087D000411C88B2B042EADB3246216AA06901F04E
:1087E00014F80FE03246FF21A06901F0BAF83246D2
:1087F000FF21206A01F0B5F8228A012102480068B1
:1088000001F0AFF8BDE8F081CC01001010B511F017
:10881000BBFD01210170002021F0A0F810BD000077
:108820002DE9F04705460C4690461F46DDE90869EC
:108830000DB1012100E0002108468821F8F730FD44
:108840000CB1012100E0002108468921F8F728FD3C
:10885000A96D09B1012100E0002108468A21F8F73D
:108860001FFD6C67C5F87880EE67012085F88000F1
:1088700085F881000FB1C5F88470B9F1000F01D0FF
:10888000C5F88890A96D01F10C0000BF2146114A7E
:10889000925D0A44906000BF00BF0120606000BF8D
:1088A00000BF0220606000BF00BF20460949895D0B
:1088B000415841F00201074A925D815000BFA86D06
:1088C000416841F00201416000BFA86DFBF763FA07
:1088D000BDE8F087CC0105082DE9F04788B0814656
:1088E0000C4615460027A2461EE004F12000A842CF
:1088F00002D24FF0200801E0A5EB040843466A4687
:108900002146484600F02FF800260AE0FF2F05D048
:108910001DF80600FF2801D104EB060A1DF80670B9
:10892000761C4645F2D32034AC42DED3FF2F03D170
:10893000504608B0BDE8F0872846FAE72DE9F04137
:1089400004460D4616460027607E10B10120BDE8A2
:10895000F08132462946A0680EF090FA002800DA2D
:1089600001273846F3E72DE9F04104460D46164647
:108970001F464FF00008607E10B10220BDE8F08174
:108980003B4632462946A0680EF054FB002801DA27
:108990004FF002084046F1E72DE9F04704460D4646
:1089A00016461F46DDF820904FF00008607E10B19B
:1089B0000320BDE8F0873B4632462946A0680EF00A
:1089C000D7FB002801DA4FF003084046F1E770B505
:1089D00002460023481E014604460AE002EBD1008D
:1089E000007801F0070680253541284000B904E0F1
:1089F0005B1C081EA1F10101F0D100BFE01A70BD9F
:108A00002DE9F04704460D4616469846DDF82090BD
:108A10000CB900BFFEE70DB900BFFEE70EB900BFFD
:108A2000FEE7207E10B10020BDE8F087256084F8C5
:108A30000480C4F82490607EF0B90EF095F93046B9
:108A40000EF0B6FAA06008B90420EDE7A16801F1C4
:108A50001C000EF053F9076AE06808B9E76007E008
:108A6000E068B0FBF7F107FB110008B10820DBE775
:108A7000A068806B206100BFE068411E084008B11B
:108A800000BFFEE7D4E90310B0FBF1F201FB1200D6
:108A900008B10820C8E7D4E90310B0FBF1F00228C0
:108AA00001D20820C0E70020BEE7000041B9012242
:108AB0000276044A127822B90122024B1A7000E0B1
:108AC00000BF70472804002030B5A1B0044600253F
:108AD00000200490012084F8310000201D4904ABDF
:108AE0000246CDE90041029005A9204631F04CFF35
:108AF000A07E20B1049810B1022021B030BDD4E98D
:108B00000310B0FBF1F00499884202D120460EF028
:108B10003AFC00201049CDE900012346024605A990
:108B20000290204631F030FF00BF0C48002322465F
:108B30000BA9009020461BF0D9FE94F8300018B124
:108B4000204610F080FDF0E7002084F83100284630
:108B5000D3E70000A7F800085BF7000883F70008D8
:108B60002DE9F04106460F4615461C460DB900BFDB
:108B7000FEE7E01DC3082A4639463046FFF7F3FEFC
:108B800021462846FFF723FFBDE8F0812DE9F0419B
:108B900005460E4614464FF0FF37F01DC108FF2270
:108BA0002846F7F73FFB44B1601EC708E85D04F0B4
:108BB0000702FF2111410840E8553846BDE8F08121
:108BC0002DE9F84F81460F4615461E46DDE90A8A13
:108BD0004FF0000BB04501D300BFFEE70DB900BF59
:108BE000FEE7424631462846FFF7D0FF0446601CA8
:108BF00010B9002000F00BB82A1939190123484692
:108C0000CDF800A0FFF7C8FE83465846F2E718BC2F
:108C1000BDE8E08F70B50646DDE90445002070BD73
:108C200070B504460D460026012C06D0022C0BD050
:108C3000032C10D0042C1CD114E029460F480068E6
:108C400034F033FD064615E029460D48006834F03F
:108C50002CFD06460EE029460A48006834F025FD42
:108C6000064607E029460848006834F01EFD06461F
:108C700000E000BF00BF304670BD0000A40000103F
:108C8000A8000010AC000010B00000102DE9F04169
:108C900004460D4616460027012C06D0022C0CD0A7
:108CA000032C12D0042C20D117E03246294611485B
:108CB000006834F0CDFC074618E0324629460E48DD
:108CC000006834F0C5FC074610E0324629460B48E0
:108CD000006834F0BDFC074608E0324629460848E3
:108CE000006834F0B5FC074600E000BF00BF38461E
:108CF000BDE8F081A4000010A8000010AC00001036
:108D0000B000001070B504460D460026012C06D0B8
:108D1000022C17D0032C28D0042C4CD138E0294643
:108D20002748006834F010FD0646294624480068AC
:108D300034F011FC28B92348407820F02000214964
:108D4000487039E029462048006834F0FDFC0646AA
:108D500029461D48006834F0FEFB28B919484078C0
:108D600020F040001749487026E02946174800685F
:108D700034F0EAFC064629461448006834F0EBFB60
:108D800028B91048407820F080000E49487013E060
:108D900029460F48006834F0D7FC064629460C489F
:108DA000006834F0D8FB28B90648807820F001002C
:108DB0000449887000E000BF00BF304670BD00006D
:108DC000A400001078020010A8000010AC000010F1
:108DD000B00000102DE9F04104460D46164600276C
:108DE000012C06D0022C19D0032C2CD0042C54D1E9
:108DF0003EE0324629462B48006834F078FC0746AE
:108E0000324629462748006834F05CFB28B92648DA
:108E1000407820F02000244948703FE0324629463F
:108E20002248006834F063FC0746324629461F4852
:108E3000006834F047FB28B91B48407820F0400018
:108E4000194948702AE0324629461948006834F02A
:108E50004EFC0746324629461548006834F032FB7E
:108E600028B91148407820F080000F49487015E07B
:108E7000324629460F48006834F039FC074632462E
:108E800029460C48006834F01DFB28B90648807854
:108E900020F001000449887000E000BF00BF3846A0
:108EA000BDE8F081A400001078020010A8000010B6
:108EB000AC000010B00000102DE9FF5F044634F054
:108EC0003FFE60620020029001900090207D4FFAEA
:108ED00080F90CB1012100E000210846B721F8F724
:108EE000DFF9616809B1012100E000210846B821DD
:108EF000F8F7D6F9B4F810A0E089C11700EB51716A
:108F0000CF10E089C11700EB51714FEAE108E08909
:108F1000C11700EB5171C9100391D4F818B0E5697D
:108F2000932005F8010B00261CE0701C80B2029013
:108F30002B480068A0B12A480068805D01280FD145
:108F4000029805F8010B08FB06B13A46284600F0E6
:108F50005CFC3D44002005F8010B21490968885557
:108F6000701C86B25645E0DB002005F8010B05F8C1
:108F7000010BE069281A0190002184F87010019813
:108F800004281ED916E00121204632F0CFFEA68B20
:108F9000AE1BB2B2E1696068436D98470090002152
:108FA000204632F0C3FE0A20FBF72BFA0098012876
:108FB00000D105E0A9F1010040B2B0F10009E2DC06
:108FC00000BFB9F1000F00DC00BF34F0B9FD616AE9
:108FD000401A6062012184F8701000F003B80000AC
:108FE000CC0100103FBCBDE8C09F000070B5044636
:108FF0002046216C8847E089C11700EB5171C910E8
:10900000228A51438DB22A46FF21A06900F0A9FCB3
:10901000228A01210248006800F0A3FC70BD000014
:10902000CC0100102DE9FF5FDDE90220010DDDF824
:1090300038B0024318D044F61050A1F2FF3141433A
:109040000D140F98012820D0A5EB0B00401C5FEAFF
:10905000000A4FF00004474EDFF81C91A04650462E
:1090600016D5CAF1000728E00F98012443A2012871
:1090700008D0002100980F9BC0E90021C0E90243FD
:1090800000F082B86FEA0B01F4E7CBF10000DEE7F5
:10909000074612E0F80707D02246334640464946C5
:1090A000F7F779FA80468946224633461046194634
:1090B000F7F771FA04460E467F10002FEAD1DDE97A
:1090C0000201BAF1000F42464B4602DAF7F763FAA3
:1090D00001E0F7F7D5FA04460E460022284BF7F7D1
:1090E0001FFC03D84FF0FF30014607E00022254B5C
:1090F00020463146F7F7A0F9F7F7C2FD102409E042
:10910000002C0ADB0A220023F7F768FC019B3032AF
:109110001A55641E50EA0102F2D1641C019AC4F18E
:10912000110314440F9A012A03D0012208430DD1E0
:109130000AE0084304D000204FF0110B0F9080E7A5
:10914000A3EB0B056D1E0DE05B4504DD4FF0000247
:1091500005F1010504E003DA4FF00002A5F1010575
:10916000002AECD000980F99C0E90231C0E900450F
:1091700086E70000000024400000F03F30000000BF
:109180000000F0430000E03F3FBCBDE8C09F00008E
:1091900010B5044600BF0548FAF7ABFE0348FAF7DE
:1091A000BCFE00BF204619F03FFC10BD004401404A
:1091B00010B504462146002029F024F910BD10B551
:1091C00004462146002029F01DF910BD10B50446C3
:1091D0002146002029F016F910BD10B5044621469D
:1091E000002029F00FF910BD10B5044621460020DB
:1091F00029F008F910BD10B504462146002029F0D9
:1092000001F910BD10B504462146002029F0FAF8F6
:1092100010BD10B504462146002029F0F3F810BD1A
:1092200010B504462146002029F0ECF810BD10B519
:1092300004462146002029F0E5F810BD10B504468B
:109240002146002029F0DEF810BD10B50446214665
:10925000002029F0D7F810BD70B504460D46E0890E
:10926000C11700EB5171C910228A51438EB2E9B285
:109270003246A06900F075FB228A0121024800688D
:1092800000F06FFB70BD0000CC0100100146887D2E
:1092900070470146C87C704770B50446A06B012832
:1092A0000AD10648D4F88811F7F756F80546D4F8DD
:1092B0008C11F7F751F870BD0020FCE79A99993DA1
:1092C00070B50446A06B01280AD10C48D4F8881167
:1092D000F7F742F80646D4F88C11F7F76FF809E073
:1092E0000748D4F88811F7F737F80646D4F88C11F8
:1092F000F7F764F80546284670BD00009A99993F33
:109300008FC2F53E70B50446A06B012805D1074811
:10931000D4F88811F7F720F804E00548D4F888114C
:10932000F7F71AF80546284670BD00009A99193FCC
:10933000CDCCCC3E2DE9F0470346154608464FEA12
:10934000E17901EB59794FEAE909A1EBC90909F083
:10935000FF060120B040C7B2D8894FEAE07900EBA0
:1093600059794FEAE904D8894FEAE07900EB597955
:109370004FEAE908D3F818C04FEAE17901EB5979CF
:109380004FEAE90904FB05CA1AF8099009EA070936
:10939000B9F1000F02D0FF20BDE8F0870020FBE705
:1093A0002DE9FC4704460D4616461F46DDE90A89AD
:1093B0003B46324629462046CDE9008911F050FA55
:1093C00000F000B80CBCBDE8F08710B58AB004A866
:1093D00005A906AB07AACDE9001008A909A8FFF75F
:1093E000DFFF9DF82400ADF80C009DF820008DF8FB
:1093F0000E009DF81C008DF80F009DF818008DF8E8
:1094000008009DF814008DF809009DF810008DF8F3
:109410000A0002A903A834F099FD044620460AB0C8
:1094200010BD70B504460D460CB1012100E00021CD
:1094300008467E21F7F734FF0DB1012100E000213D
:1094400008467F21F7F72CFF002084F85C00A56513
:109450002846FAF7A0FC70BD2DE9F04704464FF00E
:1094600000080025A946002794F8980058B900265E
:1094700004F14406D6F84C80B56AD6E90010F6F738
:1094800065FF81460BE0002604F14406D6F82880EB
:10949000756AD6E90010F6F759FF814600BF4146CC
:1094A0004846F6F701FF074694F89B00012817D1BC
:1094B00000213846F7F772FA10D800212846F7F74E
:1094C00063FA02D285F0004000E02846064639469D
:1094D000F7F764FA02D80120BDE8F0870020FBE727
:1094E00094F99B00401C68B900213846F7F74CFA04
:1094F00006D829463846F7F751FA01D80120EBE79C
:109500000020E9E700212846F7F73EFA02D285F06D
:10951000004000E02846064600213846F7F734FAB6
:1095200002D287F0004000E0384682463146F7F725
:109530002BFA01D80120CFE70020CDE703490968C5
:10954000098F0144014A126811877047A004002066
:1095500070B50446FF20A074E089C11700EB51717B
:10956000C910228A51438EB21548A0611548E061A6
:10957000154820623246FF21A06900F0F2F9324618
:10958000FF21E06900F0EDF93246FF21206A00F08A
:10959000E8F9258A2946002028F05EFF0B4908607B
:1095A000228A00210948006800F0DBF901212046E9
:1095B000A26C90472046A16D8847002070BD000036
:1095C000B80400209833002080C00020CC01001097
:1095D00010B504462146002028F03EFF10BD10B50E
:1095E00004462146002028F037FF10BD10B5044680
:1095F0002146002028F030FF10BD10B5044621465A
:10960000002028F029FF10BD10B504462146002097
:1096100028F022FF10BD10B504462146002028F096
:109620001BFF10BD10B504462146002028F014FF92
:1096300010BD10B504462146002028F00DFF10BDD6
:1096400010B504462146002028F006FF10BD30B5B5
:10965000034608E013F8014B11F8015BAC4202D05D
:109660004FF0FF3030BD101EA2F10104A2B2F1D1C3
:1096700000BFF7E730B5034608E013F8014B11F8D7
:10968000015BAC4202D04FF0FF3030BD101EA2F1A2
:109690000104A2B2F1D100BFF7E730B5034608E0FC
:1096A00013F8014B11F8015BAC4202D04FF0FF30D0
:1096B00030BD101EA2F10104A2B2F1D100BFF7E744
:1096C00030B5034608E013F8014B11F8015BAC42DA
:1096D00002D04FF0FF3030BD101EA2F10104A2B243
:1096E000F1D100BFF7E730B5034608E013F8014BAE
:1096F00011F8015BAC4202D04FF0FF3030BD101EBC
:10970000A2F10104A2B2F1D100BFF7E730B50346E0
:1097100008E013F8014B11F8015BAC4202D04FF0A6
:10972000FF3030BD101EA2F10104A2B2F1D100BF82
:10973000F7E710B503E011F8013B00F8013B131EF9
:10974000A2F10104A2B2F6D110BD10B503E011F8E8
:10975000013B00F8013B131EA2F10104A2B2F6D1B5
:1097600010BD10B503E011F8013B00F8013B131EDA
:10977000A2F10104A2B2F6D110BD10B503E011F8B8
:10978000013B00F8013B131EA2F10104A2B2F6D185
:1097900010BD10B503E011F8013B00F8013B131EAA
:1097A000A2F10104A2B2F6D110BD10B503E011F888
:1097B000013B00F8013B131EA2F10104A2B2F6D155
:1097C00010BD10B503E011F8013B00F8013B131E7A
:1097D000A2F10104A2B2F6D110BD10B503E011F858
:1097E000013B00F8013B131EA2F10104A2B2F6D125
:1097F00010BD10B503E011F8013B00F8013B131E4A
:10980000A2F10104A2B2F6D110BD10B503E011F827
:10981000013B00F8013B131EA2F10104A2B2F6D1F4
:1098200010BD10B503E011F8013B00F8013B131E19
:10983000A2F10104A2B2F6D110BD10B503E011F8F7
:10984000013B00F8013B131EA2F10104A2B2F6D1C4
:1098500010BD10B503E011F8013B00F8013B131EE9
:10986000A2F10104A2B2F6D110BD10B503E011F8C7
:10987000013B00F8013B131EA2F10104A2B2F6D194
:1098800010BD10B503E011F8013B00F8013B131EB9
:10989000A2F10104A2B2F6D110BD10B501E000F8AA
:1098A000011B131EA2F10104A2B2F8D110BD10B524
:1098B00001E000F8011B131EA2F10104A2B2F8D1CD
:1098C00010BD10B501E000F8011B131EA2F1010448
:1098D000A2B2F8D110BD10B501E000F8011B131EB3
:1098E000A2F10104A2B2F8D110BD10B501E000F858
:1098F000011B131EA2F10104A2B2F8D110BD10B5D4
:1099000001E000F8011B131EA2F10104A2B2F8D17C
:1099100010BD10B501E000F8011B131EA2F10104F7
:10992000A2B2F8D110BD10B501E000F8011B131E62
:10993000A2F10104A2B2F8D110BD10B501E000F807
:10994000011B131EA2F10104A2B2F8D110BD10B583
:1099500001E000F8011B131EA2F10104A2B2F8D12C
:1099600010BD10B501E000F8011B131EA2F10104A7
:10997000A2B2F8D110BD10B501E000F8011B131E12
:10998000A2F10104A2B2F8D110BD10B501E000F8B7
:10999000011B131EA2F10104A2B2F8D110BD10B533
:1099A00001E000F8011B131EA2F10104A2B2F8D1DC
:1099B00010BD10B501E000F8011B131EA2F1010457
:1099C000A2B2F8D110BD10B501E000F8011B131EC2
:1099D000A2F10104A2B2F8D110BD10B501E000F867
:1099E000011B131EA2F10104A2B2F8D110BD10B5E3
:1099F00001E000F8011B131EA2F10104A2B2F8D18C
:109A000010BD10B501E000F8011B131EA2F1010406
:109A1000A2B2F8D110BD10B501E000F8011B131E71
:109A2000A2F10104A2B2F8D110BD10B501E000F816
:109A3000011B131EA2F10104A2B2F8D110BD10B592
:109A400001E000F8011B131EA2F10104A2B2F8D13B
:109A500010BD10B501E000F8011B131EA2F10104B6
:109A6000A2B2F8D110BD10B501E000F8011B131E21
:109A7000A2F10104A2B2F8D110BD10B501E000F8C6
:109A8000011B131EA2F10104A2B2F8D110BD10B542
:109A900001E000F8011B131EA2F10104A2B2F8D1EB
:109AA00010BD10B501E000F8011B131EA2F1010466
:109AB000A2B2F8D110BD10B501E000F8011B131ED1
:109AC000A2F10104A2B2F8D110BD10B501E000F876
:109AD000011B131EA2F10104A2B2F8D110BD10B5F2
:109AE00001E000F8011B131EA2F10104A2B2F8D19B
:109AF00010BD01460A4600E0521C10780028FBD138
:109B0000501A704701460A4600E0521C107800289F
:109B1000FBD1501A704701460A4600E0521C1078EB
:109B20000028FBD1501A704701460A4600E0521C3B
:109B300010780028FBD1501A70472DE9FC410446EB
:109B40000CB1012100E00021084640F28B21F7F71B
:109B5000A7FB25462C462E686F68D7E90401CDE99E
:109B600000016868D0F808C097E80F00E047204679
:109B700007F047FDD6E90401CDE900012868D0F8D7
:109B800008C096E80F00E047204607F03AFDD6E906
:109B90000401CDE900012868D0F80CC096E80F0058
:109BA000E047BDE8FC812DE9FC4104460D46A07C60
:109BB000A8421AD0A574012D0CD1A168D1E90401E5
:109BC000CDE90001A668D6E902733A46D6E900015C
:109BD000B8470AE0A168D1E90401CDE90001A6680F
:109BE000F7683B4696E80700B8470020BDE8FC81CF
:109BF00010B501201FF0B2FE10BD70B504460D4631
:109C0000164694F8980028B932462946204629F08D
:109C1000CFFE70BD32462946204619F039FDF8E7DF
:109C20002DE9FE430446894633F08AFFE0670021B0
:109C3000802001514846F6F748FE21F000410546D4
:109C4000704A714BF6F754FE01D24FF00009C4F888
:109C50003090E16E606EF6F7A1FE15D2A16A206B1E
:109C6000F6F79CFE05D20021606AF6F71DFB6062E4
:109C70004BE00021206BF6F787FE46D2216B606A2D
:109C8000F6F712FB606240E0216F606EF6F77CFE33
:109C900015D2A16A206BF6F781FE05D20021606A19
:109CA000F6F702FB606230E00021206BF6F776FEEB
:109CB0002BD2216B606AF6F7F7FA606225E0A06AA2
:109CC000F6F703FE05460E464846F6F7FEFD21F080
:109CD000004107462A463346F6F722FE0AD3484695
:109CE000F6F7F3FD21F0004105460022474BF6F759
:109CF000FFFD05D20021606AF6F7D6FA606204E043
:109D0000216B606AF6F7D0FA6062606DF6F7DDFDF0
:109D100005460E464846F6F7D8FD21F000410746B5
:109D20002A463346F6F7E4FD1BD2206B0090606AAA
:109D300001900299A06CF6F70FFB06460199606C42
:109D4000F6F70AFB07460099A06BF6F705FB80467D
:109D50003946F6F7A9FA05463146F6F7A5FA6066E0
:109D60003AE0206B0090606A019033F0E9FE8021B8
:109D7000085180200059E16F091AE167E06FF6F79A
:109D800032FD07460022224BF6F77AFC0546F6F72D
:109D900083FDE067E06FF6F710FD05462B46494668
:109DA0001C48226A34F082F802900299A06CF6F7FF
:109DB000D3FA06460199606CF6F7CEFA0746009989
:109DC000A06BF6F7C9FA80463946F6F76DFA0546F4
:109DD0003146F6F769FA6066E16E606EF6F7DEFD11
:109DE00001D2E16E6166216F606EF6F7CDFD01D2A2
:109DF000216F6166216B2162616EA166606E00F069
:109E00000BB800009A9999999999B93F0000E03FE1
:109E100000408F401403001006BCBDE8F88330B545
:109E20000546039C002030BD2DE9FF4F95B09B46B1
:109E30008946064600250FE2252877D100242746CB
:109E4000F84A0121059400E0044316F8013F203B45
:109E500001FA03F01042F7D130782A2811D06FF0C0
:109E60002F033078A0F13002092A16D8059A44F061
:109E7000020402EB820203EB42021044761C0590BE
:109E8000EFE759F8042B0592002A03DA504244F414
:109E90000054059044F00204761C30782E2816D128
:109EA00016F8010F44F004042A280DD06FF02F0299
:109EB0003078A0F13003092B09D807EB870302EBB8
:109EC0004303C718761CF3E759F8047B761C3078F7
:109ED0006C280FD006DC4C2817D068280DD06A28D3
:109EE00014D104E0742810D07A280FD10DE044F486
:109EF00000140AE044F4801401E044F44014727841
:109F0000824202D104F58014761C761C30786628D3
:109F10000BD013DC582877D009DC002875D04528F1
:109F2000F6D04628F4D047281AD19DE118E06328DE
:109F300035D0642879D0652812D195E1702873D086
:109F400008DC6728F1D069286FD06E280DD06F2803
:109F500006D1B5E073282CD0752875D0782874D038
:109F60005A46179990476D1C75E1C4F302500228B8
:109F700009D003280DD0D9F8001004280DD00D60A9
:109F800009F1040967E1D9F80010EA17C1E90052A4
:109F9000F6E7D9F800100D80F2E70D70F0E719F838
:109FA000041B8DF8001000208DF80100EA46012006
:109FB00003E059F804AB4FF0FF3061074FF00001A8
:109FC00002D40DE008F101018846B9420FDA80455C
:109FD000F8DB1AF808100029F4D108E008F10101B3
:109FE00088468142FADB1AF808100029F6D1059854
:109FF0005B46A0EB080721463846179A00F097FA0F
:10A00000284400EB080507E04DE029E10DE01AF8CF
:10A01000010B5A4617999047B8F10108F7D25B46F1
:10A0200021463846179A13E142E00A220092C4F30F
:10A0300002524FF0000A022A08D059F804CB032A32
:10A040004FEAEC710AD00DE029E02AE009F107019E
:10A0500021F00702F2E802C1914609E00FFA8CFCF8
:10A060004FEAEC71042A03D14FFA8CFC4FEAEC71F1
:10A07000002907DA0A460021DCF1000C61EB02013D
:10A080002D2202E0220504D52B228DF80420012286
:10A0900003E0E20701D02022F7E7904659E00A21C9
:10A0A00002E010220DE010214FF0000A00910BE0B9
:10A0B00010224FF0000A44F004040827009203E045
:10A0C00008224FF0000A0092C4F30252022A05D07F
:10A0D00059F804CB0021032A08D009E009F107014F
:10A0E00021F00702F2E802C1914605E01FFA8CFC5C
:10A0F000042A01D10CF0FF0C4FF00008220728D5EC
:10A10000702806D0009B83F0100353EA0A0305D0A1
:10A110000EE040228DF80420012208E05CEA0102F2
:10A1200006D030228DF804208DF8050002229046DA
:10A13000009B83F0080353EA0A030AD15CEA010298
:10A1400001D1620705D530228DF804204FF00108B7
:10A150007F1E582804D034A003900EA802900DE072
:10A1600036A0F9E753466046009AF6F737FC844676
:10A170000398825C0298401E029002705CEA010023
:10A18000F0D1029806A9081A00F1200A600702D54A
:10A1900024F4803400E00127574502DDA7EB0A00D4
:10A1A00000E0002000EB0A01009005984144401AAD
:10A1B0000590E00306D45B462146179A059800F007
:10A1C000B6F90544002706E001A85A46C05D179974
:10A1D00090476D1C7F1C4745F6DBE0030CD55B46C2
:10A1E0002146179A059800F0A2F9054404E03020B2
:10A1F0005A46179990476D1C0099481E00900029F7
:10A20000F5DC08E0029802995A460078491C029150
:10A21000179990476D1CBAF10001AAF1010AF1DC0F
:10A2200065E100000928010030313233343536371A
:10A230003839616263646566000000003031323392
:10A240003435363738394142434445460000000032
:10A2500000F05BF90544761C307800287FF4ECAD03
:10A2600019B0284600F04EB9620700D4062709F15C
:10A27000070222F0070CFCE80223E14603F0004845
:10A280005FEA080C02D00FF2702C0DE05FEA045C6C
:10A2900002D50FF2682C07E05FEAC47C02D00FF20F
:10A2A000602C01E0AFF2700C4FF0FF3823F0004358
:10A2B000CDF850C065280CD006DC452809D04628CA
:10A2C0001DD047283DD13DE0662818D067287ED1B3
:10A2D00038E00021112F01DB112000E0781CCDE9CE
:10A2E000000106A90EA8FEF79DFEDDE90F010E9AFA
:10A2F00003910021009207F1010A04914DE04FF013
:10A3000000400097CDE9011006A90EA8FEF78AFECD
:10A31000DDE90F0203920E9B11990022DDF80CA0DB
:10A320000093049211B9791C00EB010AB7EB0A0003
:10A3300004D4C0F1FF3007F1010A0490AAEB070032
:10A34000019044E0012F00DA01270021112F01DDE7
:10A35000112000E03846CDE9000106A90EA8FEF75D
:10A3600061FEDDE90F010E9A039100210491009234
:10A37000BA4621070CD40399514500DA8A46BAF14E
:10A38000010F05DD009AAAF10101515C302908D0C6
:10A39000B84202DA10F1040F06DA0121CDE901100A
:10A3A00015E0AAF10101E9E7002805DC0499014460
:10A3B0000491AAEB000102E0411C514500DD8A46F0
:10A3C0000499401A401C01904FF000400290200771
:10A3D00004D40198504501DBCDF8048000208DF8AD
:10A3E0004F0002980DF14F07B0F1004F25D02B2000
:10A3F0000E9002984FF0020800280CDA40420290BA
:10A400002D200E9007E00A210298F6F7D1FA30319C
:10A41000029007F8011DB8F10001A8F10108F2DC73
:10A4200002980028EFD1791E0E980870307800F05D
:10A43000200040F0450007F8020D12A8C01B00F1F3
:10A4400007081498007800B1012000EB0A01019878
:10A4500001EBE07105984144401A401E0590E0036D
:10A4600006D45B462146179A059800F060F805442B
:10A470001498007818B15A46179990476D1CE0035C
:10A4800024D55B462146179A059800F050F80544FC
:10A490001CE00498002807DBDDE90301884203DDA6
:10A4A0000098405C179901E0179930205A46904770
:10A4B000049805F10105401C04900198401E01908C
:10A4C00004D12E205A46179990476D1CBAF100010D
:10A4D000AAF1010ADDDC05E017F8010B5A461799CD
:10A4E00090476D1CB8F10001A8F10108F4DC5B464F
:10A4F0002146179A0598ABE62D0000002B000000BE
:10A500002000000030BCBDE8C08F2DE9F0410446BA
:10A5100000251E461746880404D405E0394620204D
:10A52000B0476D1C641EF9D52846BDE8F0812DE9C1
:10A53000F041044600251E469046C80301D5302749
:10A5400000E02027880404D505E041463846B0479E
:10A550006D1C641EF9D52846BDE8F08100B50020C9
:10A560002DF0B0FD00BD10B526F072F810BD10B58D
:10A57000012006F0BDFE10BD10B500202DF020FE1C
:10A5800010BD00B504202DF09DFD00BD10B50020CC
:10A5900025F060FE042026F077F810BD10B50220EB
:10A5A00006F0A6FE10BD10B501202DF009FE10BD6D
:10A5B0000FB4BDF8040000990A690240824201D13B
:10A5C000012200E00022D0B204B070472DE9FC4720
:10A5D000054689460DB1012100E0002108465F21B2
:10A5E000F6F75EFE4FF0000AD0462C4626686768F4
:10A5F00000BF3AE0D7E90401CDE900016068D0F876
:10A6000008C097E80F00E047D6E90401CDE9000152
:10A610002068D0F808C096E80F00E0474FEA48608D
:10A620004FEA1068284606F0ECFFD7E90401CDE9AF
:10A6300000016068D0F814C097E80F00E04718B137
:10A6400008F1010000F0FF08D6E90401CDE900019E
:10A650002068D0F80CC096E80F00E047284606F0C6
:10A66000D0FF0AF1010000F0FF0ABAF1080FC1DBC8
:10A67000B9F1010F03D12846FDF76CFC02E0284632
:10A68000FFF75BFA404600F000B80CBCBDE8F0876D
:10A690007CB504460CB1012100E000210846CF2121
:10A6A000F6F7FEFDA169D1E90401CDE90001A56934
:10A6B0006E6995E80F00B0477CBD2DE9F04707466D
:10A6C000884614461D464FF000090FB1012100E0F5
:10A6D00000210846FA21F6F7E3FD0CB1012100E064
:10A6E00000210846FB21F6F7DBFD0DB1012100E05A
:10A6F00000210846FC21F6F7D3FD384632F079F800
:10A700004146384632F05DF98146002606E0FF21D9
:10A71000384632F056F9A055701CC6B2AE42F6DB90
:10A72000384632F04BF84846BDE8F0872DE9FC4149
:10A7300004462169D1E90401CDE900012669F768E1
:10A740003B4696E80700B84794F860102046226B15
:10A7500090476620015D2046226B9047054621699F
:10A76000D1E90401CDE900012669D6E902733A4630
:10A77000D6E90001B8472846BDE8FC8170B504461B
:10A78000002508E02846691C8DB244F62061884205
:10A7900000DD07E000BF2046FFF7C8FF00F0010022
:10A7A0000028EFD100BF70BD0FB4BDF804100098B1
:10A7B000816200BF04B0704770B504460D4616466E
:10A7C0000948007820F0400007490870074951F80F
:10A7D00024003246294634F0F2F8044951F82400A6
:10A7E00033F041FE70BD0000780200100000001040
:10A7F00000220265C2667047024692F8980040B98E
:10A80000002002F14400002303614364416341647A
:10A810000AE0002002F1440000238361C361036267
:10A8200003648160816300BF704700002DE9F04F31
:10A8300087B0044633F084F98246A06CAAEB00018D
:10A84000E06C814203D2022007B000F059B9C4F88D
:10A8500048A0A06AD0F800903C20005DE8B9002133
:10A860006165C4F85811C4F878112164616484F8F2
:10A870007C11C4F8309001213C200155E06A016848
:10A88000C4F88411D4F88001F5F78EFF0746D4F898
:10A890008411F5F709FDE16A0860606BF5F784FF44
:10A8A0008046216BF5F700FD07464946F6F76CF840
:10A8B0000BD2D4F88001F5F777FF0746D4F884115E
:10A8C000F5F747FDE16A086016E0606BF5F76CFF8D
:10A8D0008046216BF5F73DFD07464946F6F75EF8E1
:10A8E0000AD2D4F88001F5F75FFF0746D4F8841147
:10A8F000F5F7DAFCE16A0860012084F82400012100
:10A9000025200155206D451E2BE004F1580050F81C
:10A91000257094F8240060B13846F5F745FF80466D
:10A920004946F6F731F801D2012000E0002084F812
:10A9300024002520005D60B13846F5F735FF8046DC
:10A940004946F6F72BF801D2012100E0002125202D
:10A95000015504F1580050F82520691C40F82120C9
:10A960006D1E002DD1DA4846F5F74AFFA06594F830
:10A97000240070B3606D08B901216165606D401CF1
:10A98000D0B901216165D4F85801401CC4F85801C0
:10A9900084F87C11606C68B1D4E91010091A04F5D0
:10A9A000AE70D4F8782140F82210D4F87801401C19
:10A9B000C4F87801216C6164C4F840A04846F5F7FA
:10A9C0001FFF014604F59270D4F8582140F8221078
:10A9D00023E0FFE72520005DF8B1606D10B94FF06E
:10A9E000FF316165606D012809D1811E6165D4F870
:10A9F0005801401CC4F85801012184F87C11D4F896
:10AA000058010A2809DA4846F5F7FAFE014604F526
:10AA10009270D4F8582140F8221094F87C01002854
:10AA200063D0D4F858010C285FD1002602251AE023
:10AA300004F5927050F82520691C50F82100101A76
:10AA400007D504F5927050F8211050F82500081A27
:10AA500007E004F5927050F82520691C50F8210099
:10AA6000101A06446D1C0A2DE2DD092096FBF0F653
:10AA70003046F5F7A7FE1F4A1F4BCDE90001F5F759
:10AA80008AFD07468846D4F88011C800F5F78CFE89
:10AA90008346F5F71AFF3A464346CDE90201F5F73A
:10AAA000EFFDCDE90401F5F753FFC4F88801002656
:10AAB000012505E004F5AE7050F8250006446D1C34
:10AAC000052DF7DD052096FBF0F63046F5F76CFE18
:10AAD00007460A49F5F772FCC4F88C010021E06AC8
:10AAE00001603C2001550120AEE6002184F87C1174
:10AAF0000020A9E66E861BF0F921094000007A4487
:10AB000030BCBDE8C08F0FB4BDF80410009881615F
:10AB100000BF04B0704710B5C1650AB1012400E060
:10AB2000002480F8764010BD10B590F8983053B9E5
:10AB3000002300F1440319620AB1012400E000245B
:10AB400083F824400AE0002300F14403D9640AB1E9
:10AB5000012400E0002483F8504000BF10BD000035
:10AB600070B504460120A075E089C11700EB517152
:10AB7000C910228A51438DB22A46FF21A069FEF7EF
:10AB8000F0FE228A002102480068FEF7EAFE70BD4E
:10AB9000CC01001081637047F0B5DDE90545016126
:10ABA000426183614FF07C578762C562046300276E
:10ABB00007624762F0BD2DE9F04F04460D46DDE91E
:10ABC0000AC8099F04F13000014600264FF08009B1
:10ABD00001E001F8016BB9F1000AA9F1010B1FFABC
:10ABE0008BF9F6D100BFC560026143618762C0F88E
:10ABF0004880C0F84CC0002180F8461000F000B832
:10AC000030BCBDE8C08F70B504460D461646A5623F
:10AC1000E6620021A1630121616300213C2001550E
:10AC20000121C4F880110821204630F029FC32F0BF
:10AC300087FFA06470BD00002DE9F05F05460E4659
:10AC400017469846DDE90BABDDF82890012085F822
:10AC500099002449A82041510021AC204151B02045
:10AC600041512149B82041512049B420415195F822
:10AC70009800E0B9002405F1440454220021204644
:10AC8000FEF7FBFE6661A761C4F81C80C4F828903B
:10AC9000C4F84CA00D98A063C4F83CB0002084F820
:10ACA000240084F84800012084F8490017E00024BB
:10ACB00005F14404542200212046FEF7DEFEE66042
:10ACC0002761C4F81480C4F82490C4F828A00D9813
:10ACD000E062C4F830B0012084F8450000BF00F005
:10ACE00007B8000000004040000020C100002041E3
:10ACF00030BCBDE8C09F00002DE9F04104460D4680
:10AD0000164625610E4961610E49A1610E49E16156
:10AD1000002121626162A16225636163A663E5632C
:10AD200029463046F5F712FB07460849F5F714FBAC
:10AD3000E062074921646164A164BDE8F08100001C
:10AD40008FC2F53D6666E63ECDCC4C3D6F12033AB0
:10AD5000CDCCCC3D2DE9F04104460D4604F1140064
:10AD600001460026702701E001F8016BB7F1000CE5
:10AD7000A7F101081FFA88F7F6D100BF4562026308
:10AD80004363044941614FF07C5101644164816433
:10AD9000BDE8F0810000204170B504460D46E07C1E
:10ADA000A84213D0E57401206075E089C11700EB5B
:10ADB0005171C910228A51438EB23246FF21A069D7
:10ADC000FEF7CFFD2046A16D884700BF70BD01464C
:10ADD0000120704790F8982022B9002200F1440227
:10ADE000916204E0002200F14402516200BF70470A
:10ADF000B8231950B4231A50704790F8982022B9FC
:10AE0000002200F14402516404E0002200F14402F7
:10AE1000916300BF70474164704790F8982022B951
:10AE2000002200F14402D16104E0002200F144025A
:10AE3000516100BF704790F8982022B9002200F1BC
:10AE40004402D16204E0002200F14402D16300BF59
:10AE5000704780F87510704790F898202AB9002242
:10AE600000F1440282F84A1005E0002200F1440299
:10AE700082F8461000BF70470164704790F8982030
:10AE800022B9002200F14402916104E0002200F1A5
:10AE90004402116100BF704780F87410704790F849
:10AEA00098202AB9002200F1440282F8491005E0F6
:10AEB000002200F1440282F8451000BF7047C163D0
:10AEC000704790F8982022B9002200F144025161A5
:10AED00004E0002200F14402D16000BF704770B569
:10AEE00004460D462946204630F0CAFA70BD41633B
:10AEF00070478263C1637047C16602677047C0F8DC
:10AF0000801170472DE9F04F044616461F46324621
:10AF100008464FEAE17901EB59794FEAE909A1EBDB
:10AF2000C90909F0FF08012000FA08F000F0FF0C41
:10AF3000E0894FEAE07900EB59794FEAE903E089CB
:10AF40004FEAE07900EB59794FEAE90BA569FF2F49
:10AF500017D14FEAE17901EB59794FEAE90903FB8F
:10AF6000025A1AF8099049EA0C0908464FEAE17AB0
:10AF700001EB5A7A4FEAEA0A03FB025E0EF80A90E6
:10AF800016E04FEAE17901EB59794FEAE90903FB51
:10AF9000025A1AF8099029EA0C0908464FEAE17AA0
:10AFA00001EB5A7A4FEAEA0A03FB025E0EF80A90B6
:10AFB0000648006830B10120DFF81090D9F8009001
:10AFC00009F80200002000F003B80000CC010010D6
:10AFD00030BCBDE8C08F8267C167704710B590F87C
:10AFE00098302BB9002300F144039A63D96305E03C
:10AFF000002300F14403DA62196300BF10BD2DE99C
:10B00000FC4704460D4616461F46DDE90A893B46C5
:10B01000324629462046CDE9008930F0CDFC00F0CB
:10B0200000B80CBCBDE8F08710B590F8983033B983
:10B03000002300F1440383F848101A6406E000235B
:10B0400000F1440383F844109A6400BF10BD00006F
:10B0500004490968098990FBF1F109B2024A1268B2
:10B060001181704720020010A004002010B5016774
:10B070000AB1012400E0002480F8774010BD4A683E
:10B08000002A06D00A68531C0B6010704868401EE6
:10B090004860704710B504460CB1012100E0002162
:10B0A0000846A321F6F7FCF8D4F8880018B120462A
:10B0B000D4F888108847D4F8840018B12046D4F812
:10B0C0008410884710BD0000F0B50346002083F8C7
:10B0D0008100DC6F586F0646254F3F5DF75927F01A
:10B0E0000107DFF88CC01CF804C046F80C7000BFE4
:10B0F000DC6F586F06461E4F3F5D3744F96000BF56
:10B10000DC6F586F06461A4F3F5D37447F686FF318
:10B110000F071743DFF858C01CF804C0B444CCF83C
:10B12000047000BFDC6F586F0646114F3F5DF75942
:10B1300047F00107DFF838C01CF804C046F80C706F
:10B1400000BF002507E0681C85B24CF250308542F4
:10B1500001DD00BF03E093F881000028F3D000BFB9
:10B1600093F88100012800D1F0BD0020FCE7000029
:10B17000CC01050870B504460D4600260CB101212E
:10B1800000E00021084640F22911F6F789F8204630
:10B1900031F02FFB2946204631F013FC00212046D8
:10B1A00031F00FFC0646204631F008FB304670BDFA
:10B1B0002DE9FC4105460E4600270DB1012100E0B6
:10B1C0000021084640F23D11F6F76AF82C460CB112
:10B1D000012100E00021084640F2DA21F6F760F88C
:10B1E000A169D1E90401CDE90001D4F818C0DCF867
:10B1F0000C8043469CE80700C04700BF284631F05A
:10B20000F8FA3146284631F0DCFB0746284631F093
:10B21000D5FA3846BDE8FC812DE9FC4705460E46C7
:10B2200017464FF000080DB1012100E0002108464B
:10B230004FF4A871F6F734F82C460CB1012100E068
:10B240000021084640F2CF21F6F72AF8A169D1E99A
:10B250000401CDE90001D4F818C0DCE902934A46A4
:10B26000DCE90001C84700BF284631F0C2FA0024DB
:10B2700007E03178284631F0A4FB8046761C601C3C
:10B2800084B2BC42F5DB284631F098FA404600F023
:10B2900000B80CBCBDE8F0872DE9F04104460E462D
:10B2A000154600270CB1012100E0002108464FF4AB
:10B2B0008A71F5F7F5FF204631F09BFA31462046BA
:10B2C00031F07FFB07462946204631F07AFB2046C5
:10B2D00031F074FA3846BDE8F0810A68531C0B60FF
:10B2E0001070704770472DE9FC4104460CB10121F4
:10B2F00000E0002108460F21F5F7D2FF25462C4635
:10B300002E686F68D7E90401CDE900016868D0F8BC
:10B3100008C097E80F00E047D6E90401CDE9000135
:10B320002868D0F808C096E80F00E047204606F0ED
:10B3300068F9D7E90401CDE900016868D0F80CC0CC
:10B3400097E80F00E047204606F05BF9D6E90401D4
:10B35000CDE900012868D0F80CC096E80F00E0475E
:10B36000204606F04EF9BDE8FC812DE9FC4104467B
:10B370000CB1012100E0002108462D21F5F790FFD6
:10B3800025462C462E686F68D6E90401CDE90001F8
:10B390002868D0F80CC096E80F00E047D7E9040110
:10B3A000CDE900016868D0F80CC097E80F00E047CD
:10B3B000204606F026F9D6E90401CDE90001286807
:10B3C000D0F808C096E80F00E047D7E90401CDE9BE
:10B3D00000016868D0F808C097E80F00E0472046F1
:10B3E00006F00FF9BDE8FC810FB410B5BDF80C10E4
:10B3F0000298426921EA020302EA010443EA044393
:10B40000836100BF10BC5DF814FB000010B504465A
:10B41000024951F8240033F033F910BD0000001048
:10B420002DE9F04104460D46124951F8240033F04D
:10B4300027F90746002F1ADD0E4951F8240033F092
:10B4400014F9064696B100200EE016F8201000EB25
:10B450004002A95406EB8001498800EB40022A44CF
:10B46000A2F80110411C88B2B842EEDB00BFBDE873
:10B47000F081000000000010F0B5044605ADE0CDFD
:10B4800004F13000C1600261436185628764C66473
:10B490004FF0000C80F846C0F0BD2DE9F05F054686
:10B4A0000F4690461E46DDE90BABDDF8289095F877
:10B4B0009800F0B9002405F144046761C4F81880CD
:10B4C000E661C4F82890C4F838B0C4F83CA0002065
:10B4D00084F8240084F8480000213046F5F75EFA2D
:10B4E00003D2012084F84A0002E0002084F84A00D8
:10B4F00019E0002405F14404E760C4F81080666197
:10B50000C4F82490C4F82CB0C4F830A00021304610
:10B51000F5F744FA03D2012084F8460002E0002047
:10B5200084F8460000BF00F000B830BCBDE8C09F02
:10B5300070B504460D462946204617F0F9FB70BD4C
:10B540002DE9FC4104460CB1012100E00021084630
:10B550004021F5F7A5FE4FF0000825462C462E6841
:10B560006F68D7E90401CDE900016868D0F808C028
:10B5700097E80F00E047D6E90401CDE9000128680B
:10B58000D0F808C096E80F00E047204606F039F8EA
:10B590000CE008F1010000F0FF08B8F1FA0F05DD3A
:10B5A0002046FFF7E2FE0020BDE8FC81D7E9040158
:10B5B000CDE900016868D0F814C097E80F00E047B3
:10B5C0000028E6D1D6E90401CDE900012868D0F8C9
:10B5D0000CC096E80F00E047204606F012F8012064
:10B5E000E2E72DE9FC47064688464FF000090EB118
:10B5F000012100E0002108468821F5F751FE34467C
:10B60000276865684FF0000946E008F0800050B1F7
:10B61000D5E90401CDE900016068D0F808C095E8DB
:10B620000F00E04709E0D5E90401CDE900016068B9
:10B63000D0F80CC095E80F00E047D7E90401CDE948
:10B6400000012068D0F808C097E80F00E0473046B6
:10B6500005F0D7FF4FEA48604FEA1068D7E90401C8
:10B66000CDE900012068D0F80CC097E80F00E04752
:10B67000304605F0C6FFB9F1070F09D1D5E904013D
:10B68000CDE900016068D0F808C095E80F00E047F8
:10B6900009F1010000F0FF09B9F1080FB5DB00F076
:10B6A00000B80CBCBDE8F0877CB504462169D1E93F
:10B6B0000401CDE900012569EE68334695E80700ED
:10B6C000B0476320015D2046226B90472169D1E994
:10B6D0000401CDE900012569D5E902633246D5E9C7
:10B6E0000001B0477CBD7CB504462169D1E9040165
:10B6F000CDE900012569EE68334695E80700B047BB
:10B700006220015D2046226B90472169D1E9040146
:10B71000CDE900012569D5E902633246D5E900018A
:10B72000B0477CBD2DE9F04106460F4614461D4644
:10B730004FF000080EB1012100E000210846DE2193
:10B74000F5F7AEFD0CB1012100E000210846DF2134
:10B75000F5F7A6FD0DB1012100E000210846E0212A
:10B76000F5F79EFD304631F044F83946304631F069
:10B7700028F9804604E02178304631F022F9641C33
:10B78000281EA5F10101CDB2F5D1304631F016F8F1
:10B790004046BDE8F08170B506460D4600240BE03A
:10B7A000E00045FA00F0C1B23046FFF71AFF30461C
:10B7B000FFF7C6FE601CC4B2022CF1DB70BD0000B6
:10B7C0002DE9F04104462146012000F0DBF9054651
:10B7D00000212846F5F7D8F800D200250949284667
:10B7E000F5F7DCF800D2074D06492846F4F7B4FD1A
:10B7F00007460CF02BFA06460249F4F7DFFDBDE8D8
:10B80000F08100000000C84270B50546032D01DA42
:10B81000012100E0002108469421F5F741FD05EBE8
:10B8200005100D4901EB80042068F7F765FAD4E9AB
:10B830000101F7F763FB20688168084A1140891C01
:10B84000816000BFE06930B1E6693146012026F031
:10B85000D9FD00BF00BF70BD141E0010C0FFFF7FE8
:10B8600070B5054605EB05100E4901EB80040CB1DF
:10B87000012100E00021084640F24F11F5F710FDCC
:10B880006068F7F781FB28B16068F7F731FB206843
:10B89000F7F732FA6068F7F77CFB10B16068F7F7EA
:10B8A0002AFB70BD141E001070B5054605EB05108F
:10B8B0001E4901EB80040CB1012100E00021084683
:10B8C0004FF4B471F5F7ECFC20680168C1F3001186
:10B8D00000292AD02069401C20612068F7F70CFA63
:10B8E000D4E90101F7F70AFB228BD4E90101F7F74C
:10B8F00063FB00212068F7F77FF906463246D4E95A
:10B900000101F7F7C7FBE269D4E90101F7F784FB0E
:10B91000D4E90101F7F70EFB2068F7F732F9206848
:10B92000F7F72CF92068F7F7DFF970BD141E001047
:10B930000146002001F001020AB1421CD0B201F020
:10B9400002020AB1421CD0B201F004020AB1421C48
:10B95000D0B201F008020AB1421CD0B201F01002CC
:10B960000AB1421CD0B201F020020AB1421CD0B28E
:10B9700001F040020AB1421CD0B201F080020AB1CB
:10B98000421CD0B201F480720AB1421CD0B201F460
:10B9900000720AB1421CD0B201F480620AB1421CAA
:10B9A000D0B201F400620AB1421CD0B201F480525C
:10B9B0000AB1421CD0B201F400520AB1421CD0B20A
:10B9C00001F480420AB1421CD0B201F400420AB133
:10B9D000421CD0B201F480320AB1421CD0B201F450
:10B9E00000220AB1421CD0B201F480220AB1421CEA
:10B9F000D0B201F400320AB1421CD0B2704700004C
:10BA00002DE9F84F05460E4617469A46DDE90A89A4
:10BA1000032D01DA012100E0002108461C21F5F781
:10BA20003FFC0EB1012100E0002108461D21F5F781
:10BA300037FC0FB1012100E0002108461E21F5F777
:10BA40002FFCB8F1000F01DD012100E000210846C4
:10BA50001F21F5F725FC05EB0510454901EB800496
:10BA6000442200212046FDF786FF26606760C4F867
:10BA700008A0C4F80C90A4F814804846FFF758FFBB
:10BA8000A075A07D00FB08F02083208B4FEA400BBF
:10BA90005946012026F0E0FCE061E16909B101218D
:10BAA00000E0002108463121F5F7FAFB218B49041B
:10BAB0000A0C0021E069FDF75EFF0020009020687D
:10BAC000C16801F00301009100212068F7F7F0F848
:10BAD0007F212068F7F740F900BF20688168C90F0F
:10BAE0000029FAD120680099F7F7E2F80A20F8F760
:10BAF00088FC2068416841F01001416000BF206867
:10BB000081681C4A1140491C816000BF0A20F8F777
:10BB100078FC09F4002050B14FF480001649896880
:10BB200021F0E0710143144A916000BF00BF228BF5
:10BB3000D4E90101F7F740FA00212068F7F75CF833
:10BB400083465A46D4E90101F7F7A4FAE269D4E939
:10BB50000101F7F761FAD4E90101F7F7EBF9009871
:10BB6000032802D12068F7F7BFF800F007B80000FB
:10BB7000141E0010C0FFFF7F0003045018BCBDE876
:10BB8000E08F00002DE9F04105460E460027C5EB89
:10BB9000C5000E4901EB80040CB1012100E0002139
:10BBA00008464FF44171F5F77BFB207858B1E188E6
:10BBB000B4F902201144701AF4F7F6FD8046616969
:10BBC000F4F7CAFB07463846BDE8F08174740010EC
:10BBD00010B50446204631F049FB204631F0A6FA64
:10BBE00010BD00002DE9F04705468846032D01DA17
:10BBF000012100E0002108464FF48671F5F750FB63
:10BC00004FF00009002605EB0510184901EB8004F0
:10BC10000CB1012100E0002108464FF48871F5F7CE
:10BC20003FFB31F087FF2064E06900EB480700200C
:10BC300006E039880E44411C88B2A17D07EB41071C
:10BC4000A18A8142F5DCA08AB6FBF0F01FFA80F9E8
:10BC500031F070FF216C411AE163D4E90E10884283
:10BC600001D9E06BA0634846BDE8F087141E0010C0
:10BC70002DE9F05F06468846032E01DA012100E037
:10BC800000210846EA21F5F70BFB4FF0000B06EB0D
:10BC900006101F4901EB80040CB1012100E00021D6
:10BCA0000846ED21F5F7FCFA31F044FF6063B4F883
:10BCB00014A04FEA4A0019F09BFE0546E06900EB2C
:10BCC0004807002007E0398825F81010411C88B289
:10BCD000A17D07EB4107A18A8142F4DCA18A2846B5
:10BCE00017F0D2FEA08A401035F810B031F022FFD4
:10BCF000616B411A2163D4E90B10884201D9206B92
:10BD0000E062D94628460CF0BBF8484600F002B87D
:10BD1000141E001030BCBDE8C09F00002DE9FC5F80
:10BD200007468A46032F01DA012100E00021084678
:10BD3000BB21F5F7B5FA07EB07102C4901EB80049E
:10BD40000CB1012100E000210846BD21F5F7A8FA59
:10BD5000A08A022802DC002000F04AB831F0EAFE96
:10BD6000A062B4F814B04FEA4B0019F041FE05464A
:10BD70004FF00008A08A8610E06900EB4A09002015
:10BD800008E0B9F8001025F81010411C88B2A17D18
:10BD900009EB4109A18A8142F3DCA18A284617F008
:10BDA00073FE304604E035F810108844411C88B218
:10BDB000A18A891B8142F6DCA08AA0EB4600B8FB71
:10BDC000F0F080B2009031F0B5FEA16A411A6162D4
:10BDD000D4E90810884201D9606A20620098019075
:10BDE00028460CF04DF80198B6E70000141E00102C
:10BDF0003CBCBDE8C09F00002DE9F04705460E465B
:10BE0000032D01DA012100E000210846AB21F5F7FE
:10BE100047FA05EB05100B4901EB80040CB1012139
:10BE200000E000210846AD21F5F73AFA94F81680B3
:10BE300094F81690E769002007EB400030F81600F0
:10BE4000BDE8F087141E00102DE9F05F04460E488F
:10BE500005880D4822300688701BF4F7A5FC824641
:10BE6000601BF4F7A1FC83465146F4F7A7FA81461C
:10BE70000649F4F771FA80460549F4F715FA0746C2
:10BE8000384600F007B80000A875FF1F0000A04268
:10BE90000000F04130BCBDE8C09F00002DE9F0413A
:10BEA00004460F48008840F6B831484340F6FF7119
:10BEB000B0FBF1F63046F4F780FC05462046F4F777
:10BEC0007CFC804641462846F4F778FA0746054947
:10BED000F4F742FA06460449F4F770FABDE8F08137
:10BEE000AA75FF1F00F07F4500007A442DE9F04F4E
:10BEF00091B080460C4642461DA101A8FBF7C6FE44
:10BF000001A8F4F7ADF98146A9F10100032190FBE6
:10BF1000F1FA4FF0000B002700BF16E001A90B5CFF
:10BF200039467F1C63540BF1010B03219BFBF1F29B
:10BF300001FB12B141B9BAF1000F05DD2C233946DE
:10BF40007F1C6354AAF1010A401E0028E6DA002093
:10BF5000E05500257E1E06E0605DA15D6155A0559F
:10BF60006D1C761E00BFB542F6DB11B000F002B8C2
:10BF70002564000030BCBDE8C08F70B504460D4696
:10BF80002946204633F060FF70BD00002DE9F041E6
:10BF90000EF0A0FA9C490968096A08709B4800687D
:10BFA000408A99490968096A888098480068C08A67
:10BFB00095490968096AC88093480068006A8088C2
:10BFC00091490968096AC988401A09D58E480068EC
:10BFD000006AC0888C490968096A8988401A08E0A3
:10BFE00089480068006A808887490968096AC988A1
:10BFF000401A85490968096A088124F081FA834852
:10C000000068008C80490968096A48817F48006897
:10C01000408C7D490968096A88817C480068C08C29
:10C0200079490968096AC88178480068008D7649AD
:10C030000968096A088275490968098C734A126897
:10C04000528C8818F4F7B0FB05464FF07C51F4F79A
:10C0500083F90446F4F7EDFB6B490968096A4882E5
:10C060006A490968C98C694A1268128D8818F4F700
:10C070009BFB05464FF07C51F4F76EF90446F4F74C
:10C08000D8FB61490968096A888260490968C86AF9
:10C09000F4F793FB044621465D48F4F78FF95A49BB
:10C0A0000968096A486359490968086BF4F785FB10
:10C0B000044621465648F4F781F953490968096A4C
:10C0C000886352490968C86AF4F78DFB0646002266
:10C0D000504BF4F7D5FA0446F4F73AFC4A4909689C
:10C0E000096AC86349490968086BF4F77CFB06468E
:10C0F0000022484BF4F7C4FA0446F4F729FC4249FD
:10C100000968096A0864404A1268126A116C3E4A5A
:10C110001268126AD06BF4F7C7F804464FF07C51EE
:10C12000F4F71AF938490968096A886236490968D2
:10C1300009894800F4F746FB06460022354BF4F720
:10C140009FFA0446F4F704FC2F490968096AC8629B
:10C150002D490968096A886A4FF08141F4F7FCF8B3
:10C1600029490968096A08632B4890F8380180B9A1
:10C1700025480068006AC08823490968096AC880A0
:10C1800021480068006A80881F490968096A888018
:10C1900010E01D490968096AC8881B490968096ACD
:10C1A0008988194A1268126AD18017490968096A90
:10C1B000888000BF14480068006AC0881249096876
:10C1C000096A8988884205DD01200F490968096AE2
:10C1D000C87004E000200C490968096AC8700A4860
:10C1E0000068006A4078012805D1022006490968E4
:10C1F000096A487004E0032003490968096A487025
:10C2000024F0ACF9BDE8F08120020010A004002069
:10C210000050C34700408F40987100102DE9FC5F2B
:10C2200080461E254FF000094FF0000A0195019D40
:10C23000680019F0DDFB0746B8F1010F71D12A46FD
:10C2400000213846FDF741FC00200CE000EB4002E5
:10C25000AD49096801F5C87101EB8204A18827F88E
:10C260001010411C88B2A842F0DB6A1E002138463B
:10C270002CF097FA284605EBD071491037F8119049
:10C280002A4600213846FDF720FC002014E09E4994
:10C29000096801F50051B1F81017491E091A01EBA0
:10C2A00041029949096801F5C87101EB8204A1882E
:10C2B00027F81010411C88B2A842E8DB6A1E002152
:10C2C00038462CF06EFA284605EBD071491037F845
:10C2D00011A0BAEB090002D5A9EB0A0001E0AAEB14
:10C2E0000900B0F5FA7F05DA00208749096881F86E
:10C2F0003D0004E001208449096881F83D0082483E
:10C30000006800F50050B0F81007401E00EB400137
:10C310007D48006800F5C87000EB81064FF0000B07
:10C3200022E063E00BEB4B017748006800F5C87032
:10C3300000EB810460887188884211D123F078FD78
:10C340002188884202DA23F073FD00E020886E49DC
:10C35000096808856D49A0680968096A48620BE0A8
:10C360000BF101001FFA80FB6748006800F50050E0
:10C37000B0F810075845D5DC00BF6348006800F5E9
:10C38000C876002029E000EB40025F49096801F50A
:10C39000C87101EB820461887288891A03D571889B
:10C3A0006288891A02E061887288891A0C2912DD74
:10C3B000411E01EB41025449096801F5C87101EBC6
:10C3C00082042188504A1268D184504AA1681268B8
:10C3D000126A116209E0411C88B24B49096801F5F3
:10C3E0000051B1F810178142CDDC88E0B8F1020F9E
:10C3F0007ED14548006800F5C876002029E000EBB2
:10C4000040024149096801F5C87101EB8204618865
:10C410007288891A03D571886288891A02E0618856
:10C420007288891A0C2912DB411E01EB4102364940
:10C43000096801F5C87101EB82042188324A12684B
:10C440001184324AA1681268126AD16109E0411C64
:10C4500088B22D49096801F50051B1F810178142E1
:10C46000CDDC00BF2848006800F50050B0F8100788
:10C47000401E00EB40012448006800F5C87000EB46
:10C480008106002017E000EB40021F49096801F512
:10C49000C87101EB820461887288914209D12188B8
:10C4A000194A12685184194AA1681268126A916186
:10C4B00009E0411C88B21449096801F50051B1F83E
:10C4C00010178142DFDC00BF0F490968498C0E4A12
:10C4D0001268128D8818F4F767F94FF07C510090BC
:10C4E000F3F73AFF8346F4F7A4F90749096800E037
:10C4F00001E0888403E0F2210020F4F7D1FE384601
:10C500000BF0BEFC00F004B8A004002020020010D4
:10C510003CBCBDE8C09F000070B503460C4600253A
:10C520001748418817480068C08988420ED01548CE
:10C530000068C089401A04D512480068C089081AEA
:10C5400003E010480068C089401A85B2954204DDB6
:10C550000C480068C181002070BD0A480068B0F92D
:10C560000800002802DC1C700220F5E7054800687E
:10C570000089401E00B2034E366830810120EBE78F
:10C58000C0050010A00400202DE9FF4106460F461B
:10C59000154695F8F000F0B12A463146684603F09A
:10C5A00044FD012409E0684622F012FA05EB04116B
:10C5B0006846FFF7E2FC601CC4B295F8F000A042A8
:10C5C000F1DC68462FF01AFC05EB04126946384688
:10C5D00003F02BFD03E0FF2004B0BDE8F081002054
:10C5E000FAE700002DE9F05F81460E461446102E52
:10C5F00004D0182E03D0202E03D101E000BF00BFCD
:10C6000005E0002084F8F000FF2000F089B800BFAA
:10C6100032464946204603F06BFD06F11C008006B9
:10C620004FEA10680120C0EB2810C0B284F8F00077
:10C63000354601276EE0A5F1040A14F80AC0A5F1F9
:10C64000030A14F80A10A5F1020A14F80A20A5F149
:10C65000010A14F80A3095FBF6FA06FB1A5ABAF1E9
:10C66000000F19D16046DFF8B4A01AF801A08AEAD9
:10C67000070CDFF8A8A01AF802101AF803201AF81D
:10C6800000304FEAD71A4FF01B0B0AFB0BFA8AEA6D
:10C69000470A0AF0FF0712E0182E10DD95FBF6FAA4
:10C6A00006FB1A5ABAF1100F09D1DFF870A01AF878
:10C6B0000CC01AF801101AF802201AF80330A5EB82
:10C6C000060A0AF0FF0014F800A08AEA0C0A04F82F
:10C6D00005A000F1010A14F80AA08AEA010A05F18E
:10C6E000010B04F80BA000F1020A14F80AA08AEA70
:10C6F000020A05F1020B04F80BA000F1030A14F87A
:10C700000AA08AEA030A05F1030B04F80BA0281D0E
:10C71000C0B2054645458EDB002076E74422050879
:10C7200030BCBDE8C09F2DE9FC5F83460D46164630
:10C730001C4600270DF104094FF0010AFF22514663
:10C740004846F3F76FFD0020234632462946009005
:10C750005846FCF721F90746A4EB040887B9B8F15D
:10C76000000F0DD0A11942464846F3F73BFD0020CB
:10C77000611953464A4600905846FCF70DF90746A2
:10C78000384600F000B83CBCBDE8C09F70B58AB028
:10C7900004460E4615464FF0FF30099000200890E1
:10C7A00007900494059509A8069000201B4907AA44
:10C7B00008ABCDE9002102900246314620462EF01A
:10C7C000E3F8079858B101201549002204ABCDE9E0
:10C7D000002102900222314620462EF0D5F808981A
:10C7E000C0B10998401CA8B90898012802D894F84B
:10C7F000300060B101200A49002204ABCDE90021DC
:10C8000002900246314620462EF0BEF802E001209A
:10C8100084F8300009980AB070BD000079AA0308B6
:10C8200025C8000830B503460C462146187898B153
:10C830001D694868583085420ED99878012806D07D
:10C840009878022808D1086890F8300020B9586913
:10C850008D682860012030BD0020FCE710B531F064
:10C860006FF905490968401AC82803D20020034916
:10C87000086010BD0120FCE7940000108800001043
:10C880002DE9F0419AB007208DF8040002208DF8C0
:10C8900005003748CDF807003649CDF80B1036496A
:10C8A000CDF80F103549CDF813103549CDF81710D4
:10C8B0003449CDF81B103449CDF81F103349CDF859
:10C8C00023103349CDF827103249CDF82B103249C7
:10C8D000CDF82F103149CDF833103149CDF837104C
:10C8E0003049CDF84B103049CDF84F102F49CDF8D5
:10C8F00053102F49CDF83B102E49CDF83F102E494B
:10C90000CDF8431000BF2D48C06A441C2046F3F701
:10C910006AFF05462A4A2B4BF3F73DFE0746F4F71C
:10C9200017F8CDF8570028482849C1F8B40A002064
:10C9300027490860486001A811F030FC11F0F0FEB2
:10C9400000BF2448F7F7D5FA2248F7F7E6FA00BF08
:10C9500000BF2048F7F7CDFA10201E49096A0143AD
:10C960001C4A116200BF00BF01201AB0BDE8F0816F
:10C97000B9A700080DB4000821B40008919100087F
:10C98000CB930008218C0008058D00088D8C0008D1
:10C99000D58D0008F19B00080D880008E5B200085D
:10C9A000F9830008CFAD0008FFAF0008A19300088D
:10C9B00031B5000879CB010839B7010800440140BE
:10C9C0009A9999999999B93F4474001020130010CD
:10C9D000000000100004004010B53548B0F8BE0A51
:10C9E000401C3349A1F8BE0A00F06AF810F0C6FBFB
:10C9F000304800691221B0FBF1F02E49C8802C4864
:10CA0000007A012801D1012200E000222A4903C94D
:10CA100062F34510284A03C2254890F88B0008B1FC
:10CA2000012100E000212448D0E9002061F38612B2
:10CA30002149C1E900201E48B0F86B001F49C98A8E
:10CA4000884212D01D48C08A1949A1F86B0011F024
:10CA500075FD174A6B320E21012015F069FF144A4B
:10CA6000D21C0221012015F063FF1148B0F8BE0A64
:10CA70000321B0FBF1F201FB120098B90C4890F8C9
:10CA8000A40A012805D1C820F7F7BBFC31F06CF8E7
:10CA900008E0074890F8A50A012803D126F05AFEBD
:10CAA0001CF0D0F932F056F801202FF044FD10BDF3
:10CAB000201300104474001008000020987100102A
:10CAC0002DE9FC474FF00009264DA5F638242648ED
:10CAD00090F82400019001A803F054FBA0789DF881
:10CAE000041088420BD161781F4890F825008142DC
:10CAF00005D121781C4890F82600814201D04FF0E2
:10CB000001099DF80400A070174890F82500607096
:10CB1000154890F826002070144890F8610068705D
:10CB2000124890F86210A97090F86310E9700E48EE
:10CB300090F8276090F8287090F8298000204346EC
:10CB40003A4631460090281D03F05AFA0120A87297
:10CB5000B9F1010F04D1054A6132082115F0E8FE50
:10CB600000F006B8B91D0010447400102013001026
:10CB70000CBCBDE8F087000010B55948007820F0E3
:10CB800001005749087000244FF4806055498861BE
:10CB900000BF002018F014FA30F000FB18F0F8F98C
:10CBA000514832F097FF51480088B0F5A46F03D088
:10CBB00001204E49887002E000204C49887025F021
:10CBC000C3FC30B94FF6FF7048490880012048493E
:10CBD0000873012000F0AAF80024C434F03404F5EE
:10CBE00001742146002009F08FFB0121002009F08B
:10CBF0007DFF00242146012009F086FB0121084623
:10CC000009F074FF00BF04F52B7404F5CC7404F232
:10CC1000045430342146022009F076FB0121022021
:10CC200009F064FF0121002009F0B0FF012108464E
:10CC300009F0ACFF0121022009F0A8FF012018F043
:10CC4000BFF92A48008830B925F06EFC18B94FF6B4
:10CC5000FF702649088017F06FFC05F0F1FD25F004
:10CC600073FF22480088B0F5A46F15D04FF4A4607C
:10CC70001E49088024F0A2F900BF1E48F7F734F9D6
:10CC80001C48F7F745F900BF00BF1B48F7F72CF920
:10CC90001948F7F73DF900BF00F038F8FFF7F0FD4D
:10CCA0000BF012F827F0AAFC1449154801F09CFC7F
:10CCB0000B48007820F00100401C0949087000BFB3
:10CCC0001048F7F711F90F48F7F722F900BF00BF36
:10CCD0000D48F7F709F90C48F7F71AF900BF10BD2E
:10CCE0007802001000040048B80000100070001026
:10CCF0009871001000480140001400408DE50008C4
:10CD000069E70008001000400044014010B50648E3
:10CD10000CF09CFD01F0BCFC17F07EF8012802D15C
:10CD2000002000F003F810BD0403001070B50446A5
:10CD300024B10E49087B1AF003FB09E00DF02CFF2B
:10CD400005461CF08EFB0DF019FB05461CF07AFB26
:10CD500017F062F8012808D10DF016FB01210170CF
:10CD600020461BF03DFB0DF069FF70BD987100106F
:10CD700010B501F00AFC0CF017FD4BF602318842A9
:10CD800002D10AF0BBFF01E001F012FC10BD10B5AA
:10CD90000346002008E01C5C14B93024145401E060
:10CDA0001C5C1454441CE0B28842F4DB10BD00004B
:10CDB0002DE9F04706462848006800F17F0526481F
:10CDC000006800F17E082448006800F1D409224878
:10CDD000006800F1DE042048006800F1E00A032743
:10CDE000287800F0800088B988F800601A48006848
:10CDF000808BA9F8000040F2DC502080208826F0CB
:10CE0000EBFB287840F08000287022E008212820E1
:10CE100000F0DAFE0746012F06D12088AAF80000AC
:10CE2000304600F0C1FE14E09FB920883122012174
:10CE300000F0D8FF20802088B0F57A6F06DB09204B
:10CE400005490968D1F8F410087002E0208826F03E
:10CE5000C3FBBDE8F08700002004002070B50D4939
:10CE60000968888BF3F7A9FC04462046F3F7E1FC38
:10CE700085B22846FEF7A4FC0446074890F838011E
:10CE8000012804D121460548F3F760FA04462046FC
:10CE900070BD000020040020987100100000C842FE
:10CEA0002DE9F04106462648006800F17F05244838
:10CEB000006800F17E082248006800F1E4040327BE
:10CEC000287800F0800078B901F020F80746012F9B
:10CED00002D00320BDE8F08188F8006000202060C7
:10CEE000287840F08000287001F001F80746012FF3
:10CEF00021D1144890F8380160B9322120684843A4
:10CF00004FF47A71B0FBF1F00D490968D1F8F410D3
:10CF100008670BE03221206848434FF47A71B0FB78
:10CF2000F1F007490968D1F8F410C866304600F0FE
:10CF30003BFE0120CEE72068401C20600220C9E7AC
:10CF400020040020987100102DE9FC5F804668489D
:10CF5000006800F17F076648006800F17E0B6448B6
:10CF6000006800F1DE046248006800F1E2066048F3
:10CF70000068D23001905E48006800F1C4090025C5
:10CF80004FF0030A387800F0800018BB8BF800805F
:10CF900057490968D1F8F410C889F3F70EFC5449D1
:10CFA0000968D1F8F410C86309203070504800684F
:10CFB000D0F8F400C089208020881822002100F0D9
:10CFC00011FF2080208826F007FB387840F0800091
:10CFD00038708AE0FFF742FFC9F80000317801EBB2
:10CFE00081014800F3F7E0FB0090D9F80010F3F757
:10CFF000D5FC0DD82088F3F7E0FB3D490968D1F84E
:10D00000F4101431327841F822003078401E30702C
:10D010000198038821880A22002000F089FF8246B7
:10D02000BAF1010F4FD12088F3F7C7FB30490968E7
:10D03000D1F8F410486121882D4A1268D2F8F42002
:10D040009289881800EBD071C1F34F01284A126809
:10D05000D2F8F42091812088183825490968D1F840
:10D06000F4104882002528E0052D10DA20490968CF
:10D07000D1F8F410143151F825001E49F3F766F980
:10D080001B490968D1F8F410143141F825001849FA
:10D090000968D1F8F410143151F82500F3F7C9FBF1
:10D0A00080B2009003F014FA11490968D1F8F41025
:10D0B000143141F82500681CC5B20B2DD4DB404665
:10D0C00000F072FD08E0BAF1000F05D120881822A7
:10D0D000002100F087FE208020885F2805DC0820E2
:10D0E00003490968D1F8F410087000F005B8000091
:10D0F000200400200000C0413CBCBDE8C09F0000EF
:10D100002DE9F84F07463E48006800F17F043C488F
:10D11000006800F17E093A48006800F1D40A3848F6
:10D12000006800F1C80B3648006800F1DE0534489D
:10D13000006800F1E00632480068E43000904FF0EB
:10D140000308207800F0800060BB89F800702C484C
:10D150000068808BAAF80000FFF780FECBF8000083
:10D1600030881822012100F03DFE30800021009817
:10D17000016030882880288821490968D1F8F41096
:10D18000098A884206DB0D201D490968D1F8F41090
:10D19000087002E0288826F01FFA207840F080000E
:10D1A00020702BE01E220821142000F0CDFC8046C8
:10D1B000B8F1010F12D100F057FD012804D12078F9
:10D1C00020F08000207019E028880D490968D1F806
:10D1D000F410C881384600F0E7FC0FE0B8F1000F0A
:10D1E0000CD128881822012100F0FCFD04490968AF
:10D1F000D1F8F410C881384600F0D6FC00F002B82F
:10D200002004002018BCBDE8E08F00002DE9F05F8D
:10D2100007463648006800F17F053448006800F191
:10D220007E083248006800F1D4093048006800F1F7
:10D23000C8062E48006800F1DE044FF0030A287883
:10D2400000F08000B8B988F8007028480068808B2A
:10D25000A9F80000FFF702FE306024480068D0F80B
:10D26000F400C0892080208826F0B6F9287840F0A4
:10D270008000287037E00421282000F0E1FE82467B
:10D28000BAF1010F2FD1FFF7E9FD83461849F3F7F3
:10D2900085FB09D8208815490968D1F8F410C881A0
:10D2A000384600F081FC1EE000F0DEFC012817D1BA
:10D2B000FFF7D4FD306020881822012100F092FD94
:10D2C00020802088B0F57A6F06DB092007490968BD
:10D2D000D1F8F410087006E0208826F07DF902E00D
:10D2E000FFF7BCFD306000F005B80000200400200E
:10D2F0000000C64230BCBDE8C09F00002DE9F05FD1
:10D3000080463248006800F17F043048006800F130
:10D310007E092E48006800F1D40A2C48006800F10C
:10D32000DE052A48006800F1E0062848006800F1A0
:10D33000E40B0327207800F0800050BB00F0D7FDFD
:10D340000746012F01D000F043B889F800801F483C
:10D350000068808BAAF8000030883122002100F09C
:10D3600041FD30800020CBF80000308828802888DC
:10D370005F2806DC0B2015490968D1F8F410087005
:10D3800002E0288826F028F9207840F080002070FC
:10D390001AE01E220821142000F0D6FB0746012FB8
:10D3A00004D1207820F0800020700DE067B9288833
:10D3B0001822012100F016FD04490968D1F8F41083
:10D3C0008881404600F0F0FB00BFBCE7200400204D
:10D3D00030BCBDE8C09F00002DE9F0470646264856
:10D3E000006800F17F052448006800F17E082248AB
:10D3F000006800F1DE042048006800F1E0091E48E2
:10D40000006800F1D00A0327287800F0800060B996
:10D4100088F80060B9F800002080208826F0DCF849
:10D42000287840F08000287024E0BAF80030218885
:10D430000A22124800F07CFD0746012F09D12088FE
:10D440000D490968D1F8F4100882304600F0ACFBB1
:10D4500006E02FB920881822012100F0C3FC2080AB
:10D460002088B0F57A6F05DB072003490968D1F8F9
:10D47000F4100870BDE8F087200400200000C842C6
:10D480002DE9F04106462648006800F17F05244852
:10D49000006800F17E082248006800F1E4040327D8
:10D4A000287800F0800078B900F021FD0746012FB0
:10D4B00002D00320BDE8F08188F8006000202060E1
:10D4C000287840F08000287000F020FD0746012FEA
:10D4D00021D1144890F8380160B9322120684843BE
:10D4E0004FF47A71B0FBF1F00D490968D1F8F410EE
:10D4F000C8660BE03221206848434FF47A71B0FBD4
:10D50000F1F007490968D1F8F4100867304600F0D7
:10D510004BFB0120CEE72068401C20600220C9E7B9
:10D5200020040020987100102DE9FC5F0746364862
:10D53000006800F1CC083448006800F1D009324896
:10D540000068D230019030480068D0F8F400C06E16
:10D550002D490968D1F8F410096F0844C0F34F0051
:10D5600000906421009891FBF0FB5846F3F71CF9FA
:10D5700082462649F2F722FF06462549F2F7ECFEDD
:10D5800005464FF07C51F2F7E7FE0446C8F800402C
:10D590001D480068D0F8F40080881B490968D1F85C
:10D5A000F4104988451A002D01DB294600E0694244
:10D5B0000846F3F7F9F8824616492046F2F7FEFED0
:10D5C00083465146F2F7C8FE0646F3F732F9A9F84A
:10D5D00000000D490968D1F8F41089880A4A1268D8
:10D5E000D2F8F4205288881A002801DB014600E0B6
:10D5F0004142642291FBF2F18AB201990A803846D5
:10D6000000F0D2FA00F008B82004002000007A44AC
:10D610000000FA430000C8423CBCBDE8C09F0000C7
:10D6200010B504462648C08A4EF23F61884224D194
:10D6300024490968D1F8CC004FF08041F2F7BEFED2
:10D6400020490968D1F8F410C8671E490968D1F863
:10D65000F410C86F4FF07E51F3F7A0F902D24FF0EB
:10D660007E5004E017480068D0F8F400C06F1549F8
:10D670000968D1F8F410C86708E012480068D0F8CB
:10D68000CC0010490968D1F8F410C8670E480D495C
:10D690000968D1F8F410C1F880000A490968D1F886
:10D6A000F410C86F0949F2F757FE06490968D1F826
:10D6B000F410C1F88400204600F076FA10BD000096
:10D6C0009871001020040020CDCC4C3D000020417A
:10D6D0002DE9F04104462448006800F17E07224805
:10D6E000006800F1DE0503263C705F202880288852
:10D6F00025F072FF0421C82000F0A2FC0646012E8E
:10D7000028D11A4890F8380180B917480068808BF2
:10D7100015490968D1F8F410488013480068808ED4
:10D7200011490968D1F8F410C8800FE00E4800686C
:10D73000808B0D490968D1F8F41088800A48006888
:10D74000808E09490968D1F8F4100881204600F05C
:10D750002BFA06E02EB9102003490968D1F8F4101D
:10D760000870BDE8F08100002004002098710010CE
:10D770002DE9F04104462448006800F17E07224864
:10D78000006800F1DE0503263C704FF47A602880C3
:10D79000288825F021FF0421C82000F051FC06460E
:10D7A000012E28D1194890F8380180B91648006830
:10D7B000808B15490968D1F8F410888012480068F8
:10D7C000808E11490968D1F8F41008810FE00E48E5
:10D7D0000068808B0C490968D1F8F41048800A4829
:10D7E0000068808E08490968D1F8F410C880204686
:10D7F00000F0DAF906E02EB90F2003490968D1F8E4
:10D80000F4100870BDE8F081200400209871001029
:10D8100010B5044602200B490968D1F8F4100870CD
:10D8200008490968D1F8F80080470648006803F005
:10D8300031FD0448006803F0A9FD204600F0B4F96A
:10D8400010BD00002004002070B504461549096889
:10D85000D1F8F4108889F2F7B0FF06461249F2F7C2
:10D86000ADFD05461149F2F777FD0E490968D1F87B
:10D87000F41048670B490968D1F8F410C889F2F729
:10D880009CFF06460849F2F799FD05460749F2F75D
:10D8900063FD04490968D1F8F4108867204600F058
:10D8A00083F970BD2004002000F07F450000F03FA8
:10D8B00010B504461B480068D0F8F40080881A4967
:10D8C000488418480068D0F8F40040880884154857
:10D8D0000068D0F8F4000089C88412480068D0F8C5
:10D8E000F400C088888401F057FD0E480068D0F825
:10D8F000F40080880B490968D1F8F41049888842FF
:10D9000006DD002007490968D1F8F410488105E0D8
:10D91000012004490968D1F8F4104881204600F03C
:10D9200043F910BD20040020987100102DE9F0414A
:10D9300080463E48006800F17F063C48006800F1E0
:10D94000E2043A48006800F1E405307800F0800015
:10D9500048BB3648006803F09DFC34490968D1F89B
:10D96000F410888902F0B4FD30490968D1F8F41048
:10D9700008642E490968D1F8F410C88902F0A8FD9E
:10D980002A490968D1F8F410886601202070002027
:10D99000286000F0ACFA0746012F45D1307840F0FE
:10D9A0008000307040E0217801EB81014800F2F7FF
:10D9B000FBFE1E49096888631D491C48006803F086
:10D9C0006DFB2868401C28602868B0F5C87F0FD917
:10D9D00016480068C16D15480068D0F8F400403062
:10D9E000227840F822102078401C20700020286007
:10D9F0000E48006890F8680001280FD10B480068B5
:10DA0000C16D0A480068D0F8F4004030227840F830
:10DA100022102078401C20700020286020780A28DE
:10DA200002DB404600F0C0F8BDE8F0812004002091
:10DA3000140300102DE9F05F07464048006800F12C
:10DA40007F063E48006800F17E0B3C48006800F10C
:10DA5000D4083A48006800F1C8093848006800F165
:10DA6000DE043648006800F1E0054FF0030A307824
:10DA700000F08000F0B98BF8007030480068808BAF
:10DA8000A8F80000FFF7EAF9C9F800002B48006881
:10DA9000D0F8F400008A208020881822002100F0AD
:10DAA000A1F92080208825F097FD307840F0800093
:10DAB000307041E00821282000F086F88246BAF153
:10DAC000010F23D100F0D0F858B91C480068808BB2
:10DAD000A8F80000FFF7C2F9C9F800004FF0000AEB
:10DAE00014E020882880288814490968D1F8F410A7
:10DAF0008989884205DA11480068D0F8F4008089E5
:10DB000000E028882880384600F04EF8BAF1000F6F
:10DB100012D120881822002100F064F9208020888A
:10DB20005F2806DC0A2005490968D1F8F41008705E
:10DB300002E0208825F050FD00F002B8200400200B
:10DB400030BCBDE8C09F00002DE9F04106460F46FD
:10DB5000144603253946304600F036F80546012DB7
:10DB600007D100210F480068C0F8E4100120BDE88B
:10DB7000F08145B90B480068D0F8E400401C094921
:10DB80000968C1F8E40007480068D0F8E400A04242
:10DB900001D80220EBE7002102480068C0F8E41039
:10DBA0000020E4E7200400200649096881F87D0090
:10DBB0000449096891F87D200249096881F87F20AD
:10DBC00070470000200400202DE9F04705460E466E
:10DBD0002448006800F1B8072248006800F1C0043A
:10DBE0002048006800F1D6081E48006800F1D40AF9
:10DBF0001C48006800F1DA09387828B9012038702B
:10DC000025600320BDE8F0872068401E20600028C2
:10DC100001DD0320F6E713480068808BA8F80000B8
:10DC2000BAF80010B8F80020881A002801DB014675
:10DC300000E04142A9F80010B9F80000B04208DB4A
:10DC40000C22002107480068B830FBF7E4FE0120F1
:10DC5000D8E70C22002103480068B830FBF7DBFE50
:10DC60000020CFE72004002070B50A48006800F1CA
:10DC7000C40408480068D0F8C850FFF7EFF82060E7
:10DC800029462068F2F78AFE01D3012070BD0020EA
:10DC9000FCE700002004002070B504460E46207802
:10DCA0003A2810D1641C0948FBF735FF85B22A4693
:10DCB00006492046FBF7DEFC28B90548007840F00D
:10DCC000020003490870002070BD00007CB50020F0
:10DCD0004C0100102DE9F04104460D464FF00008BC
:10DCE0000026022D02DA0120BDE8F08120784128CB
:10DCF00039D16078542836D1022D08D11C4880686B
:10DD000050B31B4800218268084690472DE0A07858
:10DD10002B282AD12946204600F02CF80646FEB1D1
:10DD200006EB4600124901EB80008068A8B106EBC3
:10DD300046010F4A02EB81014868FBF7ECFEC7B2CF
:10DD4000EB1BD9B2E01906EB4603DFF824C00CEB5D
:10DD500083039A689047804607E04FF0030804E089
:10DD60004FF0020801E00120BEE74046BCE700009A
:10DD7000440004082DE9F0410646884600270124A6
:10DD800017E004EB4401104A02EB81014868FBF7FD
:10DD9000C2FEC5B204EB44000B4A02EB80002A46E7
:10DDA00041683046FBF766FC08B9274608E0601C6E
:10DDB000C4B204EB4400044911F820000C28E0D15F
:10DDC00000BF3846BDE8F08144000408024604481C
:10DDD000007840F00100024B1870002070470000EE
:10DDE0004C0100102DE9FC5F07460D4614464FF02C
:10DDF0000008C146384E012D36D13846F2F7DDFC19
:10DE000031460090F2F7DAFA83464FF07E51F2F78E
:10DE1000A0FA824631493046F2F79EFA5146019007
:10DE2000F2F79AFA81466CB12046F2F7C6FC8246B8
:10DE30004946F2F7A9FD03D22046F2F7BEFC00E006
:10DE4000484681463846F2F7B8FC82464946F2F722
:10DE50002BFA804622494046F2F7A0FD01D2204825
:10DE600000E04046804631E085BB3846F2F7A5FC2D
:10DE700083463146F2F7A2FA824618493046F2F755
:10DE80006BFA51460190F2F767FA81466CB1204671
:10DE9000F2F793FC82464946F2F776FD03D220461C
:10DEA000F2F78BFC00E0484681463846F2F785FCE5
:10DEB00082464946F2F74AFA80460A494046F2F756
:10DEC00063FD01D2074800E0404680464046F2F735
:10DED000B0FC80B200F008B800107445CDCCCC3D49
:10DEE00000007A450000BE423CBCBDE8C09F10B5B2
:10DEF000032404230A225F21002000F019F80446BD
:10DF0000012C01D0022010BD0120FCE710B5032434
:10DF100004230A224FF47A61044800F009F8044609
:10DF2000012C01D0022010BD0120FCE70000C842F6
:10DF30002DE9F04F85B005460E4617469846032456
:10DF40002C48006800F1DE092A48006800F1C40A84
:10DF50004FF0000B00200490A9F80060B9F8000011
:10DF600025F03AFB4146384600F06AF80446012C99
:10DF700001D0022C3CD1FEF771FFCAF80000AB467D
:10DF80005946DAF80000F2F7E1F90190F2F79DFC4A
:10DF900021F00041CDE90201F2F7DAFC0490012CF6
:10DFA00009D14FF07E510498F2F7EEFC03D801201E
:10DFB00005B000F021B8012C07D14FF07E51049834
:10DFC000F2F7ECFC01D20020F2E7022C0ED14FF068
:10DFD0007E510498F2F7D8FC08D80C22002105489D
:10DFE0000068B830FBF717FD0120E1E70220DFE70A
:10DFF0000320DDE72004002030BCBDE8C08F000016
:10E0000070B502460B460D480021402401E000F89F
:10E01000011B251EA4F10106B4B2F8D100BF0748C8
:10E0200011461C4603E011F8015B00F8015B251E58
:10E03000A4F10106B4B2F6D100BF70BD7CB50020DA
:10E040002DE9F05F064689463048006800F1B80ABD
:10E050002E48006800F1C0042C48006800F1BC059F
:10E060002A48006800F1D6072848006800F1D8085F
:10E070002648006800F1DA0B9AF8000070B9012018
:10E080008AF800004FF49660286026601F480068F8
:10E09000808BA8F80000032000F03AB82068401EEA
:10E0A0002060002804DD2868401E28600320F3E774
:10E0B00016480068808B3880B8F800103A88881AB3
:10E0C000002801DB014600E04142ABF8001038882F
:10E0D000A8F80000BBF8000048450EDB28680028BF
:10E0E00002DD26600220D7E70C22002107480068E5
:10E0F000B830FBF790FC0020CEE70C22002103484B
:10E100000068B830FBF787FC0120C5E72004002039
:10E1100030BCBDE8C09F000070B505460C46002627
:10E120004F492846F2F73AFC0DD805F0B5FE01211B
:10E130004C48F5F7C4FB012800D100E0002030B9BD
:10E1400014F044FD03E005F099FE14F0F3FC464999
:10E150002046F2F719FC04D344492046F2F71EFC8E
:10E1600001D24FF07E564248407A01285FD14149A2
:10E170002846F2F713FC04D83D4890F837010228EE
:10E1800005D03C492846F2F709FC4DD800BF802154
:10E190003948F5F794FB012800D100E0002030B9A0
:10E1A0000EF0DEFE4FF4FA7003F046FA41E0334819
:10E1B000007800F0040078BB4FF4FA7003F03CFAEA
:10E1C0002E48007800F0010030B9002000F090F8EF
:10E1D0004FF4FA7003F030FA2848007800F001009C
:10E1E000D8B1012000F084F84FF4FA7003F024FA5B
:10E1F0002248007800F0020010B9022000F078F800
:10E20000642003F019FA042000F072F81B4800782B
:10E2100040F00400194908700BE01848007840F0FD
:10E2200004001649087004E04FF07E5601E04FF0FC
:10E230007E564FF07E513046F2F7A6FB0ED180217C
:10E240000D48F5F73CFB012800D100E00020012833
:10E2500001D10EF04DFE01200849087070BD00008C
:10E260003333734000040048000020C20000A04285
:10E27000987100100000F040000C00484C010010A4
:10E2800070B504460D460CB1012100E0002108469E
:10E2900040F24F11F3F704F805B970BD104800685B
:10E2A0001049884200D1F8E70F484068A8B18020A3
:10E2B0000E4909690140814201D1012100E000219C
:10E2C000012901D1012000E00020012805D10649E3
:10E2D0002A464868214630F072FB00BFDDE70000A7
:10E2E000000000200024F40000000010000C004892
:10E2F000F0B5B5B0054600268022002115A8FBF731
:10E30000D6FA0C22002111A8FBF7D1FA54A256A18B
:10E3100011A8F9F7BBFC52A0FBF7EBFBC4B211ABA1
:10E320001A19C4F10C03D9B2C4F10C03C3F11007DC
:10E330004E4BF818FEF72BFD00208DF850002021E1
:10E3400009A8F1F776FF4A4B0FCB05AF0FC7022D97
:10E3500038D003DC3DB1012D7DD114E0042D51D026
:10E36000642D78D15EE000204249087015A8059917
:10E37000F9F78CFC15A8FBF7BCFBC6B2314615A813
:10E38000FFF77EFF68E011AA37A115A8F9F77EFC18
:10E3900015A8FBF7AEFBC7B2394615A8FFF730FE4C
:10E3A0008022002115A8FBF782FA15A80699F9F733
:10E3B0006DFC15A8FBF79DFBC6B2314615A8FFF70B
:10E3C0005FFF49E011AA28A115A8F9F75FFC15A87D
:10E3D000FBF78FFBC7B2394615A8FFF711FE802265
:10E3E000002115A8FBF763FA11AA15A80799F9F7F8
:10E3F0004DFC15A8FBF77DFBC6B2314615A8FFF70B
:10E400003FFF29E000201B49087015A80999F9F77A
:10E410003DFC15A8FBF76DFBC6B2314615A8FFF70A
:10E420002FFF19E04FF066311348CDE90210494241
:10E4300012480A46124BCDE9001012A115A8F9F7AF
:10E4400025FC15A8FBF755FBC6B2314615A8FFF70A
:10E4500017FF01E0FFE700BF00BF35B0F0BD0000CF
:10E46000475344540000000025730000327200102E
:10E47000340004084C01001066660A409999014076
:10E480009999F13F25662C25662C25660D0A00001A
:10E4900010B5044831F0ADFA08220349014831F0C3
:10E4A000C7FB10BDB80000104402001010B50020DA
:10E4B000FDF7AAF900BF1048F5F7F8FC0E48F5F78C
:10E4C00004FD00BF00BF0D48F5F7F0FC0B48F5F761
:10E4D000FCFC00BF05F0D2FC2BF0BEF9002006F0DA
:10E4E0005BFA012006F058FA06F002F816F086FCF6
:10E4F00016F01AFB10BD0000001000400014004090
:10E500001CB500BF04201749886200BF00BF03226A
:10E5100004211448F5F7A1FA00BF00BF2FF01EFC3C
:10E5200011484FF4C8710023104ACDE9001010497A
:10E530001846FDF765FA2BF0FBF9002006F0ACFA5F
:10E54000012006F0A9FA06F055F806F03FF916F09A
:10E550008BFC2DF08BFC02F0BFFB0649064815F042
:10E5600061FD1CBD00040048E07B0B000000024080
:10E5700000000450CDCC4C3EE02F001010B50CF044
:10E58000C1F90446F1F726FE10BD704710B50446E8
:10E590004BF602302CF04EFD012C04D14DF201500F
:10E5A0002CF052FD02E000202CF04EFD10BD0000CA
:10E5B00010B50B4800F098F80A480078012121EACC
:10E5C000900058B900F044F800F0CAF8012805D1CD
:10E5D0004BF602302CF02EFD16F0DAFC10BD0000D8
:10E5E000080000104C010010F8B504460D46002646
:10E5F00011480460114805602BF0E4FF0646012E27
:10E6000001D1012100E000210846B321F2F748FEC4
:10E610000A200B4B0B4A0C4900900C482BF0F8FBDE
:10E620000646012E01D1012100E000210846B62155
:10E63000F2F736FEF8BD00008403002088030020B6
:10E64000292B0308292A0308E5290308912903082F
:10E6500010B52BF0CFFF10BD70B5044665680020E3
:10E6600009498865C86508668864C86408654FF00C
:10E67000E0210861486188610448046020682FF047
:10E680006DFAA84770BD00000010024008ED00E0E0
:10E6900010B54BF602302CF0CDFC0BF08BF84CF69D
:10E6A0000201884218D1F1210020F2F7F9FD002083
:10E6B0002CF0CAFCFFF7FAFE01200849096E8143DD
:10E6C000064A116600BF00071146896D81439165B6
:10E6D00000BF0348FFF7C0FF10BD0000001002405C
:10E6E00000E006087047000038B50446002000909E
:10E6F000206810B15B282AD11FE000BF8021164896
:10E70000F5F7DDF8012800D100E00020012806D14E
:10E71000002016F01FFC012016F0A4FC05E00120EB
:10E7200016F018FC002016F09DFC00BF0B48006896
:10E73000606000BF5B20206000BF08496068096816
:10E74000081A642801D2002038BD00BFD6E7002097
:10E75000206000900320F7E7000C00487C030020B5
:10E7600010B52BF0B1FF10BD70B504460D4616462E
:10E77000034951F824003246294630F020F970BD93
:10E78000000000100149087070470000A403002039
:10E7900038B5044600200090206820B1A0F209207E
:10E7A000002831D126E000BF2CF0D4F82AF0C6FFB3
:10E7B00022F052FDFEF710F922F0FCFB456AA84753
:10E7C000012806D115F05AFB18B90121072018F0CD
:10E7D00033FE2FF0C9FD23F0A1FF2CF0C3F80D4943
:10E7E000088000BF0C480068606000BF40F209204C
:10E7F000206000BF084960680968081A642801D2CF
:10E80000002038BD00BFCFE700202060009003202B
:10E81000F7E70000100000107C03002000F10C035B
:10E8200043F82120704770B504462079A1688847D5
:10E830000546E07800F00700002802DD2088401C33
:10E840002080E078B5EBD01F13D0E078C008401CE2
:10E85000E17860F3C501E170C1F3C20002280CDB6E
:10E86000E07865F3C710E070E07820F03800E070E1
:10E8700003E0E07820F03800E070E07800F0070076
:10E88000062876D2DFE800F00326529DE7C6E0783E
:10E89000C0F38010E178B0EBD11F15D1A07820F043
:10E8A000F000A070E06810B12046E16888470020C1
:10E8B0002080A07820F00F00401CA070E07820F0AD
:10E8C0000700401CE07004E0A07820F0F0008030E9
:10E8D000A070C5E0E078C0F38010E178B0EBD11F04
:10E8E00011D0A07820F0F0001030A070206910B195
:10E8F00020462169884700202080E07820F007002A
:10E90000801CE07011E0208832280EDDA07820F015
:10E91000F0005030A070206A10B12046216A88476C
:10E92000E07820F00700401DE07099E0E078C0F347
:10E930008010E178B0EBD11F1CD1A07820F0F0005E
:10E94000A070E06810B12046E1688847A078401CBC
:10E95000A17860F30301A170606910B1204661697C
:10E96000884700202080E07820F00700C01CE0707D
:10E9700026E070E020880A2822DDA07800F00F0051
:10E9800001280AD1A07820F0F0003030A070A069F2
:10E9900090B12046A16988470EE0A07800F00F00F2
:10E9A000022809D1A07820F0F0004030A070E06982
:10E9B00010B12046E1698847E07820F00700E07058
:10E9C0004EE0E078C0F38010E178B0EBD11F19D0B1
:10E9D000A07820F0F0001030A070206910B120461F
:10E9E0002169884720880A2807DA00202080E078FB
:10E9F00020F00700801CE0700BE0E07820F00700BA
:10EA0000E07006E020880A2803DDE07820F00700A7
:10EA1000E07025E0E078C0F38010E178B0EBD11F22
:10EA20000AD1A07820F0F0006030A070606A88B150
:10EA30002046616A88470DE0A07820F0F000103091
:10EA4000A070206910B1204621698847E07820F045
:10EA50000700E07004E0E07820F00700E07000BFFD
:10EA600000BF70BD2DE9F04104460E4617461D4615
:10EA7000DDF81880204600212C2201E000F8011B5F
:10EA8000131EA2F1010C1FFA8CF2F7D100BFA0787F
:10EA900020F0F0008030A070A6602846A16888476A
:10EAA000E17860F3C711E170E07867F38610E070F9
:10EAB000257184F80580BDE8F08100000146094811
:10EAC000026805E08A4202D14FF0FF307047926A37
:10EAD000002AF7D1034800688862024801600020DC
:10EAE000F4E700000802001010B50548046803E0D0
:10EAF0002046FFF798FEA46A002CF9D110BD000053
:10EB0000080200102DE9F04104462349087AF1F784
:10EB100054FE0546204600F045F81F484088A042B4
:10EB200011D91D484088001B00EB800040001A49A5
:10EB30004988B0FBF1F73846F1F73FFE0646294613
:10EB4000F1F7B2FB0546144841691448F1F736FC69
:10EB50001149886112492846F1F7FEFB06460E4826
:10EB600081693046F1F72AFC0B49C8612046F1F76C
:10EB700024FE80460848C1694046F1F7EDFB074690
:10EB80000749F1F71BFC0646F1F753FE02490884DA
:10EB90000846008CBDE8F08134B5002000007A44BE
:10EBA0000000C8422DE9F0410446134800684FF4C4
:10EBB0007A71B0FBF1F01149486000BF4FF080401E
:10EBC000806AC8602046F1F7F8FD06460B49C9681F
:10EBD000481CF1F7F2FD074608494868F1F7EDFDDA
:10EBE00080463946F1F7EAFB05463146F1F7E6FB88
:10EBF00002494861BDE8F0810000002034B50020E2
:10EC000003B595B0002013901290119010900F90C2
:10EC10000E90159800680990F1F757FE21F0004119
:10EC20000022FE4BCDE90A01F1F706FCCDE90C010B
:10EC3000F1F78EFE1390159800680990F1F745FEE4
:10EC400021F000410022F54BCDE90A01F1F795FCD6
:10EC5000CDE90C01F1F77CFE129015980068079041
:10EC6000F1F733FE21F000410022EC4BCDE9080121
:10EC7000F1F7E2FB0022EA4BCDE90A01F1F700FDD2
:10EC8000CDE90C01F1F708FEC0B2119015980068AB
:10EC90000790F1F71AFE21F000410022DF4BCDE989
:10ECA0000801F1F76AFC0022DD4BCDE90A01F1F71A
:10ECB000E7FCCDE90C01F1F7EFFDC0B2109015981B
:10ECC00000680990F1F701FE21F000410022D44BC9
:10ECD000CDE90A01F1F7D4FCCDE90C01F1F7DCFD37
:10ECE000C0B20F90CF480068407800287ED11198BC
:10ECF000F1F779FD0022CA4BCDE90401F1F74BFC95
:10ED0000CDE908011398F1F7E0FDCDE90601DDE951
:10ED10000823F1F732FC0022C14BCDE90A01F1F7DB
:10ED2000AFFCCDE90C01F1F713FE0E90BD48006871
:10ED3000016D24311198401E51F8200001460B90BE
:10ED40000E98F1F709FB0C90B6480068016D64312C
:10ED50001198401E51F8200001460B900C98F1F7D5
:10ED6000A3FA0D90F1F765FD81B2AE480068C18647
:10ED70001098F1F738FD0022A94BCDE90401F1F715
:10ED80000AFCCDE908011298F1F79FFDCDE90601D3
:10ED9000DDE90823F1F7F1FB0022A14BCDE90A01DF
:10EDA000F1F76EFCCDE90C01F1F7D2FD0E909D4814
:10EDB0000068016D24311098401E51F82000014672
:10EDC0000B900E98F1F7C8FA0C9096480068016D08
:10EDD00064311098401E51F8200001460B900C98A9
:10EDE000F1F762FA0D90F1F724FD00E043E081B203
:10EDF0008C48006881860F98F1F7F5FC0022884B5B
:10EE0000CDE90401F1F7C7FBCDE9080115980068C9
:10EE10000590F1F75AFDCDE90601DDE90823F1F788
:10EE2000ACFB00227E4BCDE90A01F1F729FCCDE9CC
:10EE30000C01F1F78DFD0E907A480068016D2431C8
:10EE40000F98401E51F8200001460C900E98F1F7E3
:10EE500083FA0D9073480068016D64310F98401E6D
:10EE600051F8200001460C900D98F1F71DFA6D49FC
:10EE70000968C861C5E06B48006840780128F9D18D
:10EE80001198F1F7B0FC0022654BCDE90401F1F7D0
:10EE900082FBCDE908011398F1F717FDCDE90601D2
:10EEA000DDE90823F1F769FB00225D4BCDE90A019A
:10EEB000F1F7E6FBCDE90C01F1F74AFD0E90594858
:10EEC0000068016D24311198401E51F82000014660
:10EED0000B900E98F1F740FA0C9052480068016DC3
:10EEE00064311198401E51F8200001460B900C9897
:10EEF000F1F7DAF90D90F1F79CFC81B2494800680E
:10EF0000C1861098F1F76FFC0022454BCDE9040152
:10EF1000F1F741FBCDE908011298F1F7D6FCCDE9F4
:10EF20000601DDE90823F1F728FB00223C4BCDE97F
:10EF30000A01F1F7A5FBCDE90C01F1F709FD0E90EF
:10EF400038480068016D24311098401E51F82000A7
:10EF500001460B900E98F1F7FFF90C9031480068CC
:10EF6000016D64311098401E51F8200001460B904D
:10EF70000C98F1F799F90D90F1F75BFC81B22948F3
:10EF8000006881860F98F1F72EFC0022244BCDE912
:10EF90000401F1F700FBCDE9080115980068059020
:10EFA000F1F793FCCDE90601DDE90823F1F7E5FA75
:10EFB00000221B4BCDE90A01F1F762FBCDE90C0100
:10EFC000F1F7C6FC0E9017480068016D24310F98C8
:10EFD000401E51F8200001460C900E98F1F7BCF944
:10EFE0000D9010480068016D64310F98401E51F873
:10EFF000200001460C900D98F1F756F9094909686F
:10F00000C861169800680B90F1F75FFC21F0004191
:10F010000022054BCDE90C0108E00000000014407F
:10F0200000002440600100100000E03FF1F760FCA8
:10F0300071D83A480068C08E0190F1F7BEFB02908B
:10F0400036480068C069014601900298F1F77EF9E0
:10F050000390F1F73AFC21F00041CDE90601169842
:10F0600000680390F1F731FC21F00041CDE9040183
:10F07000DDE90623F1F78FFACDE90A012748006898
:10F08000C08E0790F1F7AFFBCDE90801DDE90A2357
:10F09000F1F773FACDE90C01F1F7FEFB81B21F48DD
:10F0A0000068C1861D480068808E0190F1F785FBDD
:10F0B00002901A480068C069014601900298F1F771
:10F0C00045F90390F1F701FC21F00041CDE906017B
:10F0D000169800680390F1F7F8FB21F00041CDE9A4
:10F0E0000401DDE90623F1F756FACDE90A010B48E0
:10F0F0000068808E0790F1F776FBCDE90801DDE925
:10F100000A23F1F799F9CDE90C01F1F7C5FB81B2BA
:10F1100002480068818617B000BD00006001001041
:10F120002DE9F04F8BB082460AF154040AF1080928
:10F130004FF0000B00200A902422354901A8F1F776
:10F1400051F8D4E90321891AA28801FB02F0F1F7F2
:10F150004AFB074600222F4BF1F792FA0546F1F7DA
:10F16000F7FB0A90D4E90601F1F7F0F807462A49BF
:10F17000F1F7F2F805464FF082406169F1F7ECF8DB
:10F1800006462946F1F71AF983462178890901EBE9
:10F19000410101AA52F821005946F1F7DDF8C9F8FA
:10F1A0002C002178890901EB410101AA02EB8101C0
:10F1B00048680A99F1F7D0F80646A088F1F7FDFAF9
:10F1C0000746D9F82C10F1F7C7F805463146F1F794
:10F1D000F5F8C9F83000A088F1F7EFFA0646227872
:10F1E000920902EB420201AB03EB82029168D9F86B
:10F1F0002C00F1F7B1F807460A99F1F7ADF805468A
:10F200003146F1F7DBF8C9F834000BB000F006B86E
:10F210000402040800408F40DB0F494030BCBDE8C9
:10F22000C08F70470D48C1880089814212D00B48B9
:10F2300000890A49C988401A04D50848C18800894C
:10F24000081A04E0054800890449C988401AB0F545
:10F250007A7F00DA704700BFFCE70000747400108A
:10F260002DE9FC5F07460D4690461E46DDF83090BE
:10F27000C7EBC7001C4901EB80040CB1012100E081
:10F280000021084640F2ED21F2F70AF84FF0000A9B
:10F29000D3460020019000906580A4F80480C4F853
:10F2A0001090E660E1884819F1F77EFA82462189DC
:10F2B0004819F1F779FA834631464846F1F746F89E
:10F2C000019051465846F1F741F80090DDE90010F1
:10F2D000F1F774F86061012020701821204600F0D9
:10F2E00097FFA06100F002B8747400103CBCBDE848
:10F2F000C09F000010B504462448006818B1234898
:10F3000000682EF066F94FF4807120462EF06BF9FC
:10F310001E490860096809B1012100E00021084682
:10F320005921F1F7BDFF1A481849096808611949C0
:10F330001648006841611C220021144800682EF024
:10F3400087F81C220121114800682EF081F81C2248
:10F3500002210E4800682EF07BF81C2203210B4886
:10F3600000682EF075F81C220421084800682EF071
:10F370006FF81C220521054800682EF069F81C2250
:10F380000621024800682EF063F810BD98000010B6
:10F390000D4701084B47010808B51148018C114879
:10F3A00041840F48418C0F4881840F4800231A463E
:10F3B000194600900120FFF753FF0948818C094846
:10F3C000A0F892100648C18C0648A0F89410064890
:10F3D00000231A46194600900520FFF741FF08BD9B
:10F3E00098710010747400100000C8422DE9F041BB
:10F3F00004460E4617461D463A46314604F1C00003
:10F400002CF0AEFE2A4604F1F80104F168002CF05D
:10F41000A7FED4F8F810C4F81811BDE8F0817FB544
:10F4200006460C461546617806F15800E2682CF055
:10F4300072FF69783046EA682CF06DFF04F13C00F9
:10F4400004F1340104F12C0204F11C03CDE9003273
:10F45000CDE902101B1F183A243906F158002CF090
:10F460002FFF05F13C0005F1340105F12C0205F1F7
:10F470001C03CDE90032CDE902101B1F183A2439D4
:10F4800030462CF01DFF7FBD2DE9F041C1F30A523B
:10F49000A2F2FF362F4A304B0D460446142E2FDAC7
:10F4A000002E12DAF0F7C8FF00221346F1F738FAFF
:10F4B0004CD2002DBCBF4FF00045002446DB55EA7E
:10F4C000040018BF254D19D140E0DFF894C02CFA94
:10F4D00006F705EA070C5CEA040C08BFBDE8F081FA
:10F4E000F0F7AAFF00221346F1F71AFA2ED2002DE8
:10F4F00003DD4FF48010F0400544BD43002425E0B7
:10F50000332EC8BFBDE8F081A6F1140C4FF0FF37D1
:10F5100027FA0CF73C4208BFBDE8F081F1F730F85C
:10F5200000221346F1F7FCF910D2002D0DDD142E48
:10F5300008BF6D1C09D0C6F13400012101FA00F0AA
:10F540002044A04238BF6D1C0446BC4329462046D7
:10F55000BDE8F0819C7500883CE4377E0000F03FF8
:10F56000FFFF0F002DE9F041044600BF404800684E
:10F5700040F480303E49086000BF00BF00BF3C48F7
:10F580000068C0F340400028F8D00220F4F7EAFBFE
:10F5900000BF00BF3648806800F00C000828F8D192
:10F5A00000BF3348006820F080703149086000BF18
:10F5B00000BFF4F7CFFB0028FBD194E80F0040EA2E
:10F5C000010545EA02251D43294EF668294F3E40B4
:10F5D0003543274EF56000BF00BF3046C06840F09D
:10F5E00080703146C86000BF00BF0846006840F028
:10F5F0008070086000BF00BFF4F7ACFB0128FBD1AE
:10F600000320F4F7AFFB00BF00BF1948806800F08B
:10F610000C000C28F8D120691549896821F0F00107
:10F620000143134A916000BF60691146896821F463
:10F63000E0610143916000BFA0691146896821F42F
:10F6400060510143916000BFE069F4F72DFAE06971
:10F65000F4F7F6FB0849E0690862084800680849C1
:10F66000B0FBF1F085B2284601F0E0FFBDE8F08183
:10F67000001002408C80FFF960EF002000000020A5
:10F6800040420F002DE9F84F04460025A9464FF0EF
:10F690007E56DFF8BCA00020009094F8980030B9A6
:10F6A000002004F14400C568D0F8449006E0002032
:10F6B00004F144008569D0F8389000BF49462846D7
:10F6C000F0F74AFE07460021F1F768F93DD2002124
:10F6D0002846F1F759F902D285F0004000E02846AB
:10F6E00007463146F1F750F903D84FF07E500090AD
:10F6F0002BE051463046F0F7D7FD804600212846E2
:10F70000F1F742F902D285F0004000E028460746B2
:10F710004146F1F739F916D800212846F1F734F9B6
:10F7200002D285F0004000E0284683465146F0F7BB
:10F7300010FE80463146F0F7B7FD07465146F0F718
:10F740003DFE009001E000200090009800F002B81B
:10F750000000204118BCBDE8E08F2DE9F0410446CF
:10F760000D4617462E46207840B1A078032805D1D3
:10F77000012086F83000304609F065FF0020BDE822
:10F78000F081FEB504460D4617462E46607848B116
:10F790002078032806D12146304622F0CDFCD8B18E
:10F7A0000120FEBD207801280AD10521CDE90010F5
:10F7B000062302AA3046216DF9F702FA0120F0E78C
:10F7C000607848B12078022806D1A27804F11001AF
:10F7D0003046236D2FF016FA0020E2E72DE9F041C4
:10F7E00005460F46002600242BE005EB841101F1AD
:10F7F0001C0007F083FA064606B921E005EB8410E9
:10F80000406BF169884217DB9022104910A0F8F78D
:10F8100019FA05EB8410F369426B05EB8410011DA6
:10F820001248F8F70FFA12A0F8F70CFA0020124964
:10F830000860401EBDE8F081104840F8246000BF19
:10F84000641CBC42D1D30020F4E70000F402050898
:10F850001B5B33313B32326D5B452F46414C5D20A3
:10F860002825733A25642920000000000445050876
:10F870001B5B306D0A0000003404002000300010D3
:10F8800030B503460D4614462078012807D1587834
:10F89000032802D05878022801D158682860587887
:10F8A0002070002030BD2DE9F04105460C4616467B
:10F8B000287888B92746B0463868401C386098F8E0
:10F8C0001A0010B10120BDE8F0814FF0FF32404630
:10F8D000696808F045FA00BF0020F4E72DE9F0411F
:10F8E00005460F4690463C462668287818B9012000
:10F8F0002071BDE8F081687802280CD1F06A401CC4
:10F9000030B92822294606F12800F0F76BFC16E0F2
:10F9100001202071EDE76878012810D1A068401C13
:10F92000A0606868E060A068012808D1F06A401C07
:10F9300028B92822294606F12800F0F753FC0020B8
:10F94000D7E700002DE9F0413D48006800F12404AC
:10F9500042F210753A480068007F10B9002039491A
:10F9600001E0002038490246F0F7F2FF074613F0A5
:10F970001FFE012851D13248216B006800F5187034
:10F9800015F011FF4FF492710851284620F03EFB0C
:10F990004FF488710B590959491C4FF48872115161
:10F9A000984223D83A46282104F5947020F016FE98
:10F9B00060B1012084F80C01002084F8C801207097
:10F9C0004FF48C700159001D015112E04FF4887101
:10F9D0000859F0F7F2FE80461C49F0F7BDFC0646D8
:10F9E000F0F727FF4FF48871085102E0002084F8F7
:10F9F0000C014FF4927001594FF48C700151014683
:10FA0000085920F087FC4FF48A7108530C480068AD
:10FA100081694FF4907001510FE000214FF488701C
:10FA20000151002084F80C014FF48C7001510448FE
:10FA3000006800F5187015F0A1FEBDE8F081000027
:10FA400020020010000019400000E43FCDCC4C3EE5
:10FA500070B504460CB1012100E00021084640F2D7
:10FA60002F11F1F71DFC254614B100202881688173
:10FA700070BD70B50446002500260CB1012100E0E0
:10FA80000021084640F23711F1F70AFC256805E02D
:10FA90002E466D683046F9F7D1FB0026002DF7D1D0
:10FAA0000020206070BD10B504460CB1012100E0BB
:10FAB000002108461321F1F7F3FB0020206010BD60
:10FAC0002DE9F04104460F460CB1012100E0002170
:10FAD00008464A21F1F7E4FB3846F1F7D3FB054627
:10FAE000206810B92560BDE8F081266800E07668DE
:10FAF00070680028FBD1756000BFF4E770B505465B
:10FB00000C46FE2104F580742268501C20601170A0
:10FB10004948B0F86B00010A2268501C206011703F
:10FB2000454890F86B102268501C20601170052128
:10FB30002268501C206011700EF096F92268511C4A
:10FB4000216010703C4890F868102268501C2060BA
:10FB50001170394890F869102268501C20601170AB
:10FB6000354890F871102268501C20601170206890
:10FB7000401C2060206803222F49491DF9F72DFE03
:10FB80002068C01C2060A4F5807495F88E000128C0
:10FB900003D12948B0F82D0102E02748B0F82F0121
:10FBA00006460EF061F9072844D1234890F86A1000
:10FBB00004F580742268501C206011700A212268AC
:10FBC000501C20601170310A2268501C2060117096
:10FBD0002268501C20601670174890F8AE1A2268F0
:10FBE000501C206011701448B0F86D00010A2268A2
:10FBF000501C20601170104890F86D102268501C45
:10FC0000206011700C48B0F86F00010A2268501C87
:10FC100020601170084890F86F102268501C206016
:10FC20001170054890F867102268501C2060A4F5F8
:10FC30008074117070BD00002013001070B5044670
:10FC40000D46164632462946204609F09FFA70BDF9
:10FC50000021416006218170704700007CB51B487F
:10FC6000006800F12404684615F01AFA1848DDE926
:10FC700000120369001D98471548E26B616B036C25
:10FC8000001D9847206394F80C01012815D113F04A
:10FC9000E5FC012811D00D480068007F68B920F00C
:10FCA00019FF007848B90B4A282104F5947020F018
:10FCB00095FC10B1606B15F0DEFA206B20F02AFB8A
:10FCC0000546284620F0C6FA7CBD00002002001040
:10FCD000100300100000A03E704700002DE9F0471F
:10FCE0005948006800F1240457480068D0F8208083
:10FCF000002509F02DFDA0845349096888825348E6
:10FD0000007F012840D1A08CFBF75AFD054694F8EE
:10FD10000C0101283FD12846616BF0F717FB8246A2
:10FD20000021F0F731FE06D22846616BF0F70EFB9A
:10FD300080F0004003E02846616BF0F707FB814646
:10FD4000F0F7C3FD06460022414BF0F7E9FD22D84B
:10FD50002846616BF0F7FAFA07460021F0F714FE27
:10FD600006D22846616BF0F7F1FA80F0004003E01C
:10FD70002846616BF0F7EAFA06463649F0F704FECA
:10FD800009D83548456A06E0002598F801000228A0
:10FD900001D1FFF701FB13F0C7FB012807D129466A
:10FDA0002948006800F50D7014F05AF905462A48F4
:10FDB00045620146486A0AF093FB2749C867224812
:10FDC0000068007F012804D01F480068007F0428D5
:10FDD00004D1616B6163616BA1630AE01E48816FAE
:10FDE000A163816F1848006800F5157015F07CFC60
:10FDF0006063322104F14400626B20F01BFC164862
:10FE0000C16FE163616BE06BF0F7A0FA206420F052
:10FE100063F80646216BF0F7B7FD04D820F05CF8D4
:10FE20000D4908670EE020F055F80646216BF0F703
:10FE3000B5FD04D820F04EF80749086702E00649EE
:10FE4000206B0867BDE8F087200200107474001072
:10FE50000000E43F000020417802001070B5064623
:10FE60000D460948405D012801D1112405E00648EE
:10FE7000405D08B9102400E00324044800EBC401ED
:10FE8000304616F0B3FB70BD2072001010F304086A
:10FE90002DE9F0470024A14655490968486AF0F762
:10FEA00014FD21F0004107460022524BF0F7E8FB19
:10FEB0000546F0F7F1FC84B24D490968486AF0F74D
:10FEC00004FD21F000410546F0F7E6FC80B20A216E
:10FED00090FBF1F201FB120060BB45490968486ADA
:10FEE000F0F7F3FC21F0004105460022414BF0F70A
:10FEF00017FD1FD83E480068407850B93C49096852
:10FF00000A6D611E32F81100F0F757FC3A4908609B
:10FF10006AE0374800684078012865D134490968AB
:10FF2000096D1231621E31F81200F0F746FC3249B9
:10FF3000086059E02E480068407840BB04EB84011B
:10FF40004800F0F731FC064629480068416A30460F
:10FF5000F0F7FFF905462949F0F730FA81462448C1
:10FF60000068006D2430621E50F822104846F0F7F9
:10FF7000F3F905461E480068006D6430621E50F8B3
:10FF800022102846F0F790F91B4908602CE0184829
:10FF900000684078012827D104EB84014800F0F77D
:10FFA00003FC064612480068416A3046F0F7D1F972
:10FFB00005461249F0F702FA81460D480068006DC7
:10FFC0004430621E50F822104846F0F7C5F9054645
:10FFD00007480068006D8430621E50F822102846E1
:10FFE000F0F762F90449086003480068BDE8F0874B
:10FFF0006001001000002440740100100000204146
:020000040801F1
:1000000070B5049C4FF461654D43C2EB021605EBDD
:1000100086051D4405EB4506C6EBC51504EBC50575
:10002000056005686D01056070BD10B50B7814782A
:10003000634003704B785478634043708B789478B6
:1000400063408370CB78D4786340C3700B791479A4
:10005000634003714B795479634043718B79947990
:1000600063408371CB79D4796340C3710B7A147A7E
:10007000634003724B7A547A634043728B7A947A6A
:1000800063408372CB7AD47A6340C3720B7B147B58
:10009000634003734B7B547B634043738B7B947B44
:1000A00063408373CB7BD47B6340C37310BD0A78FA
:1000B00002704A7842708A788270CA78C2700A796F
:1000C00002714A7942718A798271CA79C2710A7A57
:1000D00002724A7A42728A7A8272CA7AC2720A7B3F
:1000E00002734A7B42738A7B8273CA7BC2737047F6
:1000F00010B503E011F8013B00F8013B131EA2F11B
:100100000104E2B2F6D110BDF0B506460C46002758
:100110000025FA2C08D0204609F01EFD0746387845
:10012000FA2801D10020F0BD304609F003FD054654
:100130002878FA2801D10020F5E76C700120F2E759
:1001400070B505460C460026012D06D0032D09D0BA
:10015000052D0CD0082D11D10EE02078F0F72DFBE5
:1001600006460CE02088F0F728FB064607E02068EA
:10017000F0F723FB064602E0266800E000BF00BF60
:10018000304670BD017801F1640202707047018849
:1001900001F5FA62028070470178A1F164020270F1
:1001A000704700000EB50A49096800910849091D09
:1001B0000968019106490831096802910099C90846
:1001C000019A01EB5201029A01EB92000EBD000070
:1001D0009075FF1F70B502464FF6FF70134600245E
:1001E00013E013F8015B684000250AE000F0010607
:1001F00026B148F2014686EA600000E040106E1C1D
:10020000F5B2082DF2DB651CACB28C42E9DB70BDA7
:1002100070B505460E4609F04BFA4FF0FF3400204A
:1002200008E0295C6140C9B2044A52F8211081EA11
:100230001424401CB042F4D3E04370BD84EF00208E
:10024000F0B502463125FF20002311E012F8016BC2
:100250007040002409E000F080061EB1312686EAD5
:10026000400600E04600F0B2641C082CF3DB5B1C87
:100270008B42EBDBF0BD00002DE9F04F89B0064664
:100280000F4690469946DDF848B0002400200290C1
:100290007D694046EFF7E4FF402803D9052009B007
:1002A00000F0C0B8FF22182103A8EFF7BBFF5C489D
:1002B00004904046EFF7D4FFC0B28DF81C00CDF893
:1002C00020B09DF81C00014618310898084405909C
:1002D0000599F0681038814201D90720DFE7681CD2
:1002E00040B939463046059A22F0D4F80546401CFC
:1002F00000287DD034B902AB39463046059A2EF03D
:100300002FFD0446002C45D1FF20019000200690CF
:10031000042207A9069806F0DBFF0690042208A92C
:10032000069806F0D5FF06909DF81C2041460698D9
:1003300006F0CEFF06909DF81C009DF81C10A0EB67
:10034000010A05E0012201A9069806F0C1FF069006
:10035000BAF10000AAF1010AF4D14946089A0698B8
:1003600006F0B6FF069008990898A0EB010A05E090
:10037000012201A9069806F0ABFF0690BAF1000031
:10038000AAF1010AF4D103AA294630462FF03CFD18
:10039000044600BFF4B99DF81C30424605F118012F
:1003A0003046FCF7C0F904469DF8080058B99DF89E
:1003B0001C00034605F11800034408981A1830463B
:1003C00079682EF055FD9DF81C202B46414630469D
:1003D0002EF018FC5CB99DF81C00024605F11800CF
:1003E00011184A463046089BFCF79DF9044600E088
:1003F00013E054B901200221062303AACDE900101D
:1004000029463046F8F7DCFB04462CB99DF8080075
:1004100010B1012086F8300000E0072420463EE7B6
:100420004B56303030BCBDE8C08F00002DE9F05F86
:1004300004460E460CB1012100E00021084640F2BE
:100440001721F0F72DFF0EB1012100E00021084631
:100450004FF40671F0F724FF354600271848C08A8C
:100460004EF23F61884205D12946204600F0DBF973
:10047000E06505E0226CA16B2846AB689847E06513
:100480005421085BF0F799F9824652210A5B542106
:10049000095B501AF0F788F98346E16DEFF75CFFCE
:1004A00081460849EFF78AFF80465146EFF7FCFE88
:1004B00007463846F0F7BDF980B200F005B80000F5
:1004C000987100100000C84230BCBDE8C09F000019
:1004D0002DE9F0410446002510490968D1F8F410CF
:1004E000098A0E4A1268D2F8F420528A881AF0F764
:1004F0005BF9074609490968D1F8F410498A601A7E
:10050000F0F752F980463946EFF758FF064604499E
:10051000EFF722FF05462846BDE8F08120040020C1
:100520000000C8422DE9F04104460025A06CF0F718
:10053000CCF921F000410646F0F70AFA05464FF0E3
:100540007E512846F0F720FA03D8A06F401CA06720
:1005500003E00021A16784F86810A06FC82804D3C5
:100560000021A167012184F86810BDE8F081000036
:1005700010B50446204600F09EFB05494862486AD3
:1005800009F0AEFF0249C8670846C16F216410BD7B
:100590007802001070B504460E4AE16B906FEFF7D9
:1005A000D5FE054625F0004006460B493046F0F7DB
:1005B000F5F908D2012184F867100648816FE163DC
:1005C000216C616402E0002184F867100148806FAB
:1005D000A06370BD78020010CDCC4C3E2DE9FF5FCA
:1005E000044689464D4600200390002782468748EE
:1005F00002904FF000088649A06BEFF7DFFE8346BC
:10060000F0F717F986B25EB9D4F8F4004030711CE7
:1006100050F82170D4F8F400403050F826800BE0F8
:10062000D4F8F4004030711C50F82170D4F8F40074
:100630004030711E50F821805020005D012851D1BA
:100640000021A06CF0F7A0F903D2A06C80F000406C
:1006500000E0A06C83466F49F0F7A0F908D2D4F807
:10066000F400D0F840A0D4F8F400806E0290B3E01B
:100670000021A06CF0F788F903D2A06C80F0004054
:1006800000E0A06C83464FF07E51F0F787F926D248
:100690000021A06CF0F778F903D2A06C80F0004044
:1006A00000E0A06C83465B49F0F76EF917D8D4F8E8
:1006B000F400D0F840A00021A06CF0F765F903D257
:1006C000A06C80F0004000E0A06C53490190EFF76F
:1006D00043FE83463946EFF7E7FD02907CE0C246D1
:1006E000029779E00021A06CF0F74EF903D2A06CDC
:1006F00080F0004000E0A06C83464649F0F74EF9D8
:1007000024D2D4F8F410C86F4FF08041EFF724FEE4
:1007100001900021E06CF0F737F903D2E06C80F033
:10072000004000E0E06C3D490090EFF715FE834685
:100730000199EFF7B9FD0390AA69284603999047FC
:100740000297D4F8F400D0F840A045E00021A06C56
:10075000F0F71AF903D2A06C80F0004000E0A06C22
:1007600083464FF07E51F0F719F927D20021A06C93
:10077000F0F70AF903D2A06C80F0004000E0A06C12
:1007800083462449F0F700F918D8D4F8F400C06F74
:100790000390AA6928460399904702970021A06C0C
:1007A000F0F7F2F803D2A06C80F0004000E0A06CFB
:1007B00083464146EFF7CDFD82460DE0D4F8F410B4
:1007C000C86F4FF08041EFF7F9FD0390AA69284602
:1007D00003999047C24602970C490298F0F7DEF859
:1007E00001D20A4800E00298029000215046F0F73A
:1007F000CBF801D2002000E050468246EB6851461B
:100800002846029A984700F00BB800000000C84242
:10081000000020410000A040CDCCCC3DCDCCCC3C54
:100820003FBCBDE8C09F2DE9F04104460D462E4671
:10083000002794F86800012801D1E76D05E0226CDB
:10084000A16B3046B368984707463846BDE8F0814B
:100850002DE9F84F04460F463D464FF00009DFF8FA
:1008600050A2002000905020005D01286BD1002193
:10087000E06CF0F789F803D2E06C80F0004000E013
:10088000E06C83468B49EFF767FD06468A493046A0
:10089000F0F77AF801D2884800E0304606468749EA
:1008A000A06BEFF753FD83460021F0F76DF801D2FE
:1008B000002003E08149A06BEFF748FD80467C49AA
:1008C0004046EFF77BFD8346A16CEFF745FD804680
:1008D0003146A06CF0F762F818D2D4F8F410888989
:1008E000FFF7F6FD8146DFF8C8A1D4F8F410C86F11
:1008F0004FF08041EFF730FD834659462846AA69FC
:10090000904700212846EA699047B7E04FF07E51B2
:10091000A06CF0F743F8F8D24FF00009D4F8F410C7
:10092000C889FFF7D5FD83464146EFF7BDFC8246F7
:10093000D4F8F400C16F2846AA69904701212846DF
:10094000EA6990479AE00021E06CF0F71DF803D2C5
:10095000E06C80F0004000E0E06C83464FF07A519C
:10096000EFF7FAFC064654493046F0F70DF801D28D
:10097000514800E03046064686F0004B5846A16CD0
:10098000F0F70CF81FD254F8F41FC889FFF7A0FD48
:1009900083464B49EFF788FC82462168488AFFF777
:1009A00097FD814654F8F419C86F4FF08041EFF776
:1009B000D3FC834659462846AA6990470021284619
:1009C000EA6990475AE03F49A06CEFF7DDFF37D264
:1009D000D4F8F410C889FFF77BFD83463849EFF758
:1009E00063FC82463849A06BEFF7D8FF17D2D4F8E2
:1009F000F400C089D4F8F410898900EB010B0BEBEB
:100A0000DB714810EFF7D0FE00900098EFF711FF70
:100A10001FFA80FB5846FFF75BFD814605E0D4F8DE
:100A2000F4108889FFF754FD8146D4F8F400C16FB3
:100A30002846AA69904701212846EA6990471DE0A7
:100A4000D4F8F410C889FFF743FD83461C49EFF73B
:100A50002BFC8246D4F8F4108889FFF739FD8346D1
:100A6000A16CEFF721FC8146D4F8F400C16F284651
:100A7000AA69904701212846EA6990470C495046E7
:100A8000EFF78CFF01D20A4800E050468246002171
:100A90004846EFF779FF01D2002000E04846814642
:100AA000524649462846EB68984700F00FB80000C8
:100AB0000000C842A4707D3F0000C04000004842D2
:100AC0000000A040000080BF0000964218BCBDE8B6
:100AD000E08F000070B504460D46D4F8F400418A5A
:100AE00054200153D4F8F400018A52200153D4F861
:100AF000F400D0F88C102166207803280AD1D4F8AD
:100B0000F400418A54200153D4F8F400018A5220A1
:100B1000015314E00A48C08A4EF23F61884204D172
:100B200029462046FFF75AFD09E00548C08A4EF2E3
:100B30004061884203D129462046FFF789FE70BDF7
:100B4000987100102DE9F04104460E46354600210B
:100B5000A06CEFF719FF03D2A06C80F0004000E01A
:100B6000A06C07464FF07E51EFF70EFF10D2D4F87D
:100B7000F410D1F880002549EFF7EEFB074639461F
:100B800028462A6A9047012128466A6A90473BE036
:100B90000021A06CEFF7F8FE03D2A06C80F00040BB
:100BA00000E0A06C07464FF07E51EFF7F7FE20D82B
:100BB0000021A06CEFF7E8FE03D2A06C80F00040AB
:100BC00000E0A06C07461249EFF7DEFE11D2D4F820
:100BD000F410D1F880004FF07C51EFF7BDFB0746D1
:100BE000394628462A6A9047002128466A6A904773
:100BF0000AE0D4F8F400D0F8801028462A6A90471A
:100C0000002128466A6A9047BDE8F081CDCCCC3DF2
:100C10000000A04070B504460D46204600F026F8BE
:100C200029462046FFF78EFF29462046FFF752FF50
:100C30002046FFF777FC70BD70B504460025012102
:100C400084F864100749A06BEFF7A8FE02D84FF4B0
:100C50007A6505E00449A06BEFF796FE00D85F25A2
:100C6000284670BDCDCCC742CDCCCC3D10B5044696
:100C700094F86400012807D1002184F86410002052
:100C8000A070204600F006FB94F86700012811D1FF
:100C9000A16B206CEFF778FE01D2012100E000216A
:100CA00050200155002184F86510616CA06BEFF7AE
:100CB0004DFBE06410BD70B50446A08BEFF77DFDE1
:100CC00005462846EFF7B5FD86B23046FAF778FDBF
:100CD0000546284670BD000010B52021084809F0DF
:100CE00061FF084908600121952000F0A2F8012168
:100CF000880200F09EF80121AA2000F09AF810BDA9
:100D000000100048640200107CB511480068416979
:100D10000069CDE900010E4804680068856894E820
:100D20000F00A847FA2000F0A7FC09480168D1E9A4
:100D30000401CDE90001064804680068C56894E82C
:100D40000F00A84740F2EE2000F096FC7CBD0000AA
:100D5000640200107CB51148006841690069CDE962
:100D600000010E4804680068856894E80F00A847F1
:100D700040F2EE2000F080FC08480168D1E904014F
:100D8000CDE90001054804680068C56894E80F00D3
:100D9000A847FA2000F070FC7CBD0000640200103F
:100DA00070B5044606492046EFF7D6FA0646EFF737
:100DB00040FD85B20021284600F03BF870BD0000E0
:100DC00000AA2A457CB51148006841690069CDE94F
:100DD00000010E4804680068856894E80F00A84781
:100DE0004FF4FA7000F048FC08480168D1E90401AA
:100DF000CDE90001054804680068C56894E80F0063
:100E0000A8474FF4FA7000F037FC7CBD6402001074
:100E100010B5044614B1012C06D102E0FFF774FFAF
:100E200005E0FFF797FF02E0FFF7CCFF00BF00BF30
:100E300010BD2DE9F04706460F46F4B24FF0000909
:100E400007E004F0010018B109F1010000F0FF090A
:100E50006410002CF5D109F0010008B1A14601E0B1
:100E60004FF00109340A002505E004F0010008B143
:100E7000681CC5B26410002CF7D105F0010008B160
:100E8000002500E001257D400220FFF7C1FF384624
:100E9000FFF7BEFF34464FF0000811E004F40040B5
:100EA00018B10120FFF7B4FF02E00020FFF7B0FF08
:100EB0004FF6FF7000EA440408F101001FFA80F8C1
:100EC000B8F1100FEADB2846FFF7A2FF4846FFF70C
:100ED0009FFF0220FFF79CFFBDE8F08710B5044696
:100EE00094F87C00012802D0204600F0AFF87D2065
:100EF000005D12287BD2DFE800F00910171E252CB8
:100F00003341483A4F565D646B858E9501218020B0
:100F100001550120FCF72CFC91E0012180200155B6
:100F20000220FCF7D5FB8AE0012180200155032037
:100F3000FCF7BEFC83E00121802001550420FCF772
:100F40009FFA7CE00121802001550520FBF7A8FFD6
:100F500075E00221802001550620FCF7E5FA6EE0DD
:100F60000221802001550920FBF722FF67E00221C2
:100F7000802001550720FCF7C1F960E002218020A4
:100F800001550820FCF728FA59E00221802001557C
:100F90000A20FCF74FFD52E00221802001550B2072
:100FA000FCF7AEF84BE00221802001550C20FCF745
:100FB0002DF944E00221802001550D20FBF7C4FFEC
:100FC0003DE00221802001550E20FCF73DFC36E07B
:100FD00004211C48006880F880101B48C08A4EF22B
:100FE0003F61884204D10F20FCF71AFB09E021E0A1
:100FF0001548C08A4EF24061884202D11020FCF7A9
:101000000FFB1CE004210F48006880F880101020BE
:10101000FCF78CFC13E00521802001551120FCF722
:10102000F7FB0CE00521802001550648006800F020
:1010300022F804E00348006800F01DF800BF00BF7C
:1010400010BD0000200400209871001010B5044667
:1010500090220021D4F8F400F8F7DDFC00217D2077
:101060000155015D7F200155012084F87C00D4F8F2
:10107000F410087010BD70B504460325FCF737FF67
:101080000546012D08D16C22002104F17C00F8F7FF
:10109000C2FC012000F02CF970BD00002DE9F34FD7
:1010A000A5B082464F4800680078012802D150461A
:1010B000FFF770FA5046FFF75BFADAF84010DAF8FB
:1010C0003800EFF743F9CAF8480012F037FECAF8C3
:1010D0006C00DAF87400401CCAF87400DAF8740086
:1010E0001421B0FBF1F201FB1200002839D13E4877
:1010F000007800F00400002830D04FF0000B802270
:10110000002105A8F8F787FCDAF84800EFF7DDFBC7
:1011100004460D46DAF84000EFF7D7FB06460F46C7
:10112000DAF83800EFF7D1FB804642460B462FA194
:1011300005A8CDE90067CDE90245F6F7A7FD05A8AA
:10114000014600E0491C0A78002AFBD10A1A02F085
:10115000FF0B594605A809F09FFD00BF0021CAF802
:1011600074102549DAF83800EFF718FC05D923493F
:10117000DAF83800EFF708FC11D85046FFF75CFDAD
:101180000446EFF71AFBCAF8580001208AF802005B
:10119000DAF85800EFF74DFBAAF8040015E05046C6
:1011A0002699FFF737FD01208AF80200504626995C
:1011B000FFF73CF90446EFF700FBCAF85800DAF8ED
:1011C0005800EFF736FBAAF804000648006880785C
:1011D000012804D103490968888822F0FDF927B065
:1011E00000F00EB8200400204C01001025662C25CC
:1011F000662C25660D0A0000CDCCC742CDCCCC3D77
:1012000030BCBDE8C08F10B504464422002104F173
:101210003800F8F700FC002000F06AF810BD00006C
:1012200010B50A480A49096800F0100301229A40E3
:101230009143074A116000BF00BF032220214FF0F5
:101240009040F2F792FB00BF10BD000072004035E5
:101250000074004010B54FF6FF700B49088000BFC6
:10126000032220214FF09040F2F77FFB00BF074898
:101270000749096800F0100301229A401143044A0B
:10128000116000BF10BD000034B500207200403571
:1012900000740040FEB5044654F8F40FC56F206892
:1012A000D0F8806054F8F409D0F8847005200D4916
:1012B0004870084622F08CFA0B480C494FF07C52DB
:1012C000CDE90021029007483B4632462946D0F836
:1012D00004C0001DE04703480121026A001D904739
:1012E000FEBD0000100300100000C8420000C8C28C
:1012F00010B50446114800680078A04200D110BD26
:101300000E4800680078032806D16C2200210B48A3
:1013100000687C30F8F77FFB0848006800780128F7
:1013200006D144220021054800683830F8F773FBE5
:1013300002480068047000BFE1E7000020040020BC
:1013400070B50446002501210020FAF791FC0646FD
:10135000EFF733FA0546294604F1080014F023FAA2
:101360000646EFF766FAA08303210020FAF73AFC5D
:101370000646EFF722FA0546294604F1200014F04C
:1013800012FA0646EFF755FAA08670BD10B504466E
:1013900054F8F40F008A174908862068408A488666
:1013A0002068408808842068808848842068C08835
:1013B000888420680089C8842068807A81F83C018C
:1013C0002068C06FC1F8C4012068D0F88000C1F85F
:1013D000C8012068D0F88400C1F8D0012068B0F8B6
:1013E0006C00888354F8F409B0F87000C883FDF7E6
:1013F000D3FF10BD98710010F8B5054604220021F6
:101400006846F8F7CCFA2A460FA16846F6F73EFC84
:1014100000246846EEF724FFC6B200200FE01DF856
:101420000010302907DB392905DCA1F1300202EB7D
:101430000412D4B200E000E000BF411CC8B2B042C8
:10144000EDDB2046F8BD0000256400002DE9F043E7
:1014500003460C461746E000062190FBF1F01FFA08
:1014600080F8002045E000EB40094FEA49064FEACA
:10147000E67906EB5979C9F3C7055A5D6E1CA64299
:1014800001DA9E5D00E00026B446002106464FEAE0
:10149000E07900EB99794FEAA909A0EB8909B9F144
:1014A000000F09D0B9F1010F08D0B9F1020F0BD02C
:1014B000B9F1030F11D10DE091080EE09607B10EBE
:1014C00001EB1C16F1B208E01607B10E01EB9C16F9
:1014D000F1B202E002F03F0100BF00BF202902DAB2
:1014E00001F14006F1B2202900D100213954411CFC
:1014F00088B24045B7DBBDE8F0832DE9F04F99B0E5
:1015000005460E46144698460027582103A8EEF7D4
:1015100090FE5CB903AA3146284606F046F908B1A8
:1015200003AC03E0052019B000F068B8B8F1000F73
:101530000ED100200321CDE90010062302AA28467F
:10154000216DF7F73DFB0746012085F8A40027E051
:1015500001200421CDE90010062302AA2846216DAE
:10156000F7F72EFB074695F8A400B0B9AFB95EB106
:101570003046EEF775FE82464FF0FF335246314655
:1015800028462DF03FFB08E03CB1A2784FF0FF3336
:1015900004F1100128462DF035FB002085F8A40049
:1015A000206DE968B0FBF1F0484300F101091FBB71
:1015B000042302AA49462846F7F7D2FA01281BD18C
:1015C0000221042302AACDE9001049462846F7F774
:1015D000F7FA0746206DE968B0FBF1F000FB01FB6C
:1015E0005946284609F074F98246BAF1000F02D034
:1015F00002218AF8021000BF384694E730BCBDE8EB
:10160000C08F70B504460CB1012100E000210846EE
:1016100040F25921EFF744FE0025258900E000BF84
:10162000281EA5F101018DB2F9D170BD01490860F4
:10163000704700004403002070B504461E2094FB50
:10164000F0F594FBF0F100FB114604E047F2305056
:1016500000F012F86D1E002DF8D12EB14FF47A7102
:1016600006FB01F000F008F870BD00E000BF011EAD
:10167000A0F10100FAD1704770B5034600224FF087
:10168000E02675690D4E366803FB06F44FF0E02640
:10169000B16910E04FF0E026B06988420BD0884273
:1016A00002D20E1A324402E02E1A0E44324401468F
:1016B000A24200D300E0EDE700BF70BD440300206C
:1016C00004490978002904DD02490978491E014AC4
:1016D000117070478003002070B505460DB10121DF
:1016E00000E000210846E421EFF7DAFD002600249F
:1016F000C5B100212C4660892289904201D1002089
:1017000070BD22892379206802FB03012089401CD7
:1017100086B2E088B04202DCE088301A86B22681C8
:101720000846EDE70020EBE785B0002012E01E49F7
:10173000095C302907DB1C49095C392903DC1A499B
:10174000095C303902E01849095C373901AA1154A3
:10175000411CC8B21028EADB9DF80F009DF80E105E
:1017600040EA0110C0B28DF800009DF811009DF80C
:10177000101040EA0110C0B28DF801009DF813006E
:101780009DF8121040EA0110C0B28DF802009DF8D9
:10179000000000049DF8011040EA01209DF80210AD
:1017A000084305B070470000327200102DE9F04F79
:1017B000A9B0054608202890F948007D2790F948EF
:1017C000077DF1F75FF8064600EBD670C0F34700DF
:1017D000069027980F3000F0FF0805200590CDF8FF
:1017E000108028A9284614F0D9FC002017F006FE26
:1017F00005F1AC00002870D0002617E2A87906EBAE
:10180000C000E949088028880988884274DD05F10C
:10181000AC00E549098850F8210090F800B040225A
:10182000002117A8F8F7D9F8F0F752FC00FB068161
:10183000059800FB0610C0B20490BBF1210F73D2D3
:10184000DFE80BF0112699F2F1F0EFEE444C535B18
:101850006269737C8B9285B0BFCFDEFCECEBEAE96A
:10186000E8E7E6E5E400D14890F8340110B101283A
:1018700004D101E02A2403E02B2401E02A2400BF44
:1018800000BFCB4800EBC40117A814F0AFFEC4E1C1
:10189000C64890F8370106280ED2DFE800F0030DA5
:1018A0000507090B2C2409E02D2407E02E2405E070
:1018B0002F2403E0302401E02C2400BF00BFBC48EB
:1018C00000EBC40117A814F091FEA6E1B948827894
:1018D000B9A117A8F6F7DAF99FE1ACE10522B549FD
:1018E000C91C17A80CF06EFE97E117AA1021AF488B
:1018F0008A30FBF74CFA90E196E117AA1021AB4829
:101900009A30FBF744FA88E117AA1021A748AA30B9
:10191000FBF73DFA81E11B24A54800EBC4012246F8
:1019200017A814F00FF978E176E11C24A04800EB29
:10193000C401224617A814F005F96EE11D249C4845
:1019400000EBC401224617A814F0FCF865E102225E
:1019500099A117A8F6F79AF95FE19448027896A141
:1019600017A8F6F793F958E19048427892A117A882
:10197000F6F78CF951E18D48C08AA0F566403F38F2
:1019800010B1012804D101E0312403E0322401E048
:10199000312400BF00BF864800EBC40117A814F033
:1019A00025FE3AE181488079012801D1022000E03A
:1019B000032004467E4800EBC40117A814F016FE6D
:1019C0002BE17A4890F83E01012801D1022000E085
:1019D00003200446764800EBC40117A814F006FE65
:1019E0001BE17248407A012801D1022000E0032067
:1019F00004466F4800EBC40117A814F0F7FD0CE192
:101A00006A48807A012810D102200FE0F2E0E0E07D
:101A1000BEE05DE04CE03BE029E019E013E00DE0C2
:101A2000AEE09BE07EE06FE060E0032004466048AB
:101A300000EBC40117A814F0D9FDEEE0002117A8AF
:101A4000FEF70CFAE9E0012117A8FEF707FAE4E037
:101A5000564890F83C0108B9042000E005200446EF
:101A6000534800EBC40117A814F0C0FDD5E04F485F
:101A700090F83101C0F3800008B9062000E007208B
:101A800004464B4800EBC40117A814F0AFFDC4E0B6
:101A9000464890F83101C00908B9082000E0092043
:101AA0000446434800EBC40117A814F09FFDB4E0BE
:101AB0003E4890F83801012801D10A2000E00B20AF
:101AC00004463B4800EBC40117A814F08FFDA4E0C6
:101AD000364890F8310100F0030000F10C0434485E
:101AE00000EBC40117A814F081FD96E02F48C07ADE
:101AF00008B9122000E0132004462D4800EBC40171
:101B000017A814F073FD88E02848007B08B914205A
:101B100000E015200446264800EBC40117A814F085
:101B200065FD7AE02148807860B1012804D0022860
:101B300004D0032808D103E0172407E0182405E0A7
:101B4000192403E0162401E0162400BF00BF184842
:101B500000EBC40117A814F049FD5EE000200190DD
:101B60001FF028FA406900908047019001981E30CC
:101B7000C4B20F4800EBC40117A814F037FD4CE0C5
:101B80001A240B4800EBC40117A814F02FFD44E001
:101B90000A48019001980078012811D1222010E014
:101BA00028980408F0470408E40300209871001006
:101BB00010F3040820130010256400007474001052
:101BC000232004464B4800EBC40117A814F00EFD77
:101BD00023E04948019001980078012801D1222092
:101BE00000E023200446434800EBC40117A814F08A
:101BF000FDFC12E0404870380190019800780128FF
